:100000000C94B11A0C94E21A0C94E21A0C94E21AB1
:100010000C94E21A0C94E21A0C94E21A0C94E21A70
:100020000C94E21A0C94E21A0C94E21A0C94E21A60
:100030000C94E21A0C94E21A0C94E21A0C94E21A50
:100040000C94E21A0C949ED10C94E21A0C94E21ACD
:100050000C94E21A0C94E21A0C949BBE0C943BAAEA
:100060000C94E21A0C946B560C9461560C94E21AA0
:100070000C94E21A0C94E21A0C94E21A0C94E21A10
:100080000C9451340C94E21A0C94E21A0C94E21A77
:100090000C94E21A0C94E21A0C94E21A0C94E21AF0
:1000A0000C94E21A0C94E21A0C9423340C94E21A85
:1000B0000C94E21A0C94E21A0C94E21A0C94E21AD0
:1000C0000C94E21A0C94E21A0C94E21A0C945F3726
:1000D0000C9429370C94E21A0C94E21A0C94E21A4C
:1000E0000C94E21A084AD73B3BCE016E84BCBFFD9C
:1000F000C12F3D6C74319ABD56833DDA3D00C77FF8
:1001000011BED9E4BB4C3E916BAAAABE0000008090
:100110003F05A84CCDB2D44EB93836A9020C50B91F
:10012000918688083CA6AAAA2ABE000000803F004B
:100130000C9419FD0C94ADA40C9418FC0C94AB42D7
:100140000C9434FC0C94BAFC0C940FA90C941CFC79
:100150000C9430FC0C94A7420D9434010C94155768
:100160000C942F570C949F440C9403FC0D94980B03
:100170000C94E7560C9458420C94F9370C9442FCBA
:100180000D945F010D947A1F0C948CFC0C947FFCF1
:100190000C9438FC0C944EA90C940FFD0C943EFC6E
:1001A0000D946D0C0D94C10B0D94AD0F0C94F137A3
:1001B0000C949D370C9409570D94F80B0C9401572F
:1001C0000D94660F0C9412FC0C94B2FC0C9411A8C4
:1001D0000C9422FC0D94800C0C9405380D940C0C9E
:1001E0000D9494090C94F1FC0C94EA370C94D8FC0F
:1001F0000C9407FC0C94A0FC0D94DB030D945C059F
:100200000D9440140D9469110C9491A80C9430A590
:100210000D94FF070C94F5370C940FFC0C9420FF01
:100220000C94F1FB0C94FD560D94BA0F0D94640AD6
:100230000C9473440D942F0D0D94810F0D94780937
:100240000C9421A90C94E0440D94390F0D944A00AC
:100250000C94ECFB0C94CC370D9496100D94690F14
:100260000C9401380C9405570C9423380D94981F66
:100270000C9476A80D94D50B0D94CA020D94C80960
:100280000D94A6100C9418AA0C942FA50C94115739
:100290000C9418450C94FD370C9432A80D948F0FD4
:1002A0000D942A0B0C94AAFC0D94990F0D944509FA
:1002B0000C94E7FC0C9427570C9426FC0C941C57C8
:1002C0000C94C4FC0C9487FC0D942B0C0C940938F2
:1002D0000C94FBFC0D94F40A0C94D8560D94600F0A
:1002E0000C947CA70C94A9560C9410380C9405FD22
:1002F0000C940D570C94CEFC0C94F6560C941B38B1
:100300000C9499A70C94DB370C942AFC0C9496FC63
:100310000C940BFC4E414E494E495459494E46CD22
:10032000CCCC3D0AD7233C17B7D13877CC2B3295AC
:1003300095E6241FB14F0A000020410000C842008A
:10034000401C4620BCBE4CCA1B0E5AAEC59D740054
:10035000407A10F35A00A0724E18090010A5D4E894
:100360000000E87648170000E40B54020000CA9A27
:100370003B000000E1F50500008096980000004079
:10038000420F000000A086010000001027000000BE
:1003900000E803000000006400000000000A000004
:1003A0000000000100000000002C76D888DC674FB8
:1003B0000823DFC1DFAE59E1B1B796E5E3E453C6E8
:1003C0003AE651997696E8E6C28426EB898C9B62E0
:1003D000ED407C6FFCEFBC9C9F40F2BAA56FA5F48A
:1003E00090055A2AF75C936B6CF9676DC11BFCE0B2
:1003F000E40D47FEF520E6B500D0ED902E03009405
:100400003577050080841E080000204E0A00000099
:10041000C80C333333330F986E12831141EF8D21A3
:1004200014893BE65516CFFEE6DB18D1844B381B0A
:10043000F77C1D901DA4BBE424203284725E2281CF
:1004400000C9F124ECA1E53D27434F4D4D554E49E0
:10045000434154494F4E0044525952554E00455263
:10046000524F525300494E464F004543484F0045B6
:1004700072726F722077726974696E6720746F2070
:10048000454550524F4D210A0053544F505045445A
:100490002E20005072696E7465722073746F7070D4
:1004A00065642064756520746F206572726F727365
:1004B0002E2046697820746865206572726F7220FC
:1004C000616E6420757365204D39393920746F2051
:1004D000726573746172742E202854656D70657234
:1004E00061747572652069732072657365742E205E
:1004F0005365742069742061667465722072657337
:1005000074617274696E67290A004E6F20436865D2
:10051000636B73756D2077697468206C696E6520F4
:100520006E756D6265722C204C617374204C696E1F
:10053000653A20004E6F20436865636B73756D20CC
:1005400077697468206C696E65206E756D6265727E
:100550002C204C617374204C696E653A20006368EE
:1005600065636B73756D206D69736D617463682C61
:10057000204C617374204C696E653A20004C696EA2
:1005800065204E756D626572206973206E6F7420F0
:100590004C617374204C696E65204E756D62657296
:1005A0002B312C204C617374204C696E653A20000D
:1005B0004D3131300053657269616C207374617420
:1005C0007573206D69736D617463680A0077616982
:1005D000740A0053442072656164206572726F7200
:1005E0000A002121204B494C4C20636175736564DE
:1005F00020627920746F6F206D75636820696E6169
:1006000063746976652074696D65202D2063757249
:1006100072656E7420636F6D6D616E643A20004880
:100620006F74656E642049646C652054696D656FF4
:10063000757400486F74656E642049646C6520545D
:10064000696D656F75740A003D3D6F6E46696C613A
:100650006D656E7452756E6F75743D3D0070617599
:100660007365004D363030002066696C616D656ED3
:10067000745F72756E6F7574200066696C616D656C
:100680006E745F72756E6F757420540046696C618C
:100690006D656E7452756E6F75742054002A2A2A27
:1006A000496E6974696E67206361726420697320A2
:1006B0004F4B2A2A2A004D6564696120496E736593
:1006C00072746564004D656469612052656D6F7672
:1006D0006564004D313030305300627573793A20D3
:1006E00070617573656420666F7220696E707574D1
:1006F0000A00627573793A207061757365642066CB
:100700006F7220757365720A00627573793A207092
:10071000726F63657373696E670A002A2A2A6B69B0
:100720006C6C2A2A2A00706F7765726F6666004BC0
:10073000494C4C45442E20005072696E74657220FD
:1007400068616C7465642E206B696C6C2829206369
:10075000616C6C6564210A0053544F505045442E1F
:1007600020005072696E7465722073746F707065CA
:10077000642064756520746F206572726F72732EC9
:100780002046697820746865206572726F722061F6
:100790006E6420757365204D39393920746F20726D
:1007A0006573746172742E202854656D7065726172
:1007B000747572652069732072657365742E205399
:1007C0006574206974206166746572207265737443
:1007D000617274696E67290A006563686F3A004543
:1007E00072726F723A0042696C696E656172204C78
:1007F0006576656C696E6720477269643A0A002104
:10080000212053544F502063616C6C6564206265F5
:100810006361757365206F6620424C546F75636821
:10082000206572726F72202D20726573746172740C
:100830002077697468204D3939390A002121205305
:10084000544F502063616C6C656420626563617510
:100850007365206F6620424C546F75636820657223
:10086000726F72202D2072657374617274207769C3
:100870007468204D3939390A002F2F616374696F0C
:100880006E3A0070726F6D70745F00656E64005335
:10089000656E64204D31303820746F207265737539
:1008A0006D650A00496E736572742066696C616DCE
:1008B000656E7420616E642073656E64204D313006
:1008C000380A005265686561742066696E697368EC
:1008D00065642E0052656865617420446F6E650022
:1008E000526568656174696E672E2E2E00526568C8
:1008F000656174004865617465722054696D656F47
:1009000075740053656E64204D31303820746F204B
:1009100068656174206E6F7A7A6C650A004E6F7A32
:100920007A6C65205061726B656400486F74656E07
:100930006420746F6F20636F6C640A00706175735C
:1009400065640050617573650044697361626C652C
:1009500052756E6F75740050757267654D6F726574
:10096000005061757365640073686F770062757419
:10097000746F6E00626567696E004C6F616420463B
:10098000696C616D656E74004C6F61642046696CC2
:10099000616D656E74205400496E736572742066D3
:1009A000696C616D656E7420616E642073656E6440
:1009B000204D3130380A00726573756D65640052E0
:1009C0006573756D696E670057616974696E67203C
:1009D000666F72206865617475702E0A004C6561DF
:1009E00076696E6720473236003F537065636966EB
:1009F00069656420582C5920636F6F7264696E6159
:100A00007465206F7574206F6620626F756E6473F5
:100A10002E0A003F28522965706561742076616C4A
:100A20007565206E6F7420706C61757369626C659A
:100A30003B206D757374206265206174206C656164
:100A4000737420312E0A003F285229657065617445
:100A5000206D7573742062652073706563696669C3
:100A60006564207768656E206E6F74207573696E9B
:100A70006720616E204C43442E0A003F537065632B
:100A80006966696564206E6F7A7A6C652074656D3D
:100A90007065726174757265206E6F7420706C6120
:100AA000757369626C652E0A003F537065636966F1
:100AB0006965642066696C616D656E742073697A1E
:100AC00065206E6F7420706C61757369626C652E41
:100AD0000A003F53706563696669656420707269D6
:100AE0006D65206C656E677468206E6F7420706C25
:100AF00061757369626C652E0A003F5072696D659D
:100B0000206C656E677468206D7573742062652053
:100B1000737065636966696564207768656E206EC9
:100B20006F74207573696E6720616E204C43442E8C
:100B30000A003F537065636966696564206E6F7A69
:100B40007A6C652073697A65206E6F7420706C61B1
:100B5000757369626C652E0A003F52657472616339
:100B600074696F6E204D756C7469706C6965722064
:100B70006D7573742062652073706563696669655D
:100B8000642E0A003F53706563696669656420528C
:100B9000657472616374696F6E204D756C746970F1
:100BA0006C696572206E6F7420706C617573696218
:100BB0006C652E0A003F5370656369666965642041
:100BC0006C6179657220686569676874206E6F74FE
:100BD00020706C61757369626C652E0A0043292E62
:100BE0000A003F53706563696669656420626564E5
:100BF0002074656D7065726174757265206E6F74B6
:100C000020706C61757369626C65202834302D002A
:100C1000473236207374617274696E672E2E2E0A05
:100C2000004F46460A00466164652048656967686A
:100C3000742000426564204C6576656C696E67209F
:100C4000004661696C656420746F20656E61626C3A
:100C50006520426564204C6576656C696E670A00A4
:100C6000496E76616C6964206D6573682E0A005068
:100C7000726F62696E6720506F696E740025532031
:100C800025692F2569002E0A002F0050726F6269B6
:100C90006E67206D65736820706F696E7420002028
:100CA0002844525952554E29004732392041757413
:100CB0006F20426564204C6576656C696E67003F05
:100CC00020284C2C522C462C4229206F7574206F02
:100CD0006620626F756E64732E0A003F2856296580
:100CE00072626F7365206C6576656C20696D706CDF
:100CF00061757369626C652028302D34292E0A00D5
:100D0000426164205A2076616C75650A004E6F203E
:100D100062696C696E65617220677269640A004479
:100D20006576696174696F6E0025533A20257300FA
:100D300046696E6973686564210A003A207A3A2030
:100D400000206F662000476F696E6720746F3A203D
:100D5000580043570A00206469723A0020616E67A8
:100D60006C653A00537461727420726164697573C2
:100D70003A004D343820506F696E740025533A2084
:100D800025642F256400506F736974696F6E696EF6
:100D900067207468652070726F62652E2E2E0A00BF
:100DA0003F4C656773206F66206D6F76656D656E6D
:100DB0007420696D706C61757369626C6520283090
:100DC0002D3135292E0A003F2028582C5929206F13
:100DD0007574206F6620626F756E64732E0A005002
:100DE000726F6265206F7574206F6620626F756E1A
:100DF0006473003F53616D706C652073697A652080
:100E00006E6F7420706C61757369626C6520283434
:100E10002D3530292E0A004D3438205A2D50726F4E
:100E20006265205265706561746162696C6974798C
:100E300020546573740A003F2856296572626F73E7
:100E400065206C6576656C20696D706C6175736981
:100E5000626C652028302D34292E0A005374616E8F
:100E60006461726420446576696174696F6E3A20CA
:100E7000002052616E67653A2000204D61783A206B
:100E800000204D696E3A2000205369676D613A2059
:100E9000004D65616E3A20005741524E494E472140
:100EA000204C6F77205A204A65726B206D61792043
:100EB0006C65616420746F20756E77616E74656413
:100EC000207061757365732E0A004F4646004F4EC1
:100ED0000020204D61783A2000200020204D696ECE
:100EE0003A2000536F667420656E6473746F70737C
:100EF0003A20003D3D4F6E506F7765724C6F7373B3
:100F0000526573756D653D3D004D32342053256C3F
:100F1000642054256C64004739322E3920452573EE
:100F200000473120462564004739322E39205A25A2
:100F300073004731205A302046323030004731208C
:100F400058257320592573204633303030004D34F6
:100F5000323020532569205A2573004D3130362018
:100F600050256920532569004D32303020442573C7
:100F70000047323852305859004739322E3920450F
:100F800030205A300A47315A2573004D313039200C
:100F9000532569004D31393020532569004D3432D5
:100FA00030205330205A300020496E76616C6964DD
:100FB000206578747275646572200047322F47335C
:100FC0002062616420706172616D65746572730A7C
:100FD00000536C6565702E2E2E005A2050726F6281
:100FE000652050617374204265640A005A20507273
:100FF0006F62652050617374204265640047323827
:101000004C30004D3131372050726F62652066617F
:10101000696C65642E0A4732380A0070726F626527
:101020005F72657769706500473239205265747266
:1010300079696E670050726F62696E6720466169F8
:101040006C6564004D31313720426564206C6576F3
:10105000656C696E67206661696C65642E0A47304D
:10106000205A31300A4D3330302050323520533839
:1010700038300A4D333030205035302053300A4D4F
:101080003330302050323520533838300A4D333029
:1010900030205035302053300A4D3330302050321C
:1010A0003520533838300A4D333030205035302019
:1010B00053300A47342053310070726F62655F66A7
:1010C00061696C6564004D31313720426564206C84
:1010D0006576656C696E6720646F6E652E00205AB8
:1010E0003A200020593A200042656420583A2000F6
:1010F0004D65736820706F696E74206F7574206F12
:10110000662072616E67650A004D302053746F70FF
:10111000004D312053746F7000436F6E74696E75AB
:101120006500436C69636B20746F20526573756D45
:10113000652E2E2E004E6F204D6F76652E00456E6B
:10114000642066696C65206C6973740A0042656787
:10115000696E2066696C65206C6973740A004E6F55
:10116000206D656469610A00526573756D696E670B
:1011700020534400286E6F2066696C652900437512
:101180007272656E742066696C653A2000507269EF
:101190006E742074696D653A20000A53746174732B
:1011A0003A2046696C616D656E7420757365643AAA
:1011B00020002C204C6F6E67657374206A6F623A52
:1011C0002000546F74616C2074696D653A2000537F
:1011D000746174733A20002C204661696C65643A2E
:1011E00020002C2046696E69736865643A200050BF
:1011F00072696E74733A200053746174733A2000FC
:10120000436F6F6C696E672E2E2E0048656174699E
:101210006E672E2E2E0045202553006F6B006F66E3
:1012200066006A0465045E04570449044445425557
:10123000473A004D31313320530042656420436FFB
:101240006F6C696E672E2E2E0042656420486561C2
:1012500074696E672E2E2E00544D33442045352080
:10126000506C7573204F46462E002F2F00205200E1
:10127000416363656C65726174696F6E3A205000FA
:101280004D32303620580046523A0020466C6F7777
:101290003A20003A200020536572766F2000206FBC
:1012A0007574206F662072616E67650A00536572FF
:1012B000766F200020643A0020693A0020703A00DE
:1012C000496E76616C6964206578747275646572C4
:1012D0000A0020643A0020693A0020703A006469EC
:1012E0007300656E0043290A0061626C6564202802
:1012F0006D696E2074656D702000436F6C642065AD
:101300007874727564657320617265200050494479
:10131000204175746F74756E6500504944204175A5
:10132000746F74756E65206661696C656421204216
:101330006164206865617465722069640A004669A9
:101340006C616D656E742072756E6F757420646962
:101350007374616E636520286D6D293A20004669BB
:101360006C616D656E742072756E6F757420004DC2
:1013700034323120696E636F7272656374207061FC
:1013800072616D657465722075736167650A004DE1
:1013900065736820706F696E74206F7574206F6656
:1013A0002072616E67650A004F666673657473200C
:1013B0004170706C696564004572723A20546F6FB9
:1013C000206661722100546F6F2066617220667220
:1013D0006F6D207265666572656E636520706F69FA
:1013E0006E740A00454550524F4D204F4B0A005035
:1013F0006F7765722D6C6F7373207265636F76659E
:10140000727920004D383400446F6E652070726927
:101410006E74696E672066696C650A004D37370027
:101420004D3331004361703A004D454154504143C2
:101430004B00434F4F4C45525F54454D5045524130
:1014400054555245004348414D4245525F54454D25
:10145000504552415455524500424142595354451A
:101460005050494E470041524353004D4F54494F4D
:101470004E5F4D4F44455300544845524D414C5FDB
:1014800050524F54454354494F4E004C4F4E475FC6
:1014900046494C454E414D45004155544F524550EB
:1014A0004F52545F53445F53544154555300534477
:1014B0005F575249544500524550454154005344EA
:1014C000434152440050524F4D50545F5355505079
:1014D0004F525400454D455247454E43595F504188
:1014E0005253455200434153455F4C494748545F6E
:1014F0004252494748544E45535300544F47474C76
:10150000455F4C494748545300534F465457415246
:10151000455F504F574552004255494C445F504536
:101520005243454E54004C4556454C494E475F4446
:10153000415441005A5F50524F42450052554E4F60
:101540005554004155544F4C4556454C0050524956
:101550004E545F4A4F420050524F4752455353003A
:101560004155544F5245504F52545F54454D5000D1
:10157000564F4C554D455452494300454550524FE6
:101580004D0042494E4152595F46494C455F5452C5
:10159000414E534645520053455249414C5F584FC6
:1015A0004E5F584F4646004649524D574152455F9F
:1015B0004E414D453A4D61726C696E20322E302E8F
:1015C000375F4457372E332E3120544D3344204556
:1015D0003550534D44424220284170722032392008
:1015E000323032312031333A34383A3030292053D6
:1015F0004F555243455F434F44455F55524C3A68FF
:10160000747470733A2F2F6769746875622E636FF4
:101610006D2F496E73616E6974794175746F6D6178
:1016200074696F6E2F4D61726C696E2F747265658F
:101630002F437265616C6974794477696E5F322EED
:10164000302050524F544F434F4C5F5645525349F0
:101650004F4E3A312E30204D414348494E455F545C
:101660005950453A544D334420453520506C7573DC
:101670002045585452554445525F434F554E543AB5
:101680003120555549443A63656465326132662DAF
:10169000343161322D343734382D396231322D6393
:1016A00035356336326633363766660A0050726FF8
:1016B0006265204F6666736574205A0050726F62CF
:1016C00065204F6666736574205A00290A002074ED
:1016D0006F20003F5A206F7574206F662072616E14
:1016E0006765202800290A0020746F20003F5920D8
:1016F0006F7574206F662072616E676520282D00FB
:10170000290A0020746F20003F58206F7574206FE5
:10171000662072616E676520282D0050726F6265C9
:10172000204F666673657420580043616E6E6F7457
:10173000206F70656E207375626469722000256980
:10174000730025696D202569730025696820256966
:101750006D20256973002569642025696820256945
:101760006D20256973002569792025696420256924
:10177000682025696D20256973003D3D4477696EB9
:1017800020496E697420436F6D706C6574653D3DD2
:10179000002A2A2A4E6F7A7A6C6554656D705374EC
:1017A000617475735B325D203D003D3D4865617439
:1017B000696E6720446F6E65204368616E676520BF
:1017C00046696C616D656E743D3D002020737461E7
:1017D000727470726F677265737320003D3D77613C
:1017E000697477617920353D3D003D3D77616974CD
:1017F00077617920343D3D003D3D776169747761C3
:101800007920333D3D003D3D7761697477617920F2
:10181000313D3D003D3D6F6E5072696E7454696D8F
:10182000657253746F707065643D3D003D3D6F6E31
:10183000466163746F727952657365743D3D00272C
:101840000A0A0000272027002027002D006E6F7451
:10185000696669636174696F6E200063616E6365B8
:101860006C005072696E742041626F72746564001E
:101870004469736D6973730055492041626F7274D6
:10188000656400726573756D65004D3234002A2AF7
:101890002A43506C617920546F6E652A2A2A003DD4
:1018A0003D6F6E5072696E7454696D6572506175EA
:1018B0007365643D3D00486F6D696E6720466169E0
:1018C0006C6564006F70656E00545249474745521D
:1018D0004544003A200066696C616D656E74007A5B
:1018E0005F6D696E00795F6D617800785F6D61781A
:1018F000005265706F7274696E6720656E647374F0
:101900006F70207374617475730A0020746F6F2098
:101910006C6F6E6720657874727573696F6E207076
:10192000726576656E7465640A0020636F6C64206E
:10193000657874727573696F6E2070726576656E06
:101940007465640A00486F6D6520257325732573DF
:10195000204669727374005761726E696E673A202F
:10196000486F6D696E672042756D702044697669B5
:10197000736F72203C20310A000202040000B4435D
:101980000000B443000000000000B4430000B44372
:101990000000C8430000004100000041000000407A
:1019A0000101FF000000010000000100008000555F
:1019B0005555000000400033333300AAAA2A0049DD
:1019C00092240000002000C7711C0099991900D1D1
:1019D000451700555515003BB1130024491200115D
:1019E000111100000010000F0F0F00E3380E00432C
:1019F000790D00CCCC0C00C3300C00E8A20B0064C5
:101A0000210B00AAAA0A00703D0A009DD8090042D5
:101A10007B090092240900DCD308008888080010A4
:101A200042080000000800F0C10700878707007522
:101A3000500700711C07003EEB0600A1BC060069C0
:101A400090060066660600703E06006118060017E4
:101A5000F4050074D105005BB00500B2900500628A
:101A60007205005555050078390500B81E050005BA
:101A70000505004EEC040087D40400A1BD040090CD
:101A8000A7040049920400C17D0400EE690400C768
:101A9000560400444404005C320400082104004160
:101AA000100400000004003FF00300F8E0030026EB
:101AB000D20300C3C30300CCB503003AA803000A55
:101AC0009B0300388E0300C08103009F750300D084
:101AD000690300505E03001D530300344803009166
:101AE0003D03003333030016290300381F0300971A
:101AF000150300300C0300030303000BFA02004936
:101B0000F10200BAE802005CE002002DD802002DCC
:101B1000D0020059C80200B0C0020031B90200DA98
:101B2000B10200AAAA0200A0A30200BC9C0200FA13
:101B30009502005C8F0200DF88020082820200456D
:101B40007C02002776020027700200436A02007CB4
:101B5000640200D05E02003F590200C8530200FF39
:101B6000FDFCFAF8F6F4F2F0EEECEAE9E7E5E3E181
:101B7000E0DEDCDAD9D7D5D4D2D0CFCDCBCAC8C736
:101B8000C5C3C2C0BFBDBCBAB9B7B6B4B3B2B0AFBB
:101B9000ADACAAA9A8A6A5A4A2A1A09E9D9C9A9915
:101BA000989795949392908F8E8D8B8A898887864B
:101BB00084838281807F7E7D7B7A79787776757465
:101BC000737271706F6E6D6C6B6A6968676665645D
:101BD000636261605F5E5D5C5B5A59585857565549
:101BE0005453525150504F4E4D4C4B4A4A4948471E
:101BF0004646454443424241403F3E3E3D3C3B3BDE
:101C00003A39383837363535343332323130302F8F
:101C10002E2E2D2C2B2B2A29292827272625252433
:101C2000232322212120201F1E1E1D1C1C1B1B1ACA
:101C30001919181817161615151413131212111155
:101C4000100F0F0E0E0D0D0C0C0B0A0A09090808D7
:101C50000707060605050404030302020100003D10
:101C60003D6F6E5072696E7454696D657253746124
:101C7000727465643D3D000000B4430000B443004D
:101C800000C8430000000000000000000000003D0C
:101C90003D6F6E53746F726553657474696E6773CC
:101CA0003D3D003D3D6F6E436F6E666967757261C5
:101CB00074696F6E53746F72655772697474656E70
:101CC0003D3D0053657474696E67732053746F7281
:101CD0006564000A20696E6974207A70726F6265AB
:101CE0005F7A6F6666736574203D20003D3D6F6EC0
:101CF000436F6E66696775726174696F6E53746F56
:101D00007265526561643D3D00454550524F4D201E
:101D1000496E697469616C697A65640A003B2000E8
:101D20003A0A0020204D3630332000204400202085
:101D30004D34313220530046696C616D656E7420FC
:101D400072756E6F75742073656E736F723A0020D2
:101D500055004C0046696C616D656E74206C6F6156
:101D6000642F756E6C6F6164206C656E6774687348
:101D70003A0020204D3835312058005A2D50726FCE
:101D80006265204F66667365740020204D343133E0
:101D9000205300506F7765722D4C6F73732052651E
:101DA000636F766572793A00204400204900202054
:101DB0004D33303420500020440020490020204D75
:101DC0003330312050005049442073657474696E7B
:101DD00067733A00204A00202047323920572049B3
:101DE0000020204D3432302053004175746F204262
:101DF0006564204C6576656C696E673A0020204DFD
:101E0000323036205800486F6D65206F6666736506
:101E1000743A0020580020530020204D32303520E5
:101E20004200416476616E6365643A20423C6D69AC
:101E30006E5F7365676D656E745F74696D655F7500
:101E4000733E20533C6D696E5F66656564726174B4
:101E5000653E20543C6D696E5F74726176656C5F9F
:101E600066656564726174653E20583C6D61785F9B
:101E7000785F6A65726B3E20593C6D61785F795F6F
:101E80006A65726B3E205A3C6D61785F7A5F6A6565
:101E9000726B3E20453C6D61785F655F6A65726B71
:101EA0003E0020540020520020204D32303420507B
:101EB00000416363656C65726174696F6E2028759B
:101EC0006E6974732F7332293A20503C7072696EB8
:101ED000745F616363656C3E20523C72657472612D
:101EE00063745F616363656C3E20543C7472617619
:101EF000656C5F616363656C3E0020204D3230315C
:101F00002058004D6178696D756D20416363656C83
:101F100065726174696F6E2028756E6974732F73B2
:101F200032293A0020204D3230332058004D61785C
:101F3000696D756D206665656472617465732028CE
:101F4000756E6974732F73293A005374657073202A
:101F500070657220756E69743A0020440020204D2F
:101F60003230302053002044697361626C65640A2A
:101F70000046696C616D656E742073657474696E7A
:101F800067733A0020286D6D2900202047323120E8
:101F90002020203B20556E69747320696E206D6D82
:101FA000003D3D6F6E4C6F616453657474696E677C
:101FB000733D3D0000803B4400803B4400002041D5
:101FC000000096420000A0420000A04200004844E9
:101FD0000000BE42D0070000D007000064000000EF
:101FE0004B00000024F4D43050C38E20C2A240170E
:101FF000828B7011127A910D816CD90AA861E10867
:10200000C7586607615143061E4B5D05C145A704CD
:102010001A411104093D9803713931034036DB023E
:1020200065339102D4305402802E1D02632CEE01E0
:10203000752AC501B028A001102781018F256401F0
:102040002B244B01E0223401AC211F018D200D0116
:10205000801FFC00841EED00971DDF00B81CD2001D
:10206000E61BC600201BBC00641AB200B219A8000F
:102070000A19A0006A189900D117910040178B0027
:10208000B516840031167E00B31579003A15730039
:10209000C7146F0058146A00EE13660088136300BB
:1020A00025135E00C7125B006C1257001512540016
:1020B000C111510070114F0021114B00D610490081
:1020C0008D1047004610440002104200C00F40002F
:1020D000800F3E00420F3C00060F3B00CB0E380045
:1020E000930E37005C0E3500270E3400F30D3200DE
:1020F000C10D3100900D3000600D2E00320D2D000D
:10210000050D2C00D90C2B00AE0C2900850C2900E4
:102110005C0C2700350C27000E0C2600E80B240071
:10212000C40B2400A00B23007D0B23005A0B2100BD
:10213000390B2100180B2000F80A1F00D90A1E00D5
:10214000BB0A1E009D0A1D00800A1D00630A1C00B8
:10215000470A1B002C0A1B00110A1A00F7091A0073
:10216000DD091900C4091900AB091900920917000B
:102170007B091800630917004C0916003609160080
:10218000200916000A091500F5081500E0081400DA
:10219000CC081400B8081400A40814009008130018
:1021A0007D0812006B081300580812004608120040
:1021B0003408110023081100120811000108110051
:1021C000F0071000E0071000D0071000C007100053
:1021D000B0070F00A107100091070E0083070F0042
:1021E00074070F0065070E0057070E0049070E0021
:1021F0003B070D002E070E0020070D0013070D00F2
:1022000006070D00F9060C00ED060D00E0060C00B7
:10221000D4060C00C8060C00BC060C00B0060C006E
:10222000A4060B0099060C008D060B0082060B001D
:1022300077060B006C060B0061060A0057060B00C0
:102240004C060A0042060A0038060A002E060A005A
:1022500024060A001A060A001006090007060A00EA
:10226000FD050900F4050900EB050900E205090078
:10227000D9050900D0050900C7050900BE050900F8
:10228000B5050800AD050800A50509009C05080076
:10229000940508008C050800840508007C050800EA
:1022A000740508006C050700650508005D0507005A
:1022B000560508004E0507004705070040050800C1
:1022C00038050700310507002A0507002305070028
:1022D0001C050600160507000F0507000805060087
:1022E00002050700FB040600F5040700EE040600E3
:1022F000E8040600E2040700DB040600D50406003B
:10230000CF040600C9040600C3040600BD0406008D
:10231000B7040600B1040500AC040600A6040600DC
:10232000A00405009B040600950405009004060027
:102330008A04050085040500800406007A0405006F
:1023400075040500700405006B04050066040500B3
:10235000610405005C0405005704050052040500F3
:102360004D04050048040500430405003E04040034
:102370003A04050035040500300404002C0405006F
:1023800027040400230405001E0404001A040400AA
:1023900016040500110404000D04040009040500DE
:1023A0000404040000040400FC030400F803040017
:1023B000F4030400F0030400EC030400E803040049
:1023C000E4030400E0030400DC030400D803040079
:1023D000D4030400D0030400CC030400C8030300AA
:1023E000C503030024F404D9201BC40C5C0E98041C
:1023F000C4095F0265077101F405F900FB04B3002D
:1024000048048700C10369005803550003034500D1
:10241000BE023A008402310053022A00290225003C
:1024200004022000E4011C00C8011900AF011700DC
:102430009801140084011300710110006101100063
:1024400051010E0043010D0036010B002B010B0062
:1024500020010B00150109000C010900030108000F
:10246000FB000800F3000800EB000700E400060092
:10247000DE000600D8000600D2000600CC000500F1
:10248000C7000500C2000500BD000400B90004003B
:10249000B5000400B1000400AD000400A900040070
:1024A000A5000300A20003009F0004009B0003009E
:1024B00098000300950002009300030090000300C1
:1024C0008D0002008B0003008800020086000200DD
:1024D00084000300810002007F0002007D000200F2
:1024E0007B00020079000200770001007600020004
:1024F0007400020072000100710002006F0002000F
:102500006D0001006C0002006A0001006900020019
:102510006700010066000100650001006400020020
:102520006200010061000100600001005F00020024
:102530005D0001005C0001005B0001005A00010029
:102540005900010058000100570001005600010029
:102550005500010054000100530000005300010029
:102560005200010051000100500001004F00010025
:102570004E0000004E0001004D0001004C00010023
:102580004B0000004B0001004A000100490001001F
:10259000480000004800010047000100460000001C
:1025A0004600010045000000450001004400010014
:1025B000430000004300010042000000420001000F
:1025C0004100000041000100400001003F00000008
:1025D0003F0001003E0000003E0001003D00000001
:1025E0003D0001003C0000003C0000003C000100F8
:1025F0003B0000003B0001003A0000003A000100EF
:1026000039000000390001003800000038000000E7
:1026100038000100370000003700010036000000DC
:1026200036000000360001003500000035000000D3
:1026300035000100340000003400000034000100C7
:1026400033000000330000003300010032000000BE
:1026500032000000320001003100000031000000B3
:1026600031000100300000003000000030000100A7
:102670002F0000002F0000002F0000002F0001009D
:102680002E0000002E0000002E0001002D00000092
:102690002D0000002D0000002D0001002C00000086
:1026A0002C0000002C0000002C0001002B0000007A
:1026B0002B0000002B0000002B0001002A0000006E
:1026C0002A0000002A0000002A0001002900000062
:1026D0002900000029000000290000002900010055
:1026E000280000002800000028000000280000004A
:1026F000280001002700000027000000270000003C
:10270000270000002700010026000000260000002E
:102710002600000026000000260001002500000021
:102720002500000025000000250000002500000015
:102730002500010024000000240000002400000007
:1027400024000000240001002300000023000000FA
:1027500023000000230000002300000023000000ED
:1027600023000100220000002200000022000000DF
:1027700022000000220000002200010021000000D1
:1027800021000000210000002100000021000000C5
:1027900021000000210001002000000020000000B6
:1027A00020000000200000002000000020000000A9
:1027B00020000000200001001F0000001F0000009A
:1027C0001F0000001F0000001F0000001F0000008D
:1027D0001F0001001E0000001E0000001E0000007F
:1027E0001E0000003930000033250000871900006A
:1027F000B00F0000DB080000BD0400007402000000
:102800003F01000020436F756E7420583A00236426
:102810006566696E652044454641554C545F00002D
:10282000626564004B6420004B6920004B702000FF
:10283000504944204175746F74756E652066696EE9
:102840006973686564212050757420746865206C14
:10285000617374204B702C204B6920616E64204B97
:102860006420636F6E7374616E74732066726F6D33
:102870002062656C6F7720696E746F20436F6E669F
:10288000696775726174696F6E2E680A00504944F9
:10289000204175746F74756E65206661696C65643E
:1028A000212074696D656F75740A00504944204198
:1028B00075746F74756E65206661696C656421203E
:1028C00054656D706572617475726520746F6F20E8
:1028D000686967680A00204B643A2000204B693A17
:1028E0002000204B703A200020436C6173736963B1
:1028F00020504944200A00204E6F206F7665727385
:10290000686F6F740A002054753A2000204B753AA6
:102910002000206D61783A2000206D696E3A200019
:1029200020643A200020626961733A2000504944D3
:10293000204175746F74756E652073746172740ACA
:1029400000504944204175746F74756E652066614E
:10295000696C6564212054656D706572617475726F
:102960006520746F6F20686967680A0042656400BB
:10297000453100626564002C2073797374656D20A5
:1029800073746F7070656421204865617465725F4F
:1029900049443A200048656174696E672046616960
:1029A0006C65640048656174696E67206661696C76
:1029B0006564004D3131322053687574646F776EF1
:1029C000001000C90210012C014001220170011801
:1029D00001B0010E01F00104015002FA00B002F052
:1029E000003003E600D003DC009004D2007005C87C
:1029F00000A006BE000008B400B009AA00D00BA0D9
:102A000000600E960060118C00001582002019787D
:102A100000C01D6E00A0226400B0275A00902C5008
:102A20000000314600E0343C0010383200903A2873
:102A300000603C1E00A03D1400803E0A00203F00C4
:102A400000544845524D414C2052554E4157415932
:102A500000546865726D616C2052756E61776179A2
:102A6000004572723A204D415854454D50004D4139
:102A70005854454D502074726967676572656400EB
:102A80004572723A204D494E54454D50004D494EC5
:102A900054454D5020747269676765726564002003
:102AA0002F002042403A0020403A0020573A0020B0
:102AB000573A00496E76616C696420657874727566
:102AC0006465720A007C3C3E5E2B3D3F2F5B5D3BA4
:102AD0002C2A225C0043616E6E6F74206F70656EED
:102AE000207375626469722000534420496E6974D2
:102AF000204661696C0053442063617264206F6BEF
:102B00000A006F70656E526F6F74206661696C6544
:102B1000640A00766F6C756D652E696E6974206647
:102B200061696C65640A004E6F20534420636172D2
:102B3000640A000A4D3234004D3233202573002ED2
:102B40000A006F70656E206661696C65642C2046B2
:102B5000696C653A200046696C652073656C656335
:102B60007465640A002053697A653A200046696CEE
:102B700065206F70656E65643A2000454E442053B1
:102B80005542524F5554494E450A002220706F73EA
:102B9000002220706172656E743A220053554252D1
:102BA0004F5554494E452043414C4C207461726747
:102BB00065743A220053756263616C6C204F7665D0
:102BC00072666C6F77004578636565646564206D37
:102BD000617820535542524F5554494E4520646503
:102BE0007074683A002E0A0044656C6574696F6EF3
:102BF000206661696C65642C2046696C653A20002A
:102C000046696C652064656C657465643A0053447C
:102C1000207072696E74696E672062797465200035
:102C20004E6F74205344207072696E74696E670A27
:102C30000057726974696E6720746F2066696C65ED
:102C40003A2000667265736800646F696E670020E1
:102C500066696C653A20004E6F7720002F617574AD
:102C60006F25632E67002020506C616E6E65724286
:102C7000756666657242797465733A200020467203
:102C80006565204D656D6F72793A2000436F6D70F8
:102C9000696C65643A2041707220323920323032DA
:102CA000310A00204C61737420557064617465644E
:102CB0003A20323032312D30342D3138207C2041D1
:102CC0007574686F723A2054696E794D61636869F2
:102CD0006E657333440A00322E302E375F44573707
:102CE0002E332E310A004D61726C696E0020536FD5
:102CF0006674776172652052657365740A002057A7
:102D000061746368646F672052657365740A00209C
:102D100042726F776E206F75742052657365740A06
:102D2000002045787465726E616C2052657365741D
:102D30000A00506F77657255700A0073746172747F
:102D40000A004739310A47315A350A4739300A4DA6
:102D500038340A4D31303453300A4D313430533029
:102D6000004D31303031006572726F7220777269B8
:102D700074696E6720746F2066696C650A00446F21
:102D80006E6520736176696E672066696C652E0AD0
:102D9000004D323900456E6473746F7073002553B3
:102DA00020256320256320256320256300205A3ACF
:102DB0000020593A0020583A00656E6473746F70B1
:102DC00073206869743A200070012C01900127017A
:102DD000B0012201C0011D01F00118011002130110
:102DE00030020E016002090190020401C002FF00DE
:102DF0000003FA004003F5008003F000D003EB006D
:102E00002004E6007004E100E004DC004005D70087
:102E1000C005D2004006CD00D006C8008007C30020
:102E20003008BE00F008B900C009B400B00AAF0015
:102E3000B00BAA00D00CA500000EA000500F9B0004
:102E4000C01096005012910000148C00C01587002D
:102E5000B0178200B0197D00D01B7800001E7300EF
:102E600040206E0090226900F024640040275F003B
:102E700090295A00E02B5500102E500020304B00B6
:102E800010324600E033410090353C0010373700E7
:102E900070383200A0392D00B03A2800A03B230042
:102EA000603C1E00103D1900903D1400103E0F00C4
:102EB000703E0A00C03E0500003F0000403FFBFF9F
:102EC000803FF6FFC03FF1FF00000A0B02090C0D26
:102ED0000E080703040100000000000000000000CD
:102EE00000000000000000000000000000000000E2
:102EF000000000001211100000000000000000009F
:102F000000000000000000000000000000005072FF
:102F10006F62696E67204661696C656400205A3A89
:102F2000200020593A200042656420583A20003D94
:102F30003D6F6E55736572436F6E6669726D526553
:102F40007175697265643D3D00220A00556E6B6EB5
:102F50006F776E20636F6D6D616E643A2022002082
:102F600042002050006F6B00204500205A0020597D
:102F700000204D393220580020453A00205A3A00AE
:102F800020593A00583A0020746F6F206C6F6E67BA
:102F900020657874727573696F6E207072657665DE
:102FA0006E7465640A0020636F6C642065787472C7
:102FB0007573696F6E2070726576656E7465640AEC
:102FC0000043616E6E6F7420656E74657220737558
:102FD000626469723A20004D323520500A4D323415
:102FE00000526573756D65005549205061757365B4
:102FF000004E6F204D61746368203A004D32320AF2
:103000004D323100526566726573680050675570C5
:10301000005067446F776E0049732046696C6520E5
:10302000004973204469722000476F5570446972EB
:1030300000486173204D656469610046696C656E86
:10304000616D652053656C6563746564004D313056
:10305000303043004D313030300046696C616D6571
:103060006E7420537461742030202D203300466923
:103070006C616D656E7420537461742030202D2056
:10308000320046696C616D656E7420537461742002
:1030900030202D2031002046696C616D656E7420F2
:1030A000526573706F6E7365204E6F005265737555
:1030B0006D652059657320647572696E6720707242
:1030C000696E74000A204E6F2046696C616D656EF2
:1030D0007400496E76616C6964204F7074696F6E1C
:1030E000004D3530300053746F7265205365747431
:1030F000696E6773004265642050494420537461CF
:1031000072746564004D3939390A4D3238305030A7
:103110005331363000424C546F75636820526573EA
:103120006574004D3530320A4D35303000496E69D6
:103130007420454550524F4D00486F74656E6420B1
:10314000504944205374617274656400456E676C25
:1031500069736820416C72656164792053657400FD
:103160004368696E657365204E6F74205375707087
:103170006F7274656400496E4C616E6743686F6975
:103180006365000A202A2A2A7265636461742E64CA
:103190006174615B305D203D004732380A47312061
:1031A0004631303030205A313000556E73757070B2
:1031B0006F72746564204F7074696F6E2053656C14
:1031C00065637465640047323652323535004D31DF
:1031D00039305335350A4732380A4732390A4D34C7
:1031E00030300A4D313034533231350A4732380AE3
:1031F0004D313039533231350A4D34323053310A82
:103200004731583130305931303046353030300A5E
:1032100047315A300A4D3530300A4D31313720535D
:103220006574205A204F66667365740047312046E6
:1032300031303030205A302E30004732380A473192
:10324000204631303030205A302E30004D3530306D
:10325000005A204F6666736574203A202573004D2E
:10326000353030005A204F6666736574203A202549
:1032700073004732380A473146313530305A302EE4
:1032800030004732385A0A473146313530305A30EB
:103290002E30004D383400473146313030305A300E
:1032A0002E30004732380A473146313030305A30FC
:1032B0002E30004D616E75616C53657454656D7090
:1032C00000526571756573746564204F6666736539
:1032D00074204265796F6E64204C696D6974730067
:1032E0005A204F6666736574203A20257300526F2A
:1032F000756E64696E6720746F2073746570005218
:103300006571756573746564204F666673657420B6
:103310000053746F7020547269676765726564004A
:1033200053746F70204E6F0053746F705072696EDB
:10333000740048616E646C6520446174612041646E
:103340006A75737420322053657474696E672053F4
:10335000637265656E200048616E646C652044612F
:103360007461205072696E7446696C652033205315
:10337000657474696E672053637265656E200048DA
:10338000616E646C652044617461205072696E7472
:1033900046696C6520322053657474696E672053EA
:1033A000637265656E20004D38340048616E646C50
:1033B000652044617461205072696E7446696C6561
:1033C00020506F73740048616E646C6520446174B2
:1033D00061205072696E7446696C65205072650098
:1033E000426567696E537769746368003D3D2043A9
:1033F0006865636B6B65793D3D00726563646174FC
:103400002E61646472203D3D007265636461742EB8
:10341000646174615B305D203D3D00776169747764
:103420006179203D3D0020202A2A2A2A2A2A2A5270
:1034300054535F48616E646C65446174612A2A2A42
:103440002A2A2A2A2A2000526573656E643A2000CF
:1034500000002200250028002B002E00310034003F
:1034600002010000050108010B01000021002400F9
:1034700027002A002D003000330001010000040164
:1034800007010A01050505050705080808080202E5
:1034900002020A0A080804040404010101010101EE
:1034A00001010303030303030303040707070C0CD1
:1034B0000C0C0C0C0C0C0202020206060606060698
:1034C00006060B0B0B0B0B0B0B0B0102102020083D
:1034D000081020401020408002010201080402016F
:1034E00001020408102040808040201008040201DE
:1034F0008004020180402010080402010804020137
:1035000001020408102040800102040810204080BD
:10351000544D334420453520506C757320526561FD
:1035200064792E005072696E74696E672E2E2E00BB
:103530005072696E7420506175736564006E6F74AB
:10354000696669636174696F6E2000504944205454
:10355000756E652046696E697368656400003601A2
:10356000C20011241FBECFEFD1E2DEBFCDBF00E00D
:103570000CBF14E0A0E0B2E0E6E1F1E602E00BBF30
:1035800002C007900D92A831B107D9F726E1A8E152
:10359000B4E001C01D92A733B207E1F71AE1C0EB16
:1035A000DAE100E006C021970109802FFE010F94A7
:1035B000B82CCF3AD10780E00807A9F70F94301A4A
:1035C0000D9479300C9400009F92AF92BF92CF92ED
:1035D000DF92EF92FF920F931F93CF93DF9300D070
:1035E0001F921F92CDB7DEB7EFE5FBE10027BB27A7
:1035F000462F572FA82FAA2341F4A52F542FB85F89
:10360000AA2319F4A52F5527B85FA03138F4529595
:10361000A295452F4F70507FA42BBC5FA03428F497
:10362000550FAA1F550FAA1FBE5FA03818F4550FDB
:10363000AA1FB395550FAA1FEA0FF01F449151E03E
:10364000AA27B85081F1C8F0B0FF02C0440F551F3F
:10365000B1FF04C0440F551F440F551FB2FF06C0F1
:1036600052954295142F1F70407F512BB3FF1BC002
:10367000A52F542F44270C94531BB195B0FF02C0C3
:1036800055954795B1FF04C0559547955595479574
:10369000B2FF05C05295407F4295452B5F70B3FF46
:1036A00002C0452F5527DD24CC24BB24B2E0649F03
:1036B000D018C108B00AB00B749FC018B108B00B85
:1036C000849FB018B109659FC018B108B00B759FF1
:1036D000B018B109859FB0196A9FB018B1097A9FD7
:1036E000B0194D9DA12C99243327992722275D9D40
:1036F000A00C911C301F901F201FAD9D900C311D00
:10370000901F201F4C9DA00C911C301F901F201F4C
:103710005C9D900C311D901F201FAC9D300D911DA4
:10372000201F4B9D900C311D901F201F5B9D300D65
:10373000911D201FAB9D900D211D4B9F300D911DA4
:10374000201F5B9F900D211DAB9F200DB1E0BB247E
:10375000CC24DD24639FD018C108B00AB00B739F3E
:10376000C018B108B00B839FB018B109699FC01889
:10377000B108B00B799FB018B109899FB019629F49
:10378000B018B109729FB019D61AC70AB80A20F04A
:10379000B1E03B0F901F201F1124792F632F90E081
:1037A000822F0F900F900F900F900F90DF91CF917D
:1037B0001F910F91FF90EF90DF90CF90BF90AF904F
:1037C0009F900895AF92BF92CF92DF92EF92FF92B7
:1037D0000F931F93CF93DF93C1E4DCE004E019E083
:1037E00081E5A82E8CE0B82EC12CD12C7601C39493
:1037F00069917991899199910F94F6252889398950
:103800004A895B890F9457260F94342EF8016193EF
:103810007193819391938F01C616D706E806F90636
:1038200010F46B017C01AC16BD0611F76FEF7FEF52
:10383000CB01A70196010F94352C209314093093E6
:1038400015094093160950931709DF91CF911F91E5
:103850000F91FF90EF90DF90CF90BF90AF900895C1
:10386000CF92DF92EF92FF9280911008882309F4A3
:1038700057C0C0900C08D0900D08E0900E08F09052
:103880000F0820E030E0A901C701B6010F94F1252F
:10389000882309F445C020E030E040E05FE3C70141
:1038A000B6010F9457269B01AC010F9457262BEDC0
:1038B0003FE049E450E40F9457269B01AC0160E0DF
:1038C00070E080E89FE30F94BB2D6B017C01C092F8
:1038D000890CD0928A0CE0928B0CF0928C0C609147
:1038E000750270917602072E000C880B990B0F94CD
:1038F000F8252AE037ED43E25CE30F945726A70151
:1039000096010F9457266093710270937202809310
:10391000730290937402FF90EF90DF90CF90089520
:10392000C12CD12C80E8E82E8FE3F82ED0CF0F9356
:103930001F93CF93DF9350E0FC01E40FF51F8081CC
:10394000440F551F440F551F4A545A4FEA0188230C
:1039500029F188819981AA81BB81EB0108811981B4
:103960002A813B810097A105B10569F40C591F4FCD
:103970002F4F3F4FDA010D931D932D933C931397D7
:103980008FEF808306C0081B190B2A0B3B0B37FDFA
:10399000F7CFDF91CF911F910F910895188219826F
:1039A0001A821B82F6CFCF93DF9324E0829FC0015F
:1039B0001124EC01C951D74FFC01E35EF74F8F5E34
:1039C000974FDC012D913D914D915C91608171810A
:1039D000828193810F94C12C688379838A839B832E
:1039E000DF91CF9108958091B1059091B205A0919A
:1039F000B305B091B4058093410290934202A09325
:103A00004302B09344028091AF059091B00590932A
:103A1000780280937702089580914102909142024A
:103A2000A0914302B09144028093B1059093B205F6
:103A3000A093B305B093B40580917702909178027A
:103A40009093B0058093AF0584E690E09093780260
:103A50008093770208958091911290919212891B20
:103A6000877089F48091990D81110DC080918D0C22
:103A700090918E0C892B39F481E09091BF069111C1
:103A800003C080E0089581E00895CF93DF93DB01C8
:103A9000F9019C919130C1F0943080F094509C9346
:103AA0008830D1F480819181009771F001979183E2
:103AB0008083480F591FEA01188206C08C3539F4FB
:103AC0009C5F9C93943041F4DF91CF9108958B33A8
:103AD00039F781E08C93F8CF20813181B9016F5F94
:103AE0007F4F71836083420F531FEA018883808177
:103AF00091818F3591056CF7E7CF0F931F9381E08C
:103B000000913514109136142091371430913814E7
:103B100040913114509132146091331470913414E7
:103B2000041715072607370708F480E01F910F9147
:103B3000089590E080E00895282F90910B0883303D
:103B400021F495FD0FC094FD0FC0892F90E0B0E0E7
:103B5000A0E004C0B695A795979587952A95D2F7CA
:103B60008170089581E0089580E00895FC016591D9
:103B700075918591949108958F929F92AF92BF9283
:103B8000CF92DF92EF92FF92CF93DF93EC01809080
:103B9000E3089090E408A090E508B090E60820E0E3
:103BA00030E0A901C501B4010F94F125882309F47F
:103BB00054C0C880D980EA80FB80A7019601C50166
:103BC000B4010F94F12518160CF04CC02091DB08BD
:103BD0003091DC084091DD085091DE08C701B60144
:103BE0000F94F125882331F1C092DB08D092DC08D4
:103BF000E092DD08F092DE082091DF083091E008C5
:103C00004091E1085091E208688179818A819B8125
:103C10000F9457269B01AC0160E070E080E89FE3C1
:103C20000F94C02C60930F027093100280931102C6
:103C30009093120260910F02709110028091110214
:103C400090911202DF91CF91FF90EF90DF90CF9093
:103C5000BF90AF909F908F90089560E070E080E8F3
:103C60009FE3F0CF60E070E0CB01ECCFCF92DF922A
:103C7000EF92FF92CF93DF93EC01CC80DD80EE805A
:103C8000FF8027E137EB41ED58EBC701B6010F94F8
:103C9000212F87FD23C023E030E044EB53E4C7012C
:103CA000B6010F94F1251816CCF0C880D980EA80AF
:103CB000FB8027E137EB41ED58EBC701B6010F94CC
:103CC000212F87FD0BC0C1E023E030E044EB53E43B
:103CD000C701B6010F94F12518160CF4C0E08C2F23
:103CE000DF91CF91FF90EF90DF90CF9008952FEB71
:103CF000280F2A3108F047C0E22FF0E080914B05F1
:103D000090914C05A0914D05B0914E0504C0B6951B
:103D1000A795979587952A95D2F780FD02C0817067
:103D20000895E35DFA4FE081EE2341F180919D0714
:103D300090919E07E80FF92FF11D808190ED980F6B
:103D40009A3030F08E3251F4818180538A3098F469
:103D5000F0931C05E0931B0581E008958D3211F06E
:103D60008B3249F4818190ED980F9A3088F38E322E
:103D700011F48281EACFF0E0E0E0EACF10921C0576
:103D800010921B05E9CF80E008950E94771E8823DA
:103D900041F081E020911B0530911C05232B09F493
:103DA00080E008958F929F92AF92BF92CF92DF9260
:103DB000EF92FF92C090ED05D090EE05E090EF05F8
:103DC000F090F00520E030E0A901C701B6010F94A2
:103DD000F1258823E1F1A701960160E070E080E819
:103DE0009FE30F94BB2D6B017C018090F1059090B7
:103DF000F205A090F305B090F40520E030E0A901B1
:103E0000C501B4010F94F125882329F1A50194017E
:103E100060E070E080E89FE30F94BB2DC092F40453
:103E2000D092F504E092F604F092F7046093F8045F
:103E30007093F9048093FA049093FB04FF90EF9041
:103E4000DF90CF90BF90AF909F908F900895C12C3E
:103E5000D12C7601CACF60E070E0CB01DFCF129A9F
:103E600008955F9A80913F0C8E7F80933F0C8A9AD1
:103E700080913F0C8D7F80933F0C8091080180954D
:103E800081708093060180913F0C8B7F80933F0C63
:103E90000C942F1F269A2E9A08958C3221E09207B7
:103EA00014F08CE291E09093F6118093F5110C944C
:103EB0005DFDE9E2F6E01082118212821382148223
:103EC0000C945DFD4F925F926F927F928F929F92C2
:103ED000AF92BF92CF92DF92EF92FF920F931F9318
:103EE000CF93DF93EC012091E5053091E6054091F9
:103EF000E7055091E805688179818A819B810F945B
:103F0000C02C6B017C012091E9053091EA054091BC
:103F1000EB055091EC056C817D818E819F810F9422
:103F2000C02C4B015C01A7019601609103027091C6
:103F3000040280910502909106020F94F1258823D6
:103F400009F450C0C0920302D0920402E09205022C
:103F5000F09206022091F4043091F5044091F604A9
:103F60005091F704C701B6010F9457262B013C016D
:103F70000F94632E6B017C0120E030E0A9010F94C7
:103F8000F12587FD70C020E030E040E450E4C70137
:103F9000B6010F94212F18162CF4C12CD12CC0E49B
:103FA000EC2EFE2CA7019601C301B2010F94C02C88
:103FB0006093EC047093ED048093EE049093EF040F
:103FC000C701B6010F942D2E6093EA04062E000C53
:103FD000770B6F5F7F4F6430710514F064E070E021
:103FE0006093E804D09101021091EA04A5019401C4
:103FF00060910702709108028091090290910A0273
:104000000F94F125811133C0D11381C02091D004C8
:104010003091D1044091D2045091D3046091EC04CA
:104020007091ED048091EE049091EF040F94572667
:104030002091D4043091D5044091D6045091D704F6
:104040000F94C12CDF91CF911F910F91FF90EF90B2
:10405000DF90CF90BF90AF909F908F907F906F90A8
:104060005F904F900895C12CD12C76019BCF809208
:10407000070290920802A0920902B0920A022091CF
:10408000F8043091F9044091FA045091FB04C50101
:10409000B4010F9457264B015C010F94632E6B0102
:1040A0007C0120E030E0A9010F94F12587FDF3C0E9
:1040B00020E030E040E450E4C701B6010F94212F26
:1040C00018162CF4C12CD12CB0E4EB2EFE2CA70139
:1040D0009601C501B4010F94C02C6093F004709355
:1040E000F1048093F2049093F304C701B6010F9496
:1040F0002D2E6093EB04062E000C770B6F5F7F4F25
:104100006430710514F064E070E06093E904C091DC
:10411000EB04D11305C0809102028C1709F470C022
:104120008091EA049091EB04909302028093010243
:104130000C2E000CDD0B25E01203C0011124FC0144
:10414000EC0FFD1FEE0FFF1FEE0FFF1FE955F84F9D
:1041500020813181428153812093E4043093E5042E
:104160004093E6045093E7040091E904002E000C0C
:10417000110BFC01E00FF11FEE0FFF1FEE0FFF1FF1
:10418000E955F84F60817181828193810F94C02C31
:104190006093E0047093E1048093E2049093E3045D
:1041A0002091E80435E02303F0011124CE0FDF1F36
:1041B000CC0FDD1FCC0FDD1FC955D84F28813981A9
:1041C0004A815B812093DC043093DD044093DE045C
:1041D0005093DF04E00FF11FEE0FFF1FEE0FFF1FE4
:1041E000E955F84F60817181828193810F94C02CD1
:1041F0006093D8047093D9048093DA049093DB041D
:104200008090F0049090F104A090F204B090F30438
:104210002091E0043091E1044091E2045091E304E4
:10422000C501B4010F9457262091E4043091E504B0
:104230004091E6045091E7040F94C12C6B017C017E
:10424000C092D404D092D504E092D604F092D70460
:104250002091D8043091D9044091DA045091DB04C4
:10426000C501B4010F9457262091DC043091DD0480
:104270004091DE045091DF040F94C12CA7019601F8
:104280000F94C02C6093D0047093D1048093D20417
:104290009093D304BBCEC12CD12C760118CFCF92F2
:1042A000DF92EF92FF92CF93DF93EC0108960E948A
:1042B000BC1D6B017C0120E030E0A9010F94F125C9
:1042C00020E030E0A901882359F0CE010E94621F4E
:1042D0009B01AC01C701B6010F9457269B01AC01AD
:1042E000688579858A859B850F94C02C6887798736
:1042F0008A879B87DF91CF91FF90EF90DF90CF90DF
:1043000008952F923F924F925F926F927F928F9279
:104310009F92AF92BF92CF92DF92EF92FF920F9354
:104320001F93CF93DF93D62FC72FFC0180809180FE
:10433000A280B380C501B40120E831E541E050E03E
:104340000F94352CC9016DE671E00F94A42C6B011C
:104350007C01C501B40120E13EE040E050E00F9453
:10436000352CCA01B90128E130E040E050E00F945B
:10437000352C362E272E062F172F8CE3482E512C46
:10438000612C712CC501B401A30192010F94352C4D
:10439000B62EA72ECA01B901A30192010F94352CA4
:1043A000CB01C114D10479F1AF92BF927F936F9387
:1043B0002F923F92FF92EF92DF92CF9286E697E1A3
:1043C0009F938F93CF93DF930F9488258DB79EB7DC
:1043D0000E960FB6F8949EBF0FBE8DBF8D2F9C2FEB
:1043E000DF91CF911F910F91FF90EF90DF90CF90D1
:1043F000BF90AF909F908F907F906F905F904F9005
:104400003F902F900895E114F104C9F0AF92BF924C
:104410007F936F932F923F92FF92EF9286E597E101
:104420009F938F93CF93DF930F948825EDB7FEB7BB
:104430003C960FB6F894FEBF0FBEEDBFCFCF012B59
:10444000B9F0AF92BF927F936F932F923F928AE41D
:1044500097E19F938F93CF93DF930F9488258DB728
:104460009EB70A960FB6F8949EBF0FBE8DBFB6CF0B
:10447000892BA9F0AF92BF927F936F9382E497E16B
:104480009F938F93CF93DF930F948825EDB7FEB75B
:1044900038960FB6F894FEBF0FBEEDBF9FCFAF9218
:1044A000BF928EE397E19F938F93CF93DF930F9407
:1044B00088250F900F900F900F900F900F908ECF38
:1044C000EF92FF920F931F93CF93DF93CDB7DEB799
:1044D0008C01EDB6FEB60F943E2501962DB73EB782
:1044E000281B390B0FB6F8943EBF0FBE2DBF8DB7FA
:1044F0009EB70196B8010F9437250E9480F90FB638
:10450000F894FEBE0FBEEDBEDF91CF911F910F91CB
:10451000FF90EF9008958C38910514F08CE890E0AE
:1045200090938B1180938A110C94D3BEAB01BC0184
:1045300040933514509336146093371470933814A5
:104540008DE995E10C948BAF2F923F924F925F9241
:104550006F927F928F929F92AF92BF92CF92DF9293
:10456000EF92FF920F931F93CF93DF93CDB7DEB7F8
:1045700060970FB6F894DEBF0FBECDBF8B876C87F8
:10458000042F122F282F30E03E872D87462F50E032
:104590005A87498785E0982E929EC001939E900D80
:1045A0001124988B8F87FA01E80FF91FEE0FFF1F78
:1045B000EE0FFF1FE955F84F608171818281938171
:1045C0009B01AC010F94B32F882309F445C14B859F
:1045D000400F6C85610F949EC0011124E985FA8516
:1045E000E80FF91FEE0FFF1FEE0FFF1FE955F84F01
:1045F000C080D180E280F380040F909EA00111243E
:10460000E985FA85E40FF51FEE0FFF1FEE0FFF1F80
:10461000E955F84F0081918082807380262F30E029
:10462000EF85F889E20FF31FEE0FFF1FEE0FFF1F5C
:10463000E955F84F20807181798372817A83738183
:104640007B83610F70E0EF85F889E60FF71FEE0FAF
:10465000FF1FEE0FFF1FE955F84FF88BEF87F08132
:10466000FC83EF85F889F181FD83EF85F889F2817C
:10467000FE83EF85F889F381FF83FC01E20FF31FCE
:10468000EE0FFF1FEE0FFF1FE955F84F208128871F
:10469000A180B2806380FA01E60FF71FEE0FFF1FC3
:1046A000EE0FFF1FE955F84F408051803280138193
:1046B000202F392D482D572D602F792D882D972D9E
:1046C0000F94B32F882321F000E0912C812C712CC2
:1046D0009601A701B601C7010F94B32F882321F0DB
:1046E000C02ED92CE82CF72C2C813D814E815F8186
:1046F0006C817D818E819F810F94B32F882321F05F
:104700001C821D821E821F82222D39814A815B817B
:10471000622D79818A819B810F94B32F882339F090
:104720002C803D8139834E814A835F815B83920176
:10473000432D512FB201832D912F0F94B32F882336
:1047400021F0412C512C312C10E028853A2D4B2D95
:10475000562D68857A2D8B2D962D0F94B32F882397
:1047600021F04886A52CB32C612E85E02D853E8551
:10477000829FF001839FF00D112449855A85E40F33
:10478000F51FEE0FFF1FEE0FFF1FE955F84FFA87D9
:10479000E9879601A701B601C7010F94C12C202F0C
:1047A000392D482D572D0F94C02C6B017C01222DE3
:1047B00039814A815B81622D79818A819B810F9445
:1047C000C12C2C813D814E815F810F94C02C9B01B7
:1047D000AC01C701B6010F94C12C6B017C01288587
:1047E0003A2D4B2D562D68857A2D8B2D962D0F94B5
:1047F000C12C9201432D512F0F94C02C9B01AC0171
:10480000C701B6010F94C12C20E030E040E450E431
:104810000F94BB2DE985FA8560837183828393832E
:104820006C858B8560960FB6F894DEBF0FBECDBF4A
:10483000DF91CF911F910F91FF90EF90DF90CF907C
:10484000BF90AF909F908F907F906F905F904F90B0
:104850003F902F900C9413F860960FB6F894DEBF3B
:104860000FBECDBFDF91CF911F910F91FF90EF90C1
:10487000DF90CF90BF90AF909F908F907F906F9080
:104880005F904F903F902F90089580911B059091DD
:104890001C05009731F04AE050E070E060E00D94B4
:1048A0000C2460E070E0CB01089580911B0590918D
:1048B0001C05009731F04AE050E070E060E00D9494
:1048C000DE2260E070E0CB010895CF93DF93EB012F
:1048D0000E94C51E882319F00E945524EB01CE01C9
:1048E000DF91CF9108950E94552497FD0CC00E943E
:1048F00055246F3F71058105910509F034F40E943C
:104900005524862F089580E008958FEF0895CF9362
:10491000C62F0E94C51E882319F0CF910C947324D2
:104920008C2FCF91089580911B0590911C05892BA8
:1049300041F00E94732491E0811101C090E0892F21
:10494000089591E0FCCFCF93DF93C82FD62F0E941C
:10495000C51E882321F0DF91CF910C9493248C2FD6
:104960000E94771E811101C08D2FDF91CF91089594
:104970000E945524CB010895CF93DF93EB010E9451
:10498000C51E882321F0DF91CF910C94B824CE016D
:10499000DF91CF9108950F931F93CF9380911B05C3
:1049A00090911C050097E9F0FC018F01C1912C2F1B
:1049B0002F7D81F0C53411F0C536B9F7F8011082AA
:1049C00070E060E00F948021F801C083CF911F91C7
:1049D0000F91089570E060E0CF911F910F910D94B9
:1049E000802160E070E0CB01F1CFCF92DF92EF92B7
:1049F000FF926A017B010E94C51E882331F0FF905F
:104A0000EF90DF90CF900C94CB24C701B601FF90BC
:104A1000EF90DF90CF9008954F925F926F927F92C8
:104A20008F929F92AF92BF92CF92DF92EF92FF92BE
:104A30001F93CF93DF9300D01F92CDB7DEB71982BB
:104A40001A821B821C82CE0101964C018BE8C82E73
:104A500087E0D82E91E6E92E92E0F92E27EEA22EDD
:104A600028E0B22E10E088E5810F0E94C51EF401F7
:104A700081934F01882309F4E0C00E94CB242B01CD
:104A80003C01812F0E949C1D882309F4CCC0F701B2
:104A90002081318142815381C301B2010F94C12C25
:104AA000F60160837183828393831F5FF4E0CF0EEE
:104AB000D11C84E0E80EF11C94E0A90EB11C133067
:104AC00091F685E40E94C51E8C83882309F4C0C03A
:104AD0000E94CB246B017C0183E00E949C1D8823F3
:104AE00071F020916D0230916E0240916F025091F1
:104AF0007002C701B6010F94C12C6B017C01C092FA
:104B00009707D0929807E0929907F0929A078091C0
:104B1000E405882359F18091391482FF27C08C81E4
:104B2000882321F18981811103C08A818823F1F0D2
:104B30002DEC3CEC4CE45DE360913208709133085D
:104B400080913408909135080F94C12C9B01AC01E1
:104B50006091690270916A0280916B0290916C027F
:104B60000F94212F181614F40E9459F740E050E0DA
:104B7000BA0186E40E94F52420E030E0A9010F94F8
:104B8000212F181684F40E94CB2420E030E040E767
:104B900052E40F94BB2D60934102709342028093C4
:104BA0004302909344028091FD0B83FD28C08091C5
:104BB000AA06882321F120916D0230916E02409166
:104BC0006F025091700260919707709198078091E1
:104BD000990790919A070F94C02C2091B7063091B5
:104BE000B8064091B9065091BA060F94C12C609353
:104BF000B7067093B8068093B9069093BA060F90E3
:104C00000F900F900F90DF91CF911F91FF90EF9039
:104C1000DF90CF90BF90AF909F908F907F906F90DC
:104C20005F904F900895F501208131814281538139
:104C3000C301B2010F94C02C33CFF7018081918161
:104C4000A281B381F60180839183A283B3832DCFA8
:104C500080916D0290916E02A0916F02B0917002EE
:104C60008093970790939807A0939907B0939A071A
:104C70004ECFCF92DF92EF92FF926B017C0183E3E4
:104C8000C816D104E104F10470F082E3C81AD10817
:104C9000E108F10862E370E080E090E00E941EFD10
:104CA0000E944DC2ECCFC701B6010E941EFDFF90CD
:104CB000EF90DF90CF900C944DC2CF92DF92EF92A5
:104CC000FF920F931F93CF93DF936B017A01EC0157
:104CD000C055DB4F28813CE0389F8001399F100D83
:104CE000112427FF24C0FB011182108288818F5F6D
:104CF000888388819801280F311D87FD3A95C90165
:104D000020917C12F6012817190629F024F08881D9
:104D10008C300CF43CC080819181049680349C4995
:104D200008F475C0F60180819181049672C0888173
:104D30009801280F311D87FD3A95C90120917C12F9
:104D40002817190699F294F28881A801480F511D7D
:104D500087FD5A95FA01EE0FFF1FE40FF51FEC5C7B
:104D6000FD4E808187FFC2CF8881F801E80FF11DD9
:104D700087FDFA95CF01EE0FFF1FE80FF91FEC5CDE
:104D8000FD4E808160E08F770E94BCFBAFCF8081B9
:104D900091812881A801420F511D27FD5A959A0142
:104DA000FA01EE0FFF1FE20FF31FEC5CFD4E2181B5
:104DB0003281820F931FF70191838083888198014C
:104DC000280F311D87FD3A95F901EE0FFF1FE20F05
:104DD000F31FEC5CFD4E808187FF20C08881080FA7
:104DE000111D87FD1A95F801EE0FFF1FE00FF11F4F
:104DF000EC5CFD4E808161E08F77DF91CF911F9158
:104E00000F91FF90EF90DF90CF900C94BCFB80E46B
:104E10009CE9F701918380838FEF8883DF91CF91A5
:104E20001F910F91FF90EF90DF90CF9008950F9317
:104E30001F93CF93DF9305E51CE0CEE6D1E1F801A7
:104E400021913191419151918F0160E070E080E8B2
:104E50009FE30F94BB2D6993799389939993F1E123
:104E6000CE37DF0761F70E9498F5DF91CF911F9150
:104E70000F910C94E21BCF92DF92EF92FF92CF93AF
:104E8000DF932091400C222329F1EC0108960E9427
:104E9000BC1D6B017C0120E030E0A9010F94F125DD
:104EA00020E030E0A901882359F0CE010E94621F62
:104EB0009B01AC01C701B6010F9457269B01AC01C1
:104EC000688579858A859B850F94C12C6887798749
:104ED0008A879B87DF91CF91FF90EF90DF90CF90F3
:104EE00008952F923F924F925F926F927F928F928E
:104EF0009F92AF92BF92CF92DF92EF92FF920F9369
:104F00001F93CF93DF93CDB7DEB76C970FB6F894AE
:104F1000DEBF0FBECDBF8C015B015A834983FC010C
:104F2000EA5BFF4F208131814281538129873A8793
:104F30004B875C87CA01B9010F94F6256B017C0190
:104F4000D5012D913D914D915C910F9457260F9471
:104F50009F2D2B013C01E981FA8120813181428121
:104F60005381C701B6010F9457260F949F2D4B0113
:104F70005C01C301B2010F94342E698B7A8B8B8B49
:104F80009C8B683771058105910540F428E730E076
:104F900040E050E0298B3A8B4B8B5C8BC501B40110
:104FA0000F94342E6D877E878F87988B68377105B5
:104FB0008105910540F448E750E060E070E04D87DE
:104FC0005E876F87788BF801EE5AFF4F40805180E3
:104FD00062807380C301B2010F94F82569837A83DC
:104FE0008B839C8369897A898B899C890F94F625A8
:104FF0006D8B7E8B8F8B988F20E030E0A9016981CB
:105000007A818B819C810F94F125882309F4E1C179
:10501000A7019601C701B6010F9457264B015C0109
:105020002D893E894F89588DCA01B9010F945726A1
:105030009B01AC01C501B4010F94C02C4B015C0174
:1050400029813A814B815C81CA01B9010F94C12C3D
:105050009B01AC01C501B4010F94BB2D0F949F2D92
:105060000F94342E6D837E838F83988766277727EE
:10507000CB0164197509860997090F94F8254B012E
:105080005C016D857E858F8598890F94F6252B01AF
:105090003C0120E030E0A901C501B4010F94F125E5
:1050A000882309F49AC1A3019201C301B2010F94AC
:1050B0005726698F7A8F8B8F9C8FA7019601C70126
:1050C000B6010F9457269B01AC01698D7A8D8B8DAB
:1050D0009C8D0F94C02C6B017C01A5019401C5012E
:1050E000B4010F94C12C9B01AC01C701B6010F9410
:1050F000BB2D0F94632ED80195968D909D90AD9009
:10510000BC909897750164012D813E814F8158852F
:10511000C21AD30AE40AF50A0F94342EC61AD70A23
:10512000E80AF90AF7FE8EC02D893E894F89588D0D
:10513000CA01B9010F9457266B017C0129813A817C
:105140004B815C81CA01B9010F94C12C69877A87B0
:105150008B879C8720E030E0A90169817A818B816F
:105160009C810F94F125882309F43BC1C501B4014A
:105170000F94F62529853A854B855C850F94572633
:10518000A70196010F94C02C6D837E838F8398872F
:10519000A3019201C301B2010F9457269B01AC01F8
:1051A0006D817E818F8198850F94C12C2B013C01EC
:1051B00020E030E040E850E469817A818B819C8175
:1051C0000F9457269B01AC01C301B2010F94BB2D74
:1051D0000F949F2D2B013C0120E030E0A9010F949A
:1051E000212F18161CF0412C512C3201C301B201A1
:1051F0000F94342E6D837E838F839887861697064F
:10520000A806B90620F48D829E82AF82B8866D8191
:105210007E818F8198850F94F62529853A854B8567
:105220005C850F945726A70196010F94C12C0F940B
:105230006F2F0F94342E69877A878B879C87C12CB8
:10524000D12C760169857A858B859C8529893A8957
:105250004B895C89621B730B840B950B0F94F625AD
:1052600029813A814B815C810F94BB2D20E034E28F
:1052700044EF59E40F9457260F94342E4B015C01F0
:1052800069857A858B859C852D853E854F855889D6
:10529000621B730B840B950B0F94F62529813A81C1
:1052A0004B815C810F94BB2D20E034E244EF59E444
:1052B0000F9457260F94342E2B013C013FE68316A2
:1052C0009104A104B10408F090C0F401EE0FFF1F97
:1052D000EE0FFF1FED55F64E85919591A591B49176
:1052E0008983292E3A2EBD8B4FE644165104610462
:1052F000710408F083C0F201EE0FFF1FEE0FFF1FD5
:10530000ED55F64E45915591659174919A01CB01F9
:105310004D815E816F817885D80199964D935D931B
:105320006D937C939C974C0D5D1D6E1D7F1DF80148
:1053300045A756A767A770ABE65BFF4F49895A8917
:105340006B897C894083518362837383D5968D9268
:105350009D92AD92BC92D897F80141AE52AE63AE29
:1053600074AEFD9649814083218232825D895383E8
:105370003496208331838283938369857A858B85F4
:105380009C85D1966D937D938D939C93D4973D96F8
:105390002D853E854F8558892083318342835383F1
:1053A0006C960FB6F894DEBF0FBECDBFDF91CF91E4
:1053B0001F910F91FF90EF90DF90CF90BF90AF9033
:1053C0009F908F907F906F905F904F903F902F9025
:1053D000089560E070E0CB0141CE60E070E0CB0169
:1053E00088CE60E070E0CB01F3CEC501B4010E942D
:1053F000E41A6983272E382E9D8B76CFC301B20124
:105400000E94E41A9B0184CF809191129091921294
:10541000891B877019F490E080E0089590918E12B6
:10542000992351F0833030F48FEF890F19F0809376
:105430008E12F1CF10928E12809192122CE5829FE3
:10544000C0011124835E964FFC01208120FDE3CF33
:10545000209192122F5F277020938F123091921219
:1054600020919012321304C020918F122093901239
:10547000089590916F0081E091FD02C080E0089551
:1054800090916F009D7F90936F00089580FF04C0FE
:1054900090913F0C90FD8E7F81FF05C090913F0C55
:1054A000969590FD8D7F82FF06C090913F0C96955A
:1054B000969590FD8B7F08958F929F92AF92BF92A9
:1054C000CF92DF92EF92FF92CF93DF93209145022C
:1054D000222309F49EC0EC018091B505C82ED12C81
:1054E000F12CE12C80FF2CC0809047029090480264
:1054F000A0904902B0904A02288139814A815B819B
:10550000C501B4010F94212F181624F488829982C2
:10551000AA82BB828090530290905402A0905502C0
:10552000B0905602288139814A815B81C501B4015E
:105530000F94F12587FF04C088829982AA82BB82DA
:10554000D701C601B695A7959795879580FF2CC082
:1055500080904B0290904C02A0904D02B0904E0271
:105560002C813D814E815F81C501B4010F94212FB3
:10557000181624F48C829D82AE82BF8280905702DE
:1055800090905802A0905902B0905A022C813D810F
:105590004E815F81C501B4010F94F12587FF04C0DE
:1055A0008C829D82AE82BF8282E0F694E794D7948B
:1055B000C7948A95D1F7C0FE2CC0C0904F02D090FE
:1055C0005002E0905102F0905202288539854A85B8
:1055D0005B85C701B6010F94212F181624F4C886E5
:1055E000D986EA86FB86C0905B02D0905C02E09090
:1055F0005D02F0905E02288539854A855B85C7018A
:10560000B6010F94F12587FF04C0C886D986EA86C3
:10561000FB86DF91CF91FF90EF90DF90CF90BF900E
:10562000AF909F908F900895CF92DF92EF92FF926C
:105630000F931F93C12CD12C76018C012DE632E003
:1056400049E652E065E672E081E692E00E9494F459
:105650001F910F91FF90EF90DF90CF9008950C94E1
:1056600098F58091A205659B6EC080618093A2052C
:10567000909103018091A20591FF67C080628093A1
:10568000A2058091A2054B9B62C084608093A20515
:105690008091A2059091A105981709F45AC092E053
:1056A0009093A0058093A1058091BC06811105C04F
:1056B00080919B07882309F459C08091090680FFD7
:1056C00010C08091BD0680FD0CC080919F0584FFB5
:1056D00008C08091FF0680618093FF0680E00E94F1
:1056E000ADC680910906869580FF11C08091BD06E8
:1056F000869580FD0CC080919F0585FF08C0809134
:10570000FF0680628093FF0681E00E94ADC6809113
:1057100009068695869580FF29C08091BD068695ED
:10572000869580FF23C080919B078823F9F08091A4
:105730009F0582FF1BC08091FF0684608093FF0657
:1057400082E00C94ADC68F7E91CF8F7D98CF8B7FFA
:105750009DCF8091A005882309F4A6CF8150809326
:10576000A0058111A1CF90939F059ECF08958091B0
:10577000BC06811104C080919B07882331F062E050
:1057800070E080E090E00C94392608950F931F9309
:1057900080912C11813019F50E9451FD0091BE05B8
:1057A0001091BF052091C0053091C105601B710BA0
:1057B000820B930B28EE33E040E050E00F94352C41
:1057C0006091C2057091C3058091C4059091C50593
:1057D000620F731F841F951F1F910F910895609191
:1057E000C6057091C7058091C8059091C905D6CFAF
:1057F00010922C111092BE051092BF051092C00598
:105800001092C1051092C6051092C7051092C805E6
:105810001092C9051092C2051092C3051092C405DA
:105820001092C5050895CF92DF92EF92FF92CF9329
:10583000DF93C62FFC01C080D180E280F38020E09E
:1058400030E0A901C701B6010F94F12520E030E056
:10585000A90187FD14C020E030E048EC52E4C70104
:10586000B6010F94212F24E630E040E050E01816F6
:1058700034F0C701B6010F942D2E9B01AC01C2304C
:10588000A0F4D0E0C85ED64FAFEFB0E00F94762C16
:1058900024E630E040E050E00F94572C2F3F3105D4
:1058A00019F010F02FEF30E02883DF91CF91FF90B7
:1058B000EF90DF90CF9008958091090180FD06C0A0
:1058C0008091391483FB882780F9089580E008953A
:1058D000CF92DF92EF92FF92FC01C080D180E280F4
:1058E000F380663019F510922E0610922F06109252
:1058F000300610923106109232060E94D3BE20E08C
:1059000030E0A901C701B6010F94F12587FF1DC042
:10591000C12CD12C7601C701B6010F942E2FCB01DB
:10592000FF90EF90DF90CF900C948B220E94591F34
:1059300020E030E0A901C701B6010F94F12587FFEF
:1059400015C0C12CD12C760121C020E030E04CE004
:1059500053E4C701B6010F94212F1816E4F6C12CA9
:10596000D12C9CE0E92E93E4F92ED5CF20E030E055
:1059700046E953E4C701B6010F94212F181634F4F9
:10598000C12CD12C86E9E82E83E4F82EC701B6019C
:105990000F942E2FCB01FF90EF90DF90CF900C94BF
:1059A0004D1F90913F0C977081E0973009F080E097
:1059B000089520919D0520FF14C020E83EE3629FDA
:1059C000A001639F500D729F500D1124CA0196953E
:1059D000879596958795009731F08A950000E9F7AD
:1059E00008950C9439260895CF93DF931092FE0BFF
:1059F00010928F0C1092910C1092900C10929C05AA
:105A000010929B05CFEFDFEF8091391485FD07C021
:105A10000E94ECAAD093B812C093B712F5CF8FEFC3
:105A20009FEF9093B8128093B712DF91CF910895B2
:105A30008F929F92AF92BF92CF92DF92EF92FF929E
:105A40000F931F93CF93DF931092500510924F0541
:105A50002FE320934A0510924905109248051092B1
:105A6000470510924B0510924C0510924D0510926F
:105A70004E059C01F90190812F5F3F4F9032D1F389
:105A80009E34C9F4818190ED980F9A3020F08D32C8
:105A900011F08B3281F432969F012F5F3F4F80814E
:105AA00080538A3008F47BC09F012F5F3F4F808175
:105AB000803209F476C0F0939E07E0939D078F0132
:105AC0000F5F1F4FC0816AE270E0C8010F940F3072
:105AD000009731F0FC01319780818032E1F311822F
:105AE000CD3429F0C43519F0C73409F04BC0F801A2
:105AF00080810F5F1F4F8032D1F380538A3008F0CE
:105B000041C0C0934A0530E020E04AE0DF01119631
:105B1000429FC001439F900D11249C0120533109E5
:105B20008081280F311D87FD3A95818190ED980F76
:105B30009A30C8F130934905209348058E3261F4BC
:105B4000329690E04AE0DF0131968C9150ED580F8B
:105B50005A3058F190934705CD01DC0101964C91E4
:105B60004032D9F3CD3489F52E31310539F018F5AD
:105B70002731310519F02C31310539F5B093500535
:105B8000A0934F05DF91CF911F910F91FF90EF9060
:105B9000DF90CF90BF90AF909F908F900895F901C4
:105BA0007BCFF90181CFFD01B1CF949F800D1124EE
:105BB00090ED980FC8CF2537310538F027373105DC
:105BC000E8F2203A83E03807C9F2D0919D0740E01F
:105BD00050E0BA0110E000E0C12CD12C7601C39452
:105BE000FD0131968C91882309F47FC08132E1F464
:105BF000CD34D1F420323105B9F440934B055093A4
:105C00004C0560934D0570934E05F0935005E0935D
:105C10004F0563E270E0CF010F940F30009709F455
:105C2000B1CFFC011082AECF81548A3108F058C048
:105C3000DF019D91903291F0A0EDA90FAA30E8F01C
:105C40009E3271F4918190539A30B8F0011511058C
:105C500019F48F010150110990E013C0FD01E8CF44
:105C60009D3211F09B3291F79181A0EDA90FAA30DE
:105C700020F09E3259F79281E6CF9E2F9D1B3097E0
:105C800059F3A82FB0E04601570104C0880C991CB5
:105C9000AA1CBB1C8A95D2F7482959296A297B2955
:105CA000A35DBA4F9C9380818154DF018A3108F44F
:105CB00097CFDF018191882309F492CF90ED980F5F
:105CC0009A30B8F393ED980F923098F38B3289F3B2
:105CD000CD010196EC91E03209F082CFDC01F8CFE2
:105CE0000115110501F78D01DECF109350050093CA
:105CF0004F0540934B0550934C0560934D057093B1
:105D00004E0540CF4F925F926F927F928F929F92FB
:105D1000AF92BF92CF92DF92EF92FF92CF93DF9339
:105D200000D000D01F921F92CDB7DEB75C01DB011F
:105D3000CD90DD90ED90FC90E0918C12F0918D1261
:105D4000FE83ED8384819581A681B78189839A83BF
:105D5000AB83BC839C01AD01C701B6010F94C02C7D
:105D60002B013C01F50180809180A280B380AD8140
:105D7000BE818D919D910D90BC91A02D8D839E83B0
:105D8000AF83B88727E137EB41ED58EBC301B20190
:105D90000F94212F87FDD1C023E030E044EB53E482
:105DA000C301B2010F94F12518160CF4C6C02D8161
:105DB0003E814F815885C501B4010F94C02C2B0141
:105DC0003C0127E137EB41ED58EB0F94212F87FD84
:105DD000B4C023E030E044EB53E4C301B2010F94BC
:105DE000F12518160CF4A9C020E030E0A9016D815E
:105DF0007E818F8198850F94C12C2B013C0120E07E
:105E000030E040E450E40F94F12587FF05C0412CB9
:105E1000512C30E4632E762C27E137EB41ED58E32B
:105E2000C301B2010F94C02C9B01AC01C501B401A8
:105E30000F94212F87FD81C020E030E044EB53E434
:105E40006D817E818F8198850F94C12C2B013C013F
:105E500020E030E842EB53E40F94212F18163CF475
:105E6000412C20E8522E22EB622E23E4722E27E1F1
:105E700037EB41ED58E3C301B2010F94C12C9B01F4
:105E8000AC01C501B4010F94F12518160CF455C0EE
:105E900020E030E0A90169817A818B819C810F9497
:105EA000C12C4B015C0120E030E040EE51E40F9446
:105EB000F12587FF06C0812C912C90EEA92E91E44C
:105EC000B92E27E137EB41ED58E3C501B4010F943A
:105ED000C02C9B01AC01C701B6010F94212F87FD97
:105EE0002CC020E030E044EB53E469817A818B815F
:105EF0009C810F94C12C4B015C0120E030E046EA0C
:105F000053E40F94212F181634F4812C912C86EA37
:105F1000A82E83E4B82E27E137EB41ED58E3C50105
:105F2000B4010F94C12C9B01AC01B1E0B983C7014E
:105F3000B6010F94F12518160CF419828981289660
:105F40000FB6F894DEBF0FBECDBFDF91CF91FF90AB
:105F5000EF90DF90CF90BF90AF909F908F907F9009
:105F60006F905F904F900895E9E2F8E082EBDF01D7
:105F70001D928A95E9F708958091E405811104C086
:105F80000E94B42F0C944DB88091391482FD0C946A
:105F900059F7089580912908882361F09091DA08D3
:105FA000891308C08091391483FF04C087E698E004
:105FB0000C9417B780E00895FC01238121110C9403
:105FC0004CB30895EFE6F0E080818260808308950D
:105FD000CF92DF92EF92FF92CF93DF93C82F0E9470
:105FE000392A94E0C99FE0011124FE01E95EF94FCE
:105FF000C080D180E280F38081110E94E22FC259DB
:10600000DE4EC701B6010F94F825288139814A81F7
:106010005B810F945726DF91CF91FF90EF90DF9037
:10602000CF9008958F929F92AF92BF92CF92DF92BE
:10603000EF92FF921F93CF93DF93CDB7DEB76097B8
:106040000FB6F894DEBF0FBECDBF182F80E00E94C0
:10605000E82F4B015C018092A3059092A405A092C9
:10606000A505B092A60581E00E94E82F6B017C0196
:10607000C092A705D092A805E092A905F092AA05C2
:1060800082E00E94E82F6093AB057093AC0580938B
:10609000AD059093AE051D861E861F86188A8982DF
:1060A0009A82AB82BC82CD82DE82EF82F8866987DB
:1060B0007A878B879C8783E00E94E82F6D877E8795
:1060C0008F87988B8091400C882321F0CE01019618
:1060D0000E944F211E3FD9F480E1FE013196A1E6D6
:1060E000B2E001900D928A95E1F760960FB6F894B0
:1060F000DEBF0FBECDBFDF91CF911F91FF90EF901C
:10610000DF90CF90BF90AF909F908F90089584E0E4
:10611000189FF0011124DF01AF59BD4F81E090E0DD
:106120008C0F9D1FE80FF91F40815181628173819F
:106130004D935D936D937C931397D7CFCF92DF925E
:10614000EF92FF92CF93DF93C82F0E94392A94E0F9
:10615000C99FE0011124FE01E55FF94FC080D180A5
:10616000E280F38081110E94E22FC259DE4EC70106
:10617000B6010F94F825288139814A815B810F94FB
:106180005726DF91CF91FF90EF90DF90CF90089549
:106190000E94392A909192129093911290939012AA
:1061A00090938F1294E690938E1220ED33E030930B
:1061B0001C0920931B0981110E94E22F81E080932A
:1061C0000A060895CF93DF93CDB7DEB72C970FB6AD
:1061D000F894DEBF0FBECDBF0E9476F60E94392A2A
:1061E0009CE0E7E1F6E0DE01119601900D929A95B0
:1061F000E1F781110E94E22FCE0101960E948DC627
:106200002C960FB6F894DEBF0FBECDBFDF91CF91B5
:1062100008952F923F924F925F926F927F928F924A
:106220009F92AF92BF92CF92DF92EF92FF920F9325
:106230001F93CF93DF9300D0CDB7DEB7809061027C
:1062400090906202A0906302B09064024090650258
:10625000509066026090670270906802C090690278
:10626000D0906A02E0906B02F0906C020E94E21BF8
:106270000E94301C03E81CE187E492E09B838A8340
:1062800087E7282E8CE1382E198289810E94D31C41
:10629000C8010E94B61DEA81FB81619371938193CD
:1062A0009193FB83EA83C1010E94B61DEA81FB81C1
:1062B0006087718782879387F981FF5FF9830C5F1D
:1062C0001F4F84E0280E311CF330F9F685EF95E07E
:1062D0000E94DBF60E94D21E0E941727A50194019E
:1062E00060916102709162028091630290916402F8
:1062F0000F94F12581111CC0A301920160916502E8
:106300007091660280916702909168020F94F12566
:1063100081110EC02091690230916A0240916B0296
:1063200050916C02C701B6010F94F1258823B9F092
:106330000F900F900F90DF91CF911F910F91FF90D1
:10634000EF90DF90CF90BF90AF909F908F907F9015
:106350006F905F904F903F902F900C94E2300F9091
:106360000F900F90DF91CF911F910F91FF90EF90C1
:10637000DF90CF90BF90AF909F908F907F906F9065
:106380005F904F903F902F9008958091821190914F
:106390008311892B79F48091821190918311892B3B
:1063A00049F4209182113091831181E0232B19F45B
:1063B00080E0089581E00895109201058091220205
:1063C00090912302A0912402B091250280930106AE
:1063D00090930206A0930306B0930406089590914B
:1063E000991110929911923071F0943079F09130A6
:1063F00099F4813089F480910105882369F0109225
:1064000026020C94DC3110923E0C08958AE898E143
:1064100090938E0C80938D0C08959091391493FB7A
:10642000882780F993FF06C081E09091A015911113
:1064300001C080E00895CF93C0919E05CF7739F5D4
:106440000E940D32882319F18091311490913214F9
:10645000A0913314B09134140097A105B105B9F09F
:10646000BC01CD016D597F4F8F4F9F4F24E630E027
:1064700040E050E00F94352C609135147091361443
:1064800080913714909138140F94352CC22F8C2F93
:10649000CF910895E8E1F9E010821182089581E03A
:1064A0000895DC01EC918E2F90E0FC01EE0FFF1FB0
:1064B000E80FF91FEC5CFD4E80818F778083089593
:1064C0008F929F92AF92BF92CF92DF92EF92FF9204
:1064D0000F93CF93DF931F92CDB7DEB75C017B01A3
:1064E00049016B01C40ED51EF501808191810F9485
:1064F0000F2C8983002311F0F7018083BE016F5FA9
:106500007F4FC4010E94F5E0F501808191810196E1
:1065100091838083FFEFEF1AFF0AEC14FD0421F74B
:1065200080E00F90DF91CF910F91FF90EF90DF907F
:10653000CF90BF90AF909F908F9008950F93AB0135
:106540000091F90521E002272AEF35E0BC018AED30
:1065500095E00E9460320F910895009781F41092A7
:10656000900082E080939100109295001092940028
:10657000C19A8091710082608093710008950197A3
:1065800061F41092A00082E08093A1001092A50017
:106590001092A40089BB8093720008957F928F921D
:1065A0009F92AF92BF92CF92DF92EF92FF920F93A2
:1065B0001F93CF93DF93EC017B018881883108F032
:1065C000C3C090E0FC01EE0FFF1FE80FF91FEC5C69
:1065D000FD4E80818F770E9441E719821A8288815F
:1065E0002CE0622F0F94982C829FB001112430E090
:1065F00020E0AB01420F531FFA01EE0FFF1FE40F23
:10660000F51FEC5CFD4E908197FD08C02F5F3F4F5A
:106610002C30310571F790E00E94AD327880072D63
:1066200010E06801CC0CDD1CF601E00FF11FEC5C02
:10663000FD4E80818068808377FC86C080E2E8160A
:1066400082E0F8060CF03FC08A8128E532E0281B82
:10665000310987FD3395220F331F220F331F032E7D
:10666000000C440B550B898178E8872E912C881AF1
:10667000910887FD9394880C991C880C991C092C0F
:10668000000CAA08BB0860E070E0CB01F7FC0AC070
:10669000B701653B710514F064EB70E0072E000C48
:1066A000880B990B281939094A095B090F94252C85
:1066B00024EB30E040E050E00F94572C820E931E04
:1066C000A41EB51E740187E18715D8F0298188E8DA
:1066D00090E0821B910927FD9395880F991F880FE1
:1066E000991FE816F90604F502972FB7F894E6010A
:1066F000C00FD11FCC5CDD4E880F991F9A83898310
:106700002FBF62E370E080E090E0DF91CF911F91B6
:106710000F91FF90EF90DF90CF90BF90AF909F9040
:106720008F907F900C9439262A8188E592E0821B15
:10673000910927FD9395880F991F880F991FE816D7
:10674000F90694F6C701D0CFDF91CF911F910F9139
:10675000FF90EF90DF90CF90BF90AF909F908F9081
:106760007F900895CF93DF93EB01682F70E08DE762
:1067700092E10E94CE32688179818A819B81643F57
:1067800021E072078105910520F464EF71E080E05B
:1067900090E00E94392689B183FB882780F9DF9138
:1067A000CF910895CF93DF9300D01F92CDB7DEB77E
:1067B0008EEE92E0A0E0B0E089839A83AB83BC8345
:1067C000BE016F5F7F4F8AE50E94B2330F900F903A
:1067D0000F900F90DF91CF910895CF93DF9300D06A
:1067E0001F92CDB7DEB78EEE92E0A0E0B0E08983D5
:1067F0009A83AB83BC83BE016F5F7F4F8AE00E94A8
:10680000B2330F900F900F900F90DF91CF910895BA
:10681000CF93DF9300D01F92CDB7DEB784EF91E026
:10682000A0E0B0E089839A83AB83BC83BE016F5F35
:106830007F4F80EA0E94B2330F900F900F900F901D
:10684000DF91CF9108951F920F920FB60F921124EE
:106850000BB60F922F933F934F935F936F937F935A
:106860008F939F93AF93BF93EF93FF9348EA50E0CA
:1068700064EA70E081E090E00E945D26FF91EF9174
:10688000BF91AF919F918F917F916F915F914F9148
:106890003F912F910F900BBE0F900FBE0F901F9046
:1068A00018951F920F920FB60F9211240BB60F92EC
:1068B0002F933F934F935F936F937F938F939F9308
:1068C000AF93BF93EF93FF9348E950E064E970E022
:1068D00090E080E00E945D26FF91EF91BF91AF9123
:1068E0009F918F917F916F915F914F913F912F91E8
:1068F0000F900BBE0F900FBE0F901F9018959091A8
:10690000D10095FD0CC09091D00095FF08C08093F8
:10691000D6008091D00080648093D00008952091AB
:106920002E042F5F2F770FB607FC27C090912F04FE
:10693000921328C09091D00095FF1EC090912F0413
:1069400040912E04941306C09091D1009F7D9093A6
:10695000D10012C0E92FF0E0E25DFB4F32819F5F72
:106960009F773093D60090932F043091D0003064FD
:106970003093D000491741F3D9CF90912F0492134F
:1069800001C0FBCFE0912E04F0E0E25DFB4F82837B
:1069900020932E048091D10080628093D1000895CD
:1069A0008F929F92AF92BF92CF92DF92EF92FF921F
:1069B0000F931F93CF93DF937C0121E5E20EF11C2F
:1069C000D7014C914A3509F0A4C06C01B2E5CB0E59
:1069D000D11CF6013081353A09F09BC0EC01C05B57
:1069E000DF4F2881233008F494C08C0100561F4FDC
:1069F000D8014C93E15BFF4F308331962083EF54F5
:106A0000F1093081E05BFF4F30833038B1F43196CB
:106A1000AC54B1093C913083E854F109AF5ABF4FEF
:106A200050E040E02250330B42175307CCF48081F2
:106A300032968D934F5F5F4FF7CF233031F531386A
:106A400009F074C0FC01EC55FF4FDC01AC5ABF4F9C
:106A50002C9120833196885A9F4FDC018C91808342
:106A60004801B12CA12C888190E002968A159B05E3
:106A70000CF43FC0F40181914F010E947F340E94C9
:106A80000BE1FFEFAF1ABF0AEECF323821F5FC0160
:106A9000EC5AFF4F30814181E05BFF4F40833196DC
:106AA0003083DC01AA55BF4F50E040E02350330B48
:106AB00042175307ACF6FA01EE7FE45AFF4FE80F96
:106AC000F91F608171817C9311966C9311974E5FD1
:106AD0005F4F1296EDCF243019F6333809F6FC01DA
:106AE000EC5AFF4F20813181E05BFF4F30833196BC
:106AF000B0CF80E5DE011D928A95E9F78AE1F801C1
:106B000011928A95E9F78AE5D7018C9385EAF60117
:106B10008083DF91CF911F910F91FF90EF90DF90D5
:106B2000CF90BF90AF909F908F900895323809F02A
:106B300097CFADCFAF92BF92CF92DF92EF92FF92FD
:106B40000F931F93CF93DF93EC0184E6C82E80E26E
:106B5000D82EE12CF12C02E8A12C90E2B92E15E000
:106B60000093C613C092C713D092C813E092C91302
:106B7000F092CA13B092D013A092CF131093C31304
:106B800083E793E10E94D0348FEFC81AD80AE80A4D
:106B9000F80A88E7C81680E2D806E104F10401F794
:106BA00024E630E240E050E0BE0183E793E1DF916C
:106BB000CF911F910F91FF90EF90DF90CF90BF90FA
:106BC000AF900C9410E1CF92DF92EF92FF920F936F
:106BD0001F93CF93DF93CDB7DEB77C01CDB6DEB682
:106BE0000F943E2501962DB73EB7281B390B0FB6E3
:106BF000F8943EBF0FBE2DBF0DB71EB70F5F1F4FDE
:106C0000B701C8010F943725C8010E949A350FB605
:106C1000F894DEBE0FBECDBEDF91CF911F910F91D4
:106C2000FF90EF90DF90CF9008958F929F92AF9258
:106C3000BF92CF92DF92EF92FF920F931F93CF9369
:106C4000DF930E94F42C3AE0C32E30E2D32EE12CE5
:106C5000F12C15E002E846015701CAE0D0E010929D
:106C6000D0131092CF131093C3130093C6138092C6
:106C7000C7139092C813A092C913B092CA1383E7A6
:106C800093E10E94D03421978FEF881A980AA80ABE
:106C9000B80A209721F78AE0C80ED11CE11CF11C2C
:106CA00082EDC81680E2D806E104F104A1F6C12CF9
:106CB00020E2D22EE12CF12CD5E0C2E81092D013C4
:106CC0001092CF13D093C313C093C613C092C713AF
:106CD000D092C813E092C913F092CA1383E793E1EC
:106CE0000E94D0341092D0131092CF13D093C313BC
:106CF000C093C613D701C6018C529F4FAF4FBF4FF1
:106D00008093C7139093C813A093C913B093CA1369
:106D100083E793E10E94D0348FEFC81AD80AE80ABB
:106D2000F80A8AE0C81680E2D806E104F10431F6D8
:106D30009EEDC92E90E2D92EE12CF12CD5E0C2E8CF
:106D40001092D0131092CF13D093C313C093C613D5
:106D5000C092C713D092C813E092C913F092CA131D
:106D600083E793E10E94D0348FEFC81AD80AE80A6B
:106D7000F80A86EEC81680E2D806E104F10401F7AD
:106D8000CC24C39482E1D82EE12CF12C0AE010E04F
:106D9000D5E0C2E81093D0130093CF13D093C31360
:106DA000C093C613C092C713D092C813E092C91300
:106DB000F092CA1383E793E10E94D0341093D0136A
:106DC0000093CF13D093C313C093C613D701C6014A
:106DD0008096A11DB11D8093C7139093C813A093F3
:106DE000C913B093CA1383E793E10E94D0348FEFA5
:106DF000C81AD80AE80AF80A85E1C81682E1D80656
:106E0000E104F10439F682E190E09093D01380938D
:106E1000CF13D093C313C093C61384E190E1A0E0D5
:106E2000B0E08093C7139093C813A093C913B09395
:106E3000CA1383E793E1DF91CF911F910F91FF90E8
:106E4000EF90DF90CF90BF90AF909F908F900C9479
:106E5000D0341F920F920FB60F9211240BB60F92DF
:106E60002F938F939F93EF93FF9380912F04209103
:106E70002E04821306C08091D1008F7D8093D100B3
:106E800012C0E82FF0E0E25DFB4F92818F5F8F77B9
:106E90009093D60080932F049091D00090649093AB
:106EA000D000281741F3FF91EF919F918F912F917F
:106EB0000F900BBE0F900FBE0F901F9018951F9252
:106EC0000F920FB60F9211240BB60F920F931F93D0
:106ED0002F933F934F935F936F937F938F939F93E2
:106EE000AF93BF93CF93DF93EF93FF93C091D600FF
:106EF00000915205D091510511E01D0F1F73909123
:106F00002D04913108F09FC0E92FF0E08827E45765
:106F1000F84C8F4F0D94B82C9D37CC37DB37EA37C0
:106F2000F1372338F5372338F937FD37233801385F
:106F300005380938103823381B38C03229F028F5B5
:106F4000CA3011F0CD3031F5011731F0ED2FF0E0FE
:106F5000EF5AFA4FC283D12FD0935105FF91EF9191
:106F6000DF91CF91BF91AF919F918F917F916F9161
:106F70005F914F913F912F911F910F910F900BBEF9
:106F80000F900FBE0F901F901895CD3481F081E0C7
:106F9000CE3471F080E10CC0CA3338F4C033A0F6AF
:106FA000C03291F2CD32B1F7CFCFCD3499F782E034
:106FB00080932D04C9CFC13359F018F4C03221F2A7
:106FC000E9CF88E0C433A1F38BE0C83389F3E2CF83
:106FD00083E0EECF84E0C03359F386E0C13341F360
:106FE000D9CF85E0C833B1F6E3CF87E0C23391F65D
:106FF000DFCF89E0C13371F6DBCF8AE0C03351F6D1
:10700000D7CF8CE0C73331F6D3CF8DE0C63311F63E
:10701000CFCFC03209F498CF8EE0C33549F2BACF52
:1070200080ED8C0F8A3008F08FCF9FE090932D0475
:1070300080932C0489CFCA3019F0CD3009F084CF69
:1070400010922D0481CFCA3019F0CD3009F07CCFD9
:1070500080912D148823A1F3973089F038F495306E
:1070600079F710923C0210923E0CEACF9A3059F018
:107070009F3031F780912C040E94EF31E1CF81E005
:1070800080932806DDCF81E080932706D9CF9091A9
:10709000C00095FFFCCF8093C6000895CF93DF9387
:1070A000EC018991882319F00E944738FACF8DE0CE
:1070B0000E9447388AE0DF91CF910C944738CF92F5
:1070C000DF92EF92FF92CF936B017C01C42F4A3085
:1070D00069F4F7FE0BC0F094E094D094C094C11C06
:1070E000D11CE11CF11C8DE20E9447384C2FC701D6
:1070F000B601CF91FF90EF90DF90CF900C9485AACE
:10710000CF93DF93EC01FE0184912196882319F03F
:107110000E944738F8CFDF91CF910895CF93DF9346
:10712000D0912C118FE59CE10E9480388AE00E946A
:1071300047388091AB0C873009F449C083E08093D5
:10714000A60C81E080937E0280E190E09093D013C2
:107150008093CF1385E08093C313C2E8C093C61316
:1071600084E190E1A0E0B0E08093C7139093C8134E
:10717000A093C913B093CA1383E793E10E94D0345C
:1071800061E070E080E090E00E94D92C81E09AE517
:107190009093D0138093CF1385E390E09093D21314
:1071A0008093D11387E08093C313C093C61384E800
:1071B00090E0A0E0B0E08093C7139093C813A09331
:1071C000C913B093CA1383E793E10E94D03480912E
:1071D0002C11813089F1823061F50E94C62B6093B9
:1071E000C2057093C3058093C4059093C50581E0E3
:1071F00080932C110E9451FD6093BE057093BF05D2
:107200008093C0059093C105D23089F08091AB0680
:107210009091AC0601969093AC068093AB061092C9
:10722000CA051092CB051092CC051092CD0581E0D5
:1072300004C00E94F82BDBCF80E0DF91CF9108954E
:10724000CF93C82FCB010E94803883ED98E10E9434
:10725000803884EC98E1CC2311F089EC98E10E940D
:1072600080388AE0CF910C944738CF93DF9300D0D9
:107270001F92CDB7DEB784EF91E0A0E0B0E0898344
:107280009A83AB83BC83BE016F5F7F4F8CE30E9408
:10729000B23381EF98E10E9480388CB16BEE78E1D7
:1072A00085FB882780F90E9420398091030165EED3
:1072B00078E1869581700E94203989B16FED78E17F
:1072C00083FB882780F90E9420398CB166ED78E134
:1072D000829581700E9420394B9909C00E94ED333C
:1072E0000F900F900F900F90DF91CF9108950E9413
:1072F000D2330F900F900F900F90DF91CF910895A0
:1073000080912C118130C1F58FE998E10E9480387D
:107310008AE00E94473881E09AE59093D0138093E9
:10732000CF1387E590E09093D2138093D11387E039
:107330008093C31382E88093C61384E890E0A0E0B2
:10734000B0E08093C7139093C813A093C913B09370
:10735000CA1383E793E10E94D03482E080932C111A
:107360000E9451FD6093C6057093C7058093C805C0
:107370009093C90581E0089580E008950F931F93CD
:107380000E9451FD0091A6061091A7062091A80623
:107390003091A906011511052105310509F067C0D5
:1073A0002091A512222309F45FC0E091A31221507D
:1073B0002093A51221E02E0F2093A3123091A61244
:1073C000231302C01092A31224E0E29FF0011124C3
:1073D000E955FD4E00811181228133810093A2067F
:1073E0001093A3062093A4063093A506600F711F87
:1073F000811D911D6093A6067093A7068093A80631
:107400009093A9068091A4069091A506892B61F11D
:107410001FB7F8948EE898E10E9480388AE00E94B5
:10742000473884E096E09093D0138093CF1380EA9E
:1074300090E89093D2138093D11387E08093C31385
:1074400082E88093C61380EA90E0A0E0B0E08093E9
:10745000C7139093C813A093C913B093CA1383E7BB
:1074600093E10E94D0341FBF1F910F910895601BBC
:10747000710B820B930B97FDF7CF40981092A606E5
:107480001092A7061092A8061092A906EDCF0F93AE
:107490001F93CF93DF938C01EB019091A512209164
:1074A000A612921305C00E94BE390E944DC2F5CFAC
:1074B0008091A41234E0839FF0011124E955FD4E20
:1074C00011830083D383C2839F5F9093A5128F5F44
:1074D000281739F08093A412DF91CF911F910F915B
:1074E00008951092A412F8CFCF92DF92EF92FF92FC
:1074F0001F93CF93DF93182F662351F0109200054E
:107500001092FC041092FD041092FE041092FF04ED
:107510000E9451FD6B017C018091FC049091FD045F
:10752000A091FE04B091FF04A7019601281B390B1E
:107530004A0B5B0BDA01C901B7FD3DC02091000584
:1075400017FD13C0412F012E000C550B4C5F5F4FF0
:10755000822F022E000C990B4817590764F184EF13
:1075600091E0A0E0B0E0211724F488EE93E0A0E0E1
:10757000B0E08C0D9D1DAE1DBF1D8093FC0490934B
:10758000FD04A093FE04B093FF042170C22F30E0ED
:10759000D32F84E28C9FB0018D9F700D7C1B112432
:1075A00060597C4F82E390E00E94473A8091000549
:1075B0008F5F80930005DF91CF911F91FF90EF9037
:1075C000DF90CF900895CF93DF9300D01F92CDB777
:1075D000DEB784E198E10E9480388AE00E94473853
:1075E0008091AB0C8330D9F119821A821B821C82E4
:1075F00060E0CE0101960E94132C19821A821B8230
:107600001C8261E0CE0101960E94132C81E08093E0
:107610007D021092A50C80937E0281E09AE5909302
:10762000D0138093CF1383E390E09093D213809391
:10763000D11387E08093C31382E88093C61384E854
:1076400090E0A0E0B0E08093C7139093C813A0939C
:10765000C913B093CA1383E793E10E94D0340F900B
:107660000F900F900F90DF91CF9108956F927F92BE
:107670008F929F92AF92BF92CF92DF92EF92FF9242
:107680000F931F93CF93DF93CDB7DEB764970FB6F9
:10769000F894DEBF0FBECDBF1092D0008091D00015
:1076A00082608093D0001092D50080E18093D40056
:1076B0008091D10080618093D1008091D100886059
:1076C0008093D1008091D10080688093D100809117
:1076D000D1008F7D8093D1008AE58093C41380937D
:1076E000741385EA8093C51380937513E3E1F4E185
:1076F0008AE1DF011D928A95E9F78091A40C882325
:1077000009F473C283E090E09093D0138093CF1379
:1077100085E08093C31382E88093C6138FE190E1E4
:10772000A0E0B0E08093C7139093C813A093C9134F
:10773000B093CA1383E793E10E94D03484E690E0CB
:107740009093D0138093CF1305E00093C31312E8F6
:107750001093C61386E090E1A0E0B0E08093C713D9
:107760009093C813A093C913B093CA1383E793E10E
:107770000E94D0348BE090E09093D0138093CF138D
:107780000093C3131093C61380E092E1A0E0B0E031
:107790008093C7139093C813A093C913B093CA13CF
:1077A00083E793E10E94D0341092D0131092CF134C
:1077B0000093C3131093C61384E390E1A0E0B0E0FC
:1077C0008093C7139093C813A093C913B093CA139F
:1077D00083E793E10E94D0341092D0131092CF131C
:1077E0000093C3131093C6138AE390E1A0E0B0E0C6
:1077F0008093C7139093C813A093C913B093CA136F
:1078000083E793E10E94D0348091F3119091F411B9
:107810009093D0138093CF130093C3131093C61388
:1078200086E390E1A0E0B0E08093C7139093C81383
:10783000A093C913B093CA1383E793E10E94D03495
:1078400080918811909189119093D0138093CF13D8
:107850000093C3131093C6138CE390E1A0E0B0E053
:107860008093C7139093C813A093C913B093CA13FE
:1078700083E793E10E94D03482E090E09093D013AC
:107880008093CF130093C3131093C6138EE190E13E
:10789000A0E0B0E08093C7139093C813A093C913DE
:1078A000B093CA1383E793E10E94D03481E08093C0
:1078B0007D0270E6C72E70E1D72EE12CF12C1092DC
:1078C000D0131092CF130093C3131093C613C0921A
:1078D000C713D092C813E092C913F092CA1383E77A
:1078E00093E10E94D034BFEFCB1ADB0AEB0AFB0A0C
:1078F000E4E7CE16E0E1DE06E104F10401F7CE0193
:1079000001967C0184E1D7011D928A95E9F781E017
:107910008F9390E99F938F9398E69F938F939F9374
:1079200087EA93E09F938F93FF92EF920F944930F1
:1079300020E630E140E050E064EB73E083E793E160
:107940000E9410E12AE630E140E050E061EC73E093
:1079500083E793E10E9410E124E730E140E050E04A
:10796000B70183E793E10E9410E12EE730E140E0A8
:1079700050E06FEC73E083E793E10E9410E1109216
:10798000D0131092CF130093C3131093C6138EE03D
:1079900090E1A0E0B0E08093C7139093C813A09348
:1079A000C913B093CA1383E793E10E94D0341092B5
:1079B000D0131092CF130093C3131093C6138FE00C
:1079C00090E1A0E0B0E08093C7139093C813A09318
:1079D000C913B093CA1383E793E10E94D0340FB662
:1079E000F894DEBF0FBECDBF4AE0C42E40E2D42ED5
:1079F000E12CF12C55E0752E62E8662E4601570108
:107A00000AE010E01092D0131092CF137092C313BB
:107A10006092C6138092C7139092C813A092C913A4
:107A2000B092CA1383E793E10E94D0340150110948
:107A3000FFEF8F1A9F0AAF0ABF0A0115110511F750
:107A40008AE0C80ED11CE11CF11C92EDC91690E22F
:107A5000D906E104F10491F6C12C30E2D32EE12CD9
:107A6000F12C05E012E81092D0131092CF1300937E
:107A7000C3131093C613C092C713D092C813E092D9
:107A8000C913F092CA1383E793E10E94D034109295
:107A9000D0131092CF130093C3131093C613D701C2
:107AA000C6018C529F4FAF4FBF4F8093C713909327
:107AB000C813A093C913B093CA1383E793E10E943C
:107AC000D034AFEFCA1ADA0AEA0AFA0ABAE0CB16D9
:107AD000B0E2DB06E104F10431F62EEDC22E20E225
:107AE000D22EE12CF12C05E012E81092D013109266
:107AF000CF130093C3131093C613C092C713D09231
:107B0000C813E092C913F092CA1383E793E10E946D
:107B1000D034EFEFCE1ADE0AEE0AFE0AF6EECF16EA
:107B2000F0E2DF06E104F10401F7CC24C39482E122
:107B3000D82EE12CF12C9AE0A92EB12C05E012E808
:107B4000B092D013A092CF130093C3131093C61317
:107B5000C092C713D092C813E092C913F092CA130F
:107B600083E793E10E94D034B092D013A092CF1358
:107B70000093C3131093C613D701C6018096A11DAD
:107B8000B11D8093C7139093C813A093C913B093EA
:107B9000CA1383E793E10E94D0348FEFC81AD80A42
:107BA000E80AF80A95E1C91692E1D906E104F10460
:107BB00039F68AE797E10E9480388AE00E944738C8
:107BC00064960FB6F894DEBF0FBECDBFDF91CF91A4
:107BD0001F910F91FF90EF90DF90CF90BF90AF90EB
:107BE0009F908F907F906F90089582E090E08CCD71
:107BF0000E94363B10929A0581E080937E028CE2CF
:107C000098E10E9480388AE00C9447380F931F93C4
:107C1000CF938C01C62F84E294E10E948038C80182
:107C20000E9480388AE30E94473880E38C0F0E94CC
:107C300047388AE0CF911F910F910C94473887EA1B
:107C400095E10E94803860E087E995E10E94063E58
:107C500060E082E895E10E94063E61E08BE795E1F5
:107C60000E94063E61E080E795E10E94063E61E0E9
:107C700080E695E10E94063E60E087E595E10E947E
:107C8000063E61E08DE495E10E94063E61E083E4FA
:107C900095E10E94063E61E08CE395E10E94063E7C
:107CA00061E084E395E10E94063E61E086E295E1B1
:107CB0000E94063E61E088E195E10E94063E60E098
:107CC00089E095E10E94063E60E08BEF94E10E941E
:107CD000063E60E085EE94E10E94063E61E084EDA0
:107CE00094E10E94063E61E085EC94E10E94063E2C
:107CF00061E08EEB94E10E94063E60E087EB94E148
:107D00000E94063E61E08EEA94E10E94063E61E038
:107D100089E994E10E94063E61E08BE894E10E94CB
:107D2000063E61E088E794E10E94063E60E08BE653
:107D300094E10E94063E61E086E694E10E94063EE0
:107D400061E089E594E10E94063E60E085E494E10B
:107D50000E94063E60E082E394E10E94063E60E0FD
:107D60008CE394E10E94991D682F617089E294E18F
:107D70000C94063E80914B05827149F480914D052B
:107D80008C7829F480914E05837009F475C082E4E3
:107D90000E94771E882351F00E9445246093510C65
:107DA0007093520C8093530C9093540C83E50E9473
:107DB000771E882351F00E94CB246093810C70932E
:107DC000820C8093830C9093840C84E50E94771E30
:107DD000882351F00E94CB246093850C7093860C0D
:107DE0008093870C9093880C88E50E94771E8823E7
:107DF00051F00E94CB246093F4087093F5088093AF
:107E0000F6089093F70889E50E94771E882351F0C1
:107E10000E94CB246093F8087093F9088093FA08C5
:107E20009093FB088AE50E94771E8823B1F00E9498
:107E3000CB246093FC087093FD088093FE08909318
:107E4000FF082DEC3CEC4CEC5DE30F94F12518168B
:107E500024F088E99EE00E94803885E40E94771E25
:107E6000882351F00E94CB2460930009709301098C
:107E700080930209909303090895AF92BF92CF9225
:107E8000DF92EF920F931F93CF93DF935B01EA0191
:107E90006901882309F463C081E99EE00E9480386B
:107EA000F501608171818281938146E00E948DBAE3
:107EB000E1100BC088E89EE00E94803868817981DB
:107EC0008A819B8146E00E948DBA81E89EE00E94F3
:107ED0008038F601608171818281938143E00E9444
:107EE0008DBA8AE79EE00E948038F8016081718136
:107EF0008281938143E00E948DBA81E79EE00E94D7
:107F00008038F6012081318142815381F8016081FE
:107F10007181828193810F94C02C43E00E948DBABD
:107F2000EE20F9F08AE00E9447388CE59EE00E943E
:107F30008038688179818A819B8146E00E948DBA70
:107F40008AE00E9447388AE0DF91CF911F910F911C
:107F5000EF90DF90CF90BF90AF900C944738E11036
:107F6000E4CFDF91CF911F910F91EF90DF90CF90F1
:107F7000BF90AF9008950F931F93CF938C01C62F9E
:107F800089E798E00E948038C8010E948038CC239D
:107F900031F08AE0CF911F910F910C944738CF9127
:107FA0001F910F9108950E94A9E410923E0C109227
:107FB0003C020E940D32882351F08091391482FDD9
:107FC00006C08AE898E190938E0C80938D0C61E056
:107FD00083E898E10E94BB3F0C948E380F931F9367
:107FE000CF93DF938C016F3F19F410926D1160E015
:107FF00020916D11862F062E000C990B281719065B
:1080000009F08CF560936D1160E08DE498E10E94B9
:10801000BB3FC8010E9480388AE00E944738C801EF
:108020000F943E25800F911FEC01C01BD10BC03473
:10803000D1053CF00197FC012491207C2038D1F33C
:10804000F3CFDD27AE01B8018DE291E10F945F25FA
:10805000C35DDE4E18828DE291E1DF91CF911F91D9
:108060000F910C949A35DF91CF911F910F91089544
:1080700010923E0C10923C028091391480648093DF
:10808000391461E08BE598E10E94BB3F40E758E17D
:1080900068E778E185E00E942EE360E082E698E1FF
:1080A0000C94EE3F0F931F93CF938C01C62F60E08B
:1080B00083E898E00E94BB3FC8010E948038CC232F
:1080C00031F08AE0CF911F910F910C944738CF91F6
:1080D0001F910F91089561E08BE898E00C94524055
:1080E000EF92FF920F931F93CF937C018B01C42FCC
:1080F00060E083E898E00E94BB3FC7010E9480389F
:1081000080E20E944738C8010E948038CC2319F0D1
:108110008C2F0E9447388AE0CF911F910F91FF90DA
:10812000EF900C944738DF92EF92FF920F931F93DA
:10813000CF93DF93D82E7B018A01E9010E946B4027
:10814000D092991140E0B70184E799E00E94704015
:108150000115110531F040E0B8018DE699E00E946B
:108160007040209731F040E0BE018DE699E00E941A
:10817000704061E088E699E0DF91CF911F910F9107
:10818000FF90EF90DF900C945240AF92BF92CF924D
:10819000DF92EF92FF920F931F93CF93DF9386EEC0
:1081A00097E00E948038C0E0D7E0D15021F080E213
:1081B0000E944738FACF8C2F0E9467E1CF5FC5300D
:1081C00099F78AE00E94473807EA17E0C0E080E2AA
:1081D0000E9447388C2F0E9467E15801D5E080E269
:1081E0000E944738F501C080D180E280F380A7016A
:1081F0009601C701B6010F94B32F882369F180E27D
:108200000E9447388DE30E9447388DE30E9447382B
:108210008DE30E9447388DE30E9447388DE30E942A
:108220004738D150F4E1AF0EB11CD111D8CF8AE05C
:108230000E944738CF5F0C5F1F4FC53041F68AE080
:10824000DF91CF911F910F91FF90EF90DF90CF9032
:10825000BF90AF900C94473820E030E0A901C701EF
:10826000B6010F94212F87FD03C08BE20E9447388F
:1082700043E0C701B6010E948DBAD3CF811107C078
:108280008AEC9EE00E9480388AE00C9447388EEC9D
:108290009EE0F8CFCF93DF93EB010E948038CE01B0
:1082A000DF91CF910C9425E2CF93C62F0E948038A6
:1082B0008C2FCF910C9467E1CF92DF92EF92FF92D7
:1082C0006A017B010E94803842E0C701B601FF903D
:1082D000EF90DF90CF900C948DBACF92DF92EF9217
:1082E000FF926A017B010E9480384AE0C701B60113
:1082F000FF90EF90DF90CF900C945F38CF93DF9397
:10830000EB010E948038CE01DF91CF910C946EE199
:108310004F925F926F927F928F929F92AF92BF9295
:10832000CF92DF92EF92FF920F931F93CF93DF9341
:1083300000D000D01F921F92CDB7DEB78091990573
:1083400081110AC480919705909198059C012F5F37
:108350003F4F30939805209397058E3E924008F446
:10836000FBC38091F3119091F4119093D0138093FB
:10837000CF1305E00093C31312E81093C61386E3EE
:1083800090E1A0E0B0E08093C7139093C813A0934E
:10839000C913B093CA1383E793E10E94D03480914C
:1083A0008811909189119093D0138093CF130093EB
:1083B000C3131093C6138CE390E1A0E0B0E0809368
:1083C000C7139093C813A093C913B093CA1383E73C
:1083D00093E10E94D0348091F5119091F611909321
:1083E000D0138093CF130093C3131093C61384E369
:1083F00090E1A0E0B0E08093C7139093C813A093DE
:10840000C913B093CA1383E793E10E94D0348091DB
:108410008A1190918B119093D0138093CF13009376
:10842000C3131093C6138AE390E1A0E0B0E08093F9
:10843000C7139093C813A093C913B093CA1383E7CB
:1084400093E10E94D03481E08093990510929805C1
:10845000109297058091AB0C882339F10E942B1D57
:10846000811123C0809196058F5F8093960580913E
:108470009605853620F0109296051092AB0CE0918F
:10848000AB0CE150E73008F06AC00E2E000CFF0B79
:108490008827E25BFD4B8F4F0D94B82C5842A742C2
:1084A00073449F44E0441845AB4210929605DFCFD9
:1084B0000E94D12C882309F452C081E080937E026F
:1084C00086E098E10E9480388AE00E94473880E187
:1084D00090E09093D0138093CF1385E08093C313E3
:1084E00012E81093C61384E190E1A0E0B0E080931D
:1084F000C7139093C813A093C913B093CA1383E70B
:1085000093E10E94D03481E09AE59093D013809358
:10851000CF1386E390E09093D2138093D11387E03A
:108520008093C3131093C61384E890E0A0E0B0E0FA
:108530008093C7139093C813A093C913B093CA1321
:1085400083E793E10E94D0341092AB0C08C00E94E4
:10855000D12C882321F00E942B1D8823A9F3809120
:108560007E02882309F433C780919A058111C0C225
:1085700084E096E09093D0138093CF1380EA90E844
:108580009093D2138093D11317E01093C31302E892
:108590000093C61380EA90E0A0E0B0E08093C71398
:1085A0009093C813A093C913B093CA1383E793E1C0
:1085B0000E94D0348091790290917A02A0917B023E
:1085C000B0917C020097A105B10509F03FC210925D
:1085D000D0131092CF1315E01093C3130093C6135A
:1085E0008AE890E1A0E0B0E08093C7139093C813AD
:1085F000A093C913B093CA1383E793E10E94D034C8
:1086000089E090E09093D0138093CF131093C3131D
:108610000093C6138CE890E1A0E0B0E08093C7130C
:108620009093C813A093C913B093CA1383E793E13F
:108630000E94D0348091790290917A02A0917B02BD
:10864000B0917C020097F1E0AF07B10508F441C298
:10865000B093D013A093CF139093D2138093D113E0
:1086600087E08093C31382E88093C61388E890E183
:10867000A0E0B0E08093C7139093C813A093C913F0
:10868000B093CA1383E793E10E94D03480917902BA
:1086900090917A02A0917B02B0917C02BA2FA92F0F
:1086A000982F8827009721E0A207B10508F417C288
:1086B000B093D013A093CF139093D2138093D11380
:1086C00087E08093C31312E81093C61381EA90E009
:1086D000A0E0B0E08093C7139093C813A093C91390
:1086E000B093CA1383E793E10E94D0348091400C89
:1086F000882309F4FAC183E090E09093D01380932B
:10870000CF1385E08093C3131093C61385E490E1E3
:10871000A0E0B0E08093C7139093C813A093C9134F
:10872000B093CA1383E793E10E94D03480919A05F5
:10873000875E80939A0520919A05822F90E02536D6
:1087400008F021C29093D0138093CF1385E08093DB
:10875000C31382E88093C61380E090E1A0E0B0E00C
:108760008093C7139093C813A093C913B093CA13EF
:1087700083E793E10E94D0340E942B1D811114C223
:108780000E940D32811105C090919D0591FD0E94BE
:108790002B1D90919D0580FB91F990939D0591FD76
:1087A00003C28091391482FDFFC180912C11815048
:1087B000823008F4F9C160918A1170918B11072EF3
:1087C000000C880B990B0F94F8256B017C0120E0BD
:1087D00030E0A9010F94F125882309F4BBC660910C
:1087E000881170918911072E000C880B990B0F943A
:1087F000F8252B013C0120E030E040E050E4C701C7
:10880000B6010F94C02CA30192010F94212F1816CA
:108810000CF4C2C66091F3117091F411072E000C94
:10882000880B990B0F94F8256D837E838F8398872F
:108830006091F5117091F611072E000C880B990BC1
:108840000F94F8254B015C0120E030E040E251E458
:108850000F94C02C2D813E814F8158850F94212F7C
:1088600018160CF499C620E030E040E050E4C7014F
:10887000B6010F94C12CA30192010F94F12587FD3D
:1088800010C020E030E040E251E4C501B4010F9493
:10889000C12C2D813E814F8158850F94F12587FF92
:1088A0006AC684E190E09093D0138093CF1385E063
:1088B0008093C31382E88093C61384E190E1A0E023
:1088C000B0E08093C7139093C813A093C913B093DB
:1088D000CA1383E793E10E94D0348091A60C8111E2
:1088E0007CC682E07AC688EF97E10E9480388AE0F1
:1088F0000E94473881E09AE59093D0138093CF137C
:1089000080E490E09093D2138093D11317E01093FA
:10891000C31382E88093C61384E890E0A0E0B0E03F
:108920008093C7139093C813A093C913B093CA132D
:1089300083E793E10E94D0341093AB0C10CE80916A
:10894000950C882309F40BCE0E94D12C882309F4BE
:1089500006CE0E942B1D811102CE8AEE97E10E9465
:1089600080388AE00E9447388091960C90E0B0E011
:10897000A0E0895B9F4FAE4FB54A21E03AE53093C6
:10898000D0132093CF139093D2138093D11387E009
:108990008093C31382E88093C61384E890E0A0E03C
:1089A000B0E08093C7139093C813A093C913B093FA
:1089B000CA1383E793E10E94D0341092950CC4CD82
:1089C0000E94D12C882309F4CACD0E942B1D81114D
:1089D000C6CD81E080937E021092AB0C8CED97E1C6
:1089E0000E9480388AE00E94473881E09AE590939F
:1089F000D0138093CF138EE490E09093D2138093A2
:108A0000D11387E08093C31382E88093C61384E870
:108A100090E0A0E0B0E08093C7139093C813A093B8
:108A2000C913B093CA1383E793E10E94D03497CD62
:108A30000E942B1D811193CD19821A821B821C82E8
:108A400062E0CE0101960E94F6F47ECD0196A11D52
:108A5000B11D35E0B695A795979587953A95D1F7CD
:108A60000197A109B1090097E1E0AE07B10548F10E
:108A7000B093D013A093CF139093D2138093D113BC
:108A80001093C31312E81093C6138AE890E1A0E094
:108A9000B0E08093C7139093C813A093C913B09309
:108AA000CA1383E793E10E94D03488E090E090936A
:108AB000D0138093CF1385E08093C3131093C61314
:108AC000A9CD9093D0138093CF1385E08093C313E7
:108AD000D9CF9093D0138093CF1385E0C2CD9093DC
:108AE000D0138093CF1385E0ECCD82E090E005CEEB
:108AF0008A3F08F020CE8EEF80939A058BEC97E1A9
:108B00000E9480388AE00E94473881E080937E028C
:108B100081E09AE59093D0138093CF138DE290E09B
:108B20009093D2138093D11387E08093C31382E88C
:108B30008093C61384E890E0A0E0B0E08093C71370
:108B40009093C813A093C913B093CA1383E793E11A
:108B50000E94D0341092990528960FB6F894DEBF83
:108B60000FBECDBFDF91CF911F910F91FF90EF907E
:108B7000DF90CF90BF90AF909F908F907F906F903D
:108B80005F904F900895845691099093D0138093ED
:108B9000CF1385E08093C31382E88093C61381E0EE
:108BA00090E1A0E0B0E0DCCD8CE090E09093D013B9
:108BB0008093CF1315E01093C31382E88093C613FC
:108BC00084E190E1A0E0B0E08093C7139093C813D4
:108BD000A093C913B093CA1383E793E10E94D034E2
:108BE0000E94C62B20E13EE040E050E00F94352C7F
:108BF0002115310581E04807510508F470C05093F4
:108C0000D0134093CF133093D2132093D11387E026
:108C10008093C31312E81093C61380E190E1A0E0A3
:108C2000B0E08093C7139093C813A093C913B09377
:108C3000CA1383E793E10E94D0340E94C62B20E13F
:108C40003EE040E050E00F94352C2CE330E040E073
:108C500050E00F94352C3093D0132093CF1305E0C0
:108C60000093C3131093C61382E190E1A0E0B0E03B
:108C70008093C7139093C813A093C913B093CA13DA
:108C800083E793E10E94D0340E941B32882309F4C9
:108C90005CC48F5F80939505E82EF12C833330F50B
:108CA000EE0CFF1CF092D013E092CF130093C3138D
:108CB0001093C6138EE090E1A0E0B0E08093C7135C
:108CC0009093C813A093C913B093CA1383E793E199
:108CD0000E94D0341092D0131092CF132BC0309337
:108CE000D0132093CF131093C31394CF84E690E056
:108CF0009093D0138093CF130093C3131093C61394
:108D00008EE090E1A0E0B0E08093C7139093C81389
:108D1000A093C913B093CA1383E793E10E94D034A0
:108D2000A2E3EA1AA0E8FA0AEE0CFF1CF092D013B4
:108D3000E092CF130093C3131093C6138FE090E11A
:108D4000A0E0B0E08093C7139093C813A093C91319
:108D5000B093CA1383E793E10E94D0340E941B3280
:108D600090E09093D0138093CF1385E08093C3134A
:108D700082E88093C61386E190E1A0E0B0E08093A2
:108D8000C7139093C813A093C913B093CA1383E772
:108D900093E10E94D03420E030E0A9016091881274
:108DA0007091891280918A1290918B120F94C12C2C
:108DB00020E030E048EC52E40F9457260F942D2E1B
:108DC0007093D0136093CF1305E00093C31312E8A0
:108DD0001093C61386E290E1A0E0B0E08093C71341
:108DE0009093C813A093C913B093CA1383E793E178
:108DF0000E94D03480917502909176029093D013A6
:108E00008093CF130093C3131093C61380E093E1B4
:108E1000A0E0B0E08093C7139093C813A093C91348
:108E2000B093CA1383E793E10E94D03420E030E08E
:108E300040E251E46091550C7091560C8091570CB2
:108E40009091580C0F9457260F94342E7093D01392
:108E50006093CF130093C3131093C61382E492E17F
:108E6000A0E0B0E08093C7139093C813A093C913F8
:108E7000B093CA1383E793E10E94D03420E030E03E
:108E800040E251E46091590C70915A0C80915B0C56
:108E900090915C0C0F9457260F94342E7093D0133E
:108EA0006093CF130093C3131093C61386E492E12B
:108EB000A0E0B0E08093C7139093C813A093C913A8
:108EC000B093CA1383E793E10E94D03420E030E0EE
:108ED00040E251E460915D0C70915E0C80915F0CFA
:108EE0009091600C0F9457260F94342E7093D013EA
:108EF0006093CF130093C3131093C6138AE492E1D7
:108F0000A0E0B0E08093C7139093C813A093C91357
:108F1000B093CA1383E793E10E94D03420E030E09D
:108F200040E251E46091610C7091620C8091630C9D
:108F30009091640C0F9457260F94342E7093D01395
:108F40006093CF130093C3131093C6138EE492E182
:108F5000A0E0B0E08093C7139093C813A093C91307
:108F6000B093CA1383E793E10E94D03420E030E04D
:108F700048EC52E4609180127091811280918212CB
:108F8000909183120F9457260F942D2E7093D01327
:108F90006093CF130093C3131093C61386E392E13B
:108FA000A0E0B0E08093C7139093C813A093C913B7
:108FB000B093CA1383E793E10E94D03420E030E0FD
:108FC00048EC52E46091841270918512809186126F
:108FD000909187120F9457260F942D2E7093D013D3
:108FE0006093CF130093C3131093C6138AE392E1E7
:108FF000A0E0B0E08093C7139093C813A093C91367
:10900000B093CA1383E793E10E94D0348091850224
:10901000909186029093D0138093CF130093C31343
:109020001093C61382E592E1A0E0B0E08093C713ED
:109030009093C813A093C913B093CA1383E793E125
:109040000E94D03480918302909184029093D01337
:109050008093CF130093C3131093C61384E592E15A
:10906000A0E0B0E08093C7139093C813A093C913F6
:10907000B093CA1383E793E10E94D03420E030E03C
:1090800040E251E46091F8117091F9118091FA1168
:109090009091FB110F9457260F94342E7093D01398
:1090A0006093CF130093C3131093C61386E592E128
:1090B000A0E0B0E08093C7139093C813A093C913A6
:1090C000B093CA1383E793E10E94D0342CEA35ECC5
:1090D00047E25EE36091FC117091FD118091FE11F9
:1090E0009091FF110F94BB2D20E030E040E251E45D
:1090F0000F9457260F94342E7093D0136093CF1390
:109100000093C3131093C6138AE592E1A0E0B0E088
:109110008093C7139093C813A093C913B093CA1335
:1091200083E793E10E94D0342CEA35EC47E25EE31A
:1091300060910012709101128091021290910312BD
:109140000F94572620E030E040E251E40F94572678
:109150000F94342E7093D0136093CF130093C313E6
:109160001093C6138EE592E1A0E0B0E08093C713A0
:109170009093C813A093C913B093CA1383E793E1E4
:109180000E94D03420E030E040E251E460918D1143
:1091900070918E1180918F11909190110F9457269C
:1091A0000F94342E7093D0136093CF130093C31396
:1091B0001093C61382E692E1A0E0B0E08093C7135B
:1091C0009093C813A093C913B093CA1383E793E194
:1091D0000E94D0342CEA35EC47E25EE360919111B5
:1091E0007091921180919311909194110F94BB2DD5
:1091F00020E030E040E251E40F9457260F94342EE3
:109200007093D0136093CF130093C3131093C613BE
:1092100086E692E1A0E0B0E08093C7139093C81374
:10922000A093C913B093CA1383E793E10E94D0348B
:109230002CEA35EC47E25EE360919511709196114E
:1092400080919711909198110F94572620E030E06B
:1092500040E251E40F9457260F94342E7093D013AC
:109260006093CF130093C3131093C6138AE692E161
:10927000A0E0B0E08093C7139093C813A093C913E4
:10928000B093CA1383E793E10E94D03480919F0C7E
:10929000811105C08091A10C882309F46DC06091F3
:1092A000F3117091F411072E000C880B990B0F9499
:1092B000F82520E030E048EC52E40F9457266B018B
:1092C0007C016091F5117091F611072E000C880B4E
:1092D000990B0F94F8259B01AC01C701B6010F94BF
:1092E000BB2D0F94342E6536710510F064E670E0E6
:1092F0007093D0136093CF1305E00093C31312E86B
:109300001093C61384E290E1A0E0B0E08093C7130D
:109310009093C813A093C913B093CA1383E793E142
:109320000E94D0346091F3117091F411072E000C5B
:10933000880B990B0F94F8256B017C0120E030E03D
:109340004AE253E40F94212F181624F480919F0CC5
:10935000811146C16091F5117091F611072E000C34
:10936000880B990B0F94F8259B01AC01C701B6013E
:109370000F94212F87FFAFC18091950C882339F17D
:109380008091940C91E0980F9093940C90E09093BE
:10939000D0138093CF1385E08093C31382E880932A
:1093A000C61382E490E1A0E0B0E08093C7139093ED
:1093B000C813A093C913B093CA1383E793E10E9423
:1093C000D0348091940C8A3010F01092940C0E944A
:1093D0005C2C882309F4B5C16091A90C7091AA0C8A
:1093E000EE24E394F12C61157105A9F090E080E082
:1093F0000F94F62520E030E040E85EE30F94572616
:109400000F949F2D20E030E040E85FE30F94C12CE3
:109410000F94342E7B0101E010E080918F0C8111BC
:1094200002C010E000E08091B7129091B8128F3F17
:10943000980711F40E94E2B39093B8128093B71288
:10944000080F191FB80190E080E00F94F62520E086
:1094500030E040E85EE30F9457260F949F2D4B01B8
:109460005C01F092D013E092CF1305E00093C31398
:1094700012E81093C61380E193E1A0E0B0E080937E
:10948000C7139093C813A093C913B093CA1383E76B
:1094900093E10E94D034C501B4010F94342E70932F
:1094A000D0136093CF130093C3131093C61382E1BC
:1094B00093E1A0E0B0E08093C7139093C813A0930A
:1094C000C913B093CA1383E793E10E94D03403E138
:1094D00014E1AAE1FA2E8091510590915205209154
:1094E000930530919405891B8F7309F449C12A3182
:1094F00031050CF0DBC190915105809152054FEF81
:109500005FEF981749F0E82FF0E0EF5AFA4F4281E9
:109510008F5F8F7380935205F901ED5EFB4E4083A0
:10952000809113148A3509F0B3C162E070E080E0E5
:1095300090E00E94D92C809193059091940501961A
:109540009093940580939305C6CF1092D0131092F8
:10955000CF13ACCB6091F5117091F611072E000C72
:10956000880B990B0F94F82520E030E0A9010F94A7
:10957000F125811134C98CE090E09093D013809351
:10958000CF1385E08093C31382E88093C61384E1F0
:1095900090E1A0E0B0E0F3CB8DE090E09093D013A9
:1095A0008093CF1385E08093C31382E88093C61322
:1095B00084E190E1A0E0B0E08093C7139093C813DA
:1095C000A093C913B093CA1383E793E10E94D034E8
:1095D0008091A60C811101C081E08093A60CDBCBA9
:1095E00010929F0C20E030E040E251E46091970C33
:1095F0007091980C8091990C90919A0C0F94572629
:109600000F942D2E7093D0136093CF130093C31338
:109610001093C61384E590E1A0E0B0E08093C713F7
:109620009093C813A093C913B093CA1383E793E12F
:109630000E94D03420E030E040E251E460919B0C85
:1096400070919C0C80919D0C90919E0C0F945726CC
:109650000F942D2E7093D0136093CF130093C313E8
:109660001093C61388E590E1A0E0B0E08093C713A3
:109670009093C813A093C913B093CA1383E793E1DF
:109680000E94D0348AEA97E10E9480388AE00E94E2
:10969000473881E09AE59093D0138093CF1381E40B
:1096A00090E09093D2138093D11387E08093C313FB
:1096B0001093C61384E890E0A0E0B0E08093C71355
:1096C0009093C813A093C913B093CA1383E793E18F
:1096D0000E94D03451CE6091A10C662309F44CCE87
:1096E000062E000C770B81E997E10E947E418AE00B
:1096F0000E9447381092A10C84E090E09093D01320
:109700008093CF1385E08093C31312E81093C613A0
:109710008EE890E1A0E0B0E08093C7139093C81367
:10972000A093C913B093CA1383E793E10E94D03486
:1097300081E09AE59093D0138093CF1383E590E076
:10974000B0CF1092D0131092CF1305E00093C31343
:1097500012E81093C61380E193E1A0E0B0E080939B
:10976000C7139093C813A093C913B093CA1383E788
:1097700093E10E94D0341092D0131092CF1393CE65
:10978000121613060CF492C08091771390917813FF
:10979000A0917913B0917A138C34E0E19E07A10572
:1097A000B10509F4D7C98A349041A105B10509F47E
:1097B000D1C920E030E040E251E460916102709153
:1097C000620280916302909164020F9457260F9475
:1097D0002D2E7093D0136093CF1305E00093C31325
:1097E00012E81093C61388E490E1A0E0B0E0809303
:1097F000C7139093C813A093C913B093CA1383E7F8
:1098000093E10E94D03420E030E040E251E46091E6
:1098100065027091660280916702909168020F94D0
:1098200057260F942D2E7093D0136093CF1300936F
:10983000C3131093C6138AE490E1A0E0B0E08093D4
:10984000C7139093C813A093C913B093CA1383E7A7
:1098500093E10E94D03420E030E040E251E4609196
:10986000690270916A0280916B0290916C020F9470
:1098700057260F942D2E7093D0136093CF1300931F
:10988000C3131093C6138CE490E1A0E0B0E056C976
:10989000121613060CF01FCEF8012F2D11922A95E7
:1098A000E9F7109294051092930515CE90917413D8
:1098B00080911314981321C0909175138091141402
:1098C00098131BC023303105C4F090911514909368
:1098D000731380911614809376139330D1F4982FDC
:1098E0009D7F9038B1F4909117149F3409F059C0BE
:1098F000909118149B3409F054C0E3E1F4E18AE13B
:10990000DF011D928A95E9F7109294051092930554
:109910003BCF833809F045C08091171490911814FB
:10992000982789279827B0E0A0E080937713909339
:109930007813A0937913B0937A13C0901914D12C93
:10994000F12CE12CC0927B13D0927C13E0927D131A
:10995000F0927E132AE134E140E050E0BA014C1568
:109960005D056E057F0508F04AC0DB01CA01B695AA
:10997000A795979587950696880F991FFC01ED5836
:10998000FC4ED9018C9111969C91892798278927A3
:10999000918380834E5F5F4F6F4F7F4F2E5F3F4FAE
:1099A000DECF813861F58091171490E0B0E0A0E03F
:1099B0008093771390937813A0937913B0937A13CD
:1099C00080911814482F50E070E060E040937B13C2
:1099D00050937C1360937D1370937E13A9E1B4E1DF
:1099E000EFE7F3E190E030E020E08217930739F0F1
:1099F0004D9150E0419351932F5F3F4FF6CFE3E1FC
:109A0000F4E18AE1DF011D928A95E9F7109294054D
:109A1000109293050E9401FEB7CE3F924F925F9243
:109A20006F927F928F929F92AF92BF92CF92DF926E
:109A3000EF92FF920F931F93CF93DF9380914D0589
:109A400087FD38C080914E058370A1F5C0918C12BE
:109A5000D0918D12488159816A817B818BE197E198
:109A60000E945C414C815D816E817F818EE69FE228
:109A70000E945C41409188125091891260918A1233
:109A800070918B128BE69FE20E945C418AE0DF912D
:109A9000CF911F910F91FF90EF90DF90CF90BF90EB
:109AA000AF909F908F907F906F905F904F903F907E
:109AB0000C944738609080127090811280908212CE
:109AC00090908312A0908412B0908512009186121B
:109AD00010918712C0908812D0908912E0908A125B
:109AE000F0908B1288E50E94C51EC82F882309F4C8
:109AF0009AC00E94CB24362E472E582ED92F20E014
:109B000030E044EB53EC0F94212F87FD0DC020E093
:109B100030E044EB53E4632D742D852D9D2F0F947D
:109B2000F12518160CF081C068E671E088E097E135
:109B30000E947E4168E671E083E097E10E947E41E9
:109B400080E097E10E948038C0E089E50E94C51E50
:109B5000882361F10E94CB24362E472E582ED92F10
:109B600020E030E044EB53EC0F94212F87FD0DC033
:109B700020E030E044EB53E4632D742D852D9D2FC0
:109B80000F94F12518160CF055C068E671E08DEEC3
:109B900096E10E947E4168E671E088EE96E10E94BF
:109BA0007E4185EE96E10E948038C0E08AE50E9401
:109BB000C51E882309F443C00E94CB246B017C019D
:109BC00020E030E040E151EC0F94212F87FD0AC0E6
:109BD00020E030E040E151E4C701B6010F94F125E7
:109BE00018166CF567EF7FEF83ED96E10E947E41DA
:109BF00069E070E08EEC96E10E947E418BEC96E18C
:109C0000DF91CF911F910F91FF90EF90DF90CF9058
:109C1000BF90AF909F908F907F906F905F904F908C
:109C20003F900C948038C1E090CF632C742C852C2D
:109C30009D2E8BCFA32CB42C052D1D2FB7CFCC235D
:109C4000E1F0C301D4018093801290938112A0931C
:109C50008212B0938312C501D8018093841290932D
:109C60008512A0938612B0938712C0928812D09268
:109C70008912E0928A12F0928B12DF91CF911F919C
:109C80000F91FF90EF90DF90CF90BF90AF909F909B
:109C90008F907F906F905F904F903F9008958FEDE1
:109CA00097E00C94803889ED97E00C94803884E636
:109CB00090E09093DB058093DA051092FB051092FB
:109CC000FA050C94D4DBEF92FF920F931F93CF937E
:109CD000DF93CDB7DEB762970FB6F894DEBF0FBE45
:109CE000CDBF0E94462A882309F43FC04EEF53E0BF
:109CF00082FF02C042EE53E02EEF33E081FF02C04C
:109D000024EE33E080FD2EC08EEF93E05F934F93FF
:109D10003F932F939F938F9385E499E19F938F9324
:109D20008E010F5F1F4F1F930F930F9488250E9482
:109D3000534EC8010E944E38C8010E9471E40FB60C
:109D4000F894DEBF0FBECDBF81E062960FB6F894E7
:109D5000DEBF0FBECDBFDF91CF911F910F91FF905E
:109D6000EF90089586EE93E0D1CF80E0EECFCF92D2
:109D7000DF92EF92FF928AE50E94C51E882309F4C4
:109D80005AC00E94CB2420E030E040E050EC0F9419
:109D9000F125C12CD12CE12C90ECF92E87FD0FC0C0
:109DA0000E94CB2420E030E040E050E40F94212FCB
:109DB00018160CF462C00E94CB246B017C01209128
:109DC0005D0C30915E0C40915F0C5091600CC701AE
:109DD000B6010F9457260F942D2ECB010E948AFDB9
:109DE00080E50E94771E81114EC0A7019601609107
:109DF00088127091891280918A1290918B120F941F
:109E0000C12C609388127093891280938A12909368
:109E10008B120E94534E409188125091891260918A
:109E20008A1270918B128CEB96E10E945C418AE061
:109E30000E94473805C083E50E94C51E8111A1CF4D
:109E400080914D0587FD24C080914E05837001F5FA
:109E50000E94534E409188125091891260918A124B
:109E600070918B128DEA96E10E945C418AE0FF902E
:109E7000EF90DF90CF900C944738C12CD12CE12C7F
:109E800080E4F82E9CCF0E9493248111AECFD8CFCE
:109E900082E50E94771E8111DBCFFF90EF90DF906B
:109EA000CF900895CF9384E50E94C51EC0E088231B
:109EB000D9F00E947324C82F1816B4F40E94534E90
:109EC0008DE40E94473880914805909149050E9491
:109ED00025E26C2FCC0F770B88EA9FE00E947E4131
:109EE0008AE00E944738CFEF8C2FCF9108954F9290
:109EF0005F926F927F928F929F92AF92BF92CF921A
:109F0000DF92EF92FF92CF93DF93CDB7DEB72C971E
:109F10000FB6F894DEBF0FBECDBF4090E70850905B
:109F2000E8086090E9087090EA08209147023091B3
:109F300048024091490250914A02C301B2010F9474
:109F4000C12C69837A838B839C838090EB089090EB
:109F5000EC08A090ED08B090EE0820914B023091F3
:109F60004C0240914D0250914E02C501B4010F9434
:109F7000C12C6D837E838F839887C090EF08D0902B
:109F8000F008E090F108F090F20820914F02309133
:109F900050024091510250915202C701B6010F94F4
:109FA000C12C69877A878B879C87209153023091D7
:109FB00054024091550250915602C301B2010F94D0
:109FC000C12C2B013C012091570230915802409145
:109FD000590250915A02C501B4010F94C12C4B0192
:109FE0005C0120915B0230915C0240915D025091D6
:109FF0005E02C701B6010F94C12C6B017C010E9467
:10A00000534E83EE9EE00E94803883E50E94771EC7
:10A01000882321F00E949324809345028091450279
:10A02000811151C08AEC9EE00E9480388BED9EE049
:10A030000E94803849815A816B817C8183E19EE155
:10A040000E945C414D815E816F8178858EE69FE242
:10A050000E945C4149855A856B857C858BE69FE231
:10A060000E945C4189ED9EE00E94803881ED9EE077
:10A070000E948038B301A20183E19EE10E945C410D
:10A08000B501A4018EE69FE20E945C41B701A601E2
:10A090008BE69FE20E945C418AE02C960FB6F89412
:10A0A000DEBF0FBECDBFDF91CF91FF90EF90DF906D
:10A0B000CF90BF90AF909F908F907F906F905F9068
:10A0C0004F900C9447388EEC9EE0AECF5F926F922B
:10A0D0007F928F929F92AF92BF92CF92DF92EF9238
:10A0E000FF920F931F93CF93DF931F92CDB7DEB7ED
:10A0F0007C0139018B015B01A40EB51ED12CC12C52
:10A10000A016B10609F450C0F70180809180F801D3
:10A1100051908F015982C4010F940F2C5816B9F138
:10A12000652DC4010F94172CFFEFCF1ADF0AC6016B
:10A130008F779927892B21F162E070E080E090E031
:10A140000E941EFDC4010F940F2C99818917F9F00C
:10A150000E94534E8FE694E00E94803881E00F9079
:10A16000DF91CF911F910F91FF90EF90DF90CF90F3
:10A17000BF90AF909F908F907F906F905F90089569
:10A1800062E070E080E090E00E943926DBCFBE0103
:10A190006F5F7F4FC3010E94F5E0F70180819181DD
:10A1A000019691838083ACCF80E0D9CFDF92EF928C
:10A1B000FF920F931F93CF93DF93CDB7DEB7CA5AA9
:10A1C000D1090FB6F894DEBF0FBECDBFCF55DF4F1C
:10A1D000188219821A821B82C15AD0408091E803EA
:10A1E0009091E903A091EA03B091EB03CB55DF4FC7
:10A1F00088839983AA83BB83C55AD04084E690E0C4
:10A200009093DB058093DA051092FB051092FA0516
:10A210001092FC052AEF35E044E050E0BE016B559A
:10A220007F4F8AED95E00E9466508091DA0590910B
:10A23000DB0502969093DB058093DA051092FB050F
:10A240001092FA0581E0C655DF4F8883CA5AD04084
:10A25000CE0186559F4F0E94F9D12AEF35E048E4A0
:10A2600050E061E47CE08AED95E00E9466502AEFC0
:10A2700035E040E150E064EF78E08AED95E00E943F
:10A2800066508AE097EDA3EABCE3CF55DF4F8883A1
:10A290009983AA83BB83C15AD040CE018F559F4F6B
:10A2A0000E94F0D18DE198E00E940BD286E292E00C
:10A2B0000E9402D282E292E00E94F0D18091E308F3
:10A2C0009091E408A091E508B091E60889839A830B
:10A2D000AB83BC838E010F5F1F4FC8010E94F0D17A
:10A2E000CF55DF4F188219821A821B82C15AD04083
:10A2F0007E018DE6E80EF11C83E0D7018C93898303
:10A30000CE018F559F4F0E94F0D1C7010E94F9D115
:10A31000C8010E94F9D14AE0D42EDA94DD2031F050
:10A32000CE018F559F4F0E94F0D1F7CF80E892E188
:10A330000E940BD2CF55DF4F188219821A821B82DE
:10A34000C15AD0403AE0D32EDA94DD2031F0CE016C
:10A350008F559F4F0E94F0D1F7CF85E0D82ED9823C
:10A36000F701D082C8010E94F9D1C7010E94F9D13A
:10A370002AEF35E048E050E06DEE75E08AED95E0BB
:10A380000E9466502AEF35E048E050E065EE75E047
:10A390008AED95E00E9466502AEF35E044E650E0F1
:10A3A00067EA77E08AED95E00E94665019828FEFA8
:10A3B000D7018C93C8010E9402D2C7010E94F9D133
:10A3C0002AEF35E044E050E064EF72E08AED95E07A
:10A3D0000E9466508091BE068983C8010E9402D205
:10A3E000198A1A8A1B8A1C8A80E090E0A0E8BFE3E1
:10A3F0008D879E87AF87B88B8091F8119091F91166
:10A40000A091FA11B091FB1189839A83AB83BC832D
:10A410002CEA35EC47E25EE36091FC117091FD118E
:10A420008091FE119091FF110F94BB2D6D837E835F
:10A430008F8398872CEA35EC47E25EE36091001247
:10A440007091011280910212909103120F9457267D
:10A4500069877A878B879C872AEF35E044E150E053
:10A46000B8018AED95E00E94665084E190E09A83FD
:10A470008983C8010E94DED180918D1190918E1147
:10A48000A0918F11B091901189839A83AB83BC8383
:10A490002CEA35EC47E25EE36091911170919211E4
:10A4A00080919311909194110F94BB2D6D837E83B5
:10A4B0008F8398872CEA35EC47E25EE36091951133
:10A4C0007091961180919711909198110F94572641
:10A4D00069877A878B879C87C8010E94E7D18CE0C7
:10A4E000EBE8F2E0D80101900D928A95E1F7C801FE
:10A4F0000E94E7D11982C8010E94F9D18FE790E04C
:10A500009A838983C8010E94DED1E7E9F2E0D8018D
:10A5100001900D92DA94E1F72AEF35E045E050E042
:10A52000B8018AED95E00E9466508091E405898328
:10A53000C8010E9402D280E2ECE9F2E0D801019069
:10A540000D928A95E1F72AEF35E040E250E0B8013C
:10A550008AED95E00E946650F7011082C7010E94C3
:10A5600002D280E198E00E9402D28CE098E00E9442
:10A57000F0D1CF55DF4F188219821A821B82C15A3F
:10A58000D040CE018F559F4F0E94F0D180E2D8017C
:10A590001D928A95E9F72AEF35E040E250E0B801D4
:10A5A0008AED95E00E946650FE01F99688E0DF0191
:10A5B0001D928A95E9F744E650E060E070E0498337
:10A5C0005A836B837C834D835E836F83788783E0BC
:10A5D00090E0A0E0B0E089879A87AB87BC874D8781
:10A5E0005E876F87788B498B5A8B6B8B7C8B8D8BBF
:10A5F0009E8BAF8BB88F898F9A8FAB8FBC8F8D8FCF
:10A600009E8FAF8FB8A38EE190E0A0E0B0E089A369
:10A610009AA3ABA3BCA38DA39EA3AFA3B8A789A7FE
:10A620009AA7ABA7BCA78DA79EA7AFA7B8AB89ABCE
:10A630009AABABABBCAB8DAB9EABAFABB8AF2AEFBD
:10A6400035E040E450E0B8018AED95E00E946650A4
:10A6500090E1D92EF8018D2D11928A95E9F72AEF14
:10A6600035E040E150E0B8018AED95E00E94665087
:10A67000D8011D92DA94E9F72AEF35E040E150E085
:10A68000B8018AED95E00E946650CF55DF4F1882E1
:10A6900019821A821B82C15AD040CE018F559F4F1A
:10A6A0000E94F0D12CE0D22EF8018D2D11928A95C6
:10A6B000E9F72AEF35E04CE050E0B8018AED95E08B
:10A6C0000E9466508CE6D8011D928A95E9F72AEF20
:10A6D00035E04CE650E0B8018AED95E00E94665006
:10A6E0008EEC95E00E94E7D12AEF35E048E050E09B
:10A6F0006CED75E08AED95E00E946650F7011192CD
:10A70000DA94E9F7C755DF4F1882C95AD04080E084
:10A7100090E0A0E4B0E4C356DF4F88839983AA8316
:10A72000BB83CD59D040C7010E940BD2CE018755C3
:10A730009F4F0E94F9D1CE0183569F4F0E94F0D1C6
:10A7400080E3D7011D928A95E9F78FE89CE10E948A
:10A7500080388AE00E9447382AEF35E040E350E035
:10A76000B7018AED95E00E9466508091FC05811149
:10A7700028C00091DA051091DB058091FA059091CF
:10A78000FB05F7019183808384E690E09093DB05DD
:10A790008093DA052AEF35E044E050E064E073E0AE
:10A7A0008AED95E00E946650C7010E94DED191E0DB
:10A7B0000536134009F490E08091FC05892B8093C5
:10A7C000FC058091FC05811105C060E083EC9CE1F3
:10A7D0000E94EE3F83EA9CE10E9480388AE00E945A
:10A7E00047389091FC0581E08927C655DF4F0FB6A9
:10A7F000F894DEBF0FBECDBFDF91CF911F910F91B7
:10A80000FF90EF90DF900895CF93DF9300D01F92D9
:10A81000CDB7DEB78091AA068823C1F083E390E02C
:10A820009C838B831A8219829E012F5F3F4F40E1E8
:10A8300050E06BEA76E0CE0103960E94665083EA10
:10A840009CE10E9480388AE00E9447380F900F9068
:10A850000F900F90DF91CF910895CF92DF92EF92FA
:10A86000FF92CF93C82F80912C118150823008F035
:10A8700069C00E94E33A10922C110E9451FD60932E
:10A88000C6057093C7058093C8059093C905C0900D
:10A89000CA05D090CB05E090CC05F090CD050E9484
:10A8A000C62BAB01BC014093CA055093CB05609306
:10A8B000CC057093CD058091AF069091B006A09124
:10A8C000B106B091B2068C199D09AE09BF09840F7B
:10A8D000951FA61FB71F8093AF069093B006A09355
:10A8E000B106B093B206C1110AC0C1E00E9404547F
:10A8F0008C2FCF91FF90EF90DF90CF9008958091B3
:10A90000AD069091AE0601969093AE068093AD068B
:10A910000E94C62BC090B306D090B406E090B50656
:10A92000F090B606C616D706E806F906F0F60E94BD
:10A93000C62B6093B3067093B4068093B5069093CC
:10A94000B606D3CFC0E0D2CF81E00C942D540E9444
:10A9500000BF0E94A45480E00E9420F9809100076B
:10A960008130A1F40E944F4E82E697E00E94803829
:10A9700060E088E597E00E94EE3F6EE571E080E0E0
:10A9800090E00E94392688E0809300070895CF92D6
:10A99000DF92EF92FF921F93CF93DF9300D01F922D
:10A9A000CDB7DEB78EEEC82E82E0D82EE12CF12C8A
:10A9B000C982DA82EB82FC82BE016F5F7F4F8AE53B
:10A9C0000E94B23381110EC010E0812F0F900F90C2
:10A9D0000F900F90DF91CF911F91FF90EF90DF903C
:10A9E000CF9008950E940834C982DA82EB82FC82FB
:10A9F000BE016F5F7F4F8AE50E94B233182F882314
:10AA000019F30E944F4E8CE398E00E9480380E9418
:10AA1000A754DBCFCF92DF92EF92FF921F93CF9399
:10AA2000DF9300D01F92CDB7DEB78EEEC82E82E046
:10AA3000D82EE12CF12CC982DA82EB82FC82BE0195
:10AA40006F5F7F4F8AE00E94B23381110EC010E029
:10AA5000812F0F900F900F900F90DF91CF911F914A
:10AA6000FF90EF90DF90CF9008950E9408340E94ED
:10AA7000D2330E94ED330E94D233C982DA82EB8254
:10AA8000FC82BE016F5F7F4F8AE00E94B233182FB5
:10AA90008823E9F20E944F4E8FEF97E00E948038A2
:10AAA0000E94A754D5CFCF93DF9300D01F921F925F
:10AAB000CDB7DEB781E08093AA0680E1EBEAF6E04D
:10AAC000DF011D928A95E9F70E94045486E18D8387
:10AAD00082E390E09C838B831A8219829E012F5F10
:10AAE0003F4F41E050E0BE016B5F7F4FCE010396C8
:10AAF0000E9466500F900F900F900F900F90DF9173
:10AB0000CF910895CF93DF93CDB7DEB7A8970FB657
:10AB1000F894DEBF0FBECDBF8C01F42E0E9400BFA3
:10AB20000E944F4E88E397E00E948038011511057E
:10AB300011F40FE217E080919D0580FD79C08160DE
:10AB400080939D058BE197E00E9480388AE00E9407
:10AB50004738CC24C3948AE5D82ED092D013C09223
:10AB6000CF138FE090E09093D2138093D11397E0AE
:10AB7000792E7092C31322E8E22EE092C61334E8D5
:10AB8000832E912CA12CB12C8092C7139092C813C4
:10AB9000A092C913B092CA1383E793E10E94D03404
:10ABA000D092D013C092CF1388E590E09093D21347
:10ABB0008093D1137092C313E092C6138092C7138F
:10ABC0009092C813A092C913B092CA1383E793E17D
:10ABD0000E94D0348AE289838A838B838C83F80134
:10ABE000DE011596BE016F5F7F4FCD01861B970B6F
:10ABF0002491319621110CC0FB01E80FF91F8AE264
:10AC00009F01261B370B2832310524F48193F8CF9E
:10AC10002D93EBCF20E630E140E050E083E793E175
:10AC20000E9410E16AE070E080E090E00E94D92C80
:10AC300061E086E297E00E94BB3F89EE93E030E658
:10AC4000019729F0232F2A950000E9F7F9CFF8940E
:10AC500089EE93E038EE019729F0232F2A95000022
:10AC6000E9F7F9CF0E9400BFFF2031F00E94311FA9
:10AC70000E944A1FA895FECF0E942F1FF9CF8091F6
:10AC8000FF06882319F01092FF06089540E070E057
:10AC900060E086EB98E10E9482558091AC0C909127
:10ACA000AD0C2FEF3FEF981751F0E92FF0E0E4558E
:10ACB000F34F228130E09F5F9F779093AD0CC901E5
:10ACC00008951F920F920FB60F9211240F900FBE8E
:10ACD0000F901F9018951F920F920FB60F9211248C
:10ACE0000BB60F920F931F932F933F934F935F9346
:10ACF0006F937F938F939F93AF93BF93CF93DF9384
:10AD0000EF93FF93C091C6000091AD0CD091AC0CB5
:10AD100011E01D0F1F7790912B04913108F09FC017
:10AD2000E92FF0E08827E856F94A8F4F0D94B82CA8
:10AD3000A956D856E756F656FD562F5701572F57A6
:10AD4000055709572F570D57115715571C572F5790
:10AD50002757C03229F028F5CA3011F0CD3031F52F
:10AD6000011731F0ED2FF0E0E455F34FC283D12FFE
:10AD7000D093AC0CFF91EF91DF91CF91BF91AF9148
:10AD80009F918F917F916F915F914F913F912F9103
:10AD90001F910F910F900BBE0F900FBE0F901F9041
:10ADA0001895CD3481F081E0CE3471F080E10CC093
:10ADB000CA3338F4C033A0F6C03291F2CD32B1F7C5
:10ADC000CFCFCD3499F782E080932B04C9CFC13324
:10ADD00059F018F4C03221F2E9CF88E0C433A1F36E
:10ADE0008BE0C83389F3E2CF83E0EECF84E0C03359
:10ADF00059F386E0C13341F3D9CF85E0C833B1F6CA
:10AE0000E3CF87E0C23391F6DFCF89E0C13371F63B
:10AE1000DBCF8AE0C03351F6D7CF8CE0C73331F6B1
:10AE2000D3CF8DE0C63311F6CFCFC03209F498CF1F
:10AE30008EE0C33549F2BACF80ED8C0F8A3008F02E
:10AE40008FCF9FE090932B0480932C0489CFCA303E
:10AE500019F0CD3009F084CF10922B0481CFCA3085
:10AE600019F0CD3009F07CCF80912D148823A1F307
:10AE7000973089F038F4953079F710923C021092AF
:10AE80003E0CEACF9A3059F09F3031F780912C0474
:10AE90000E94EF31E1CF81E080932806DDCF81E091
:10AEA00080932706D9CF8EBD0DB407FEFDCF089540
:10AEB0008FEF8EBD0DB407FEFDCF8EB50895909136
:10AEC00064009B7F90936400982F906A96959CBD38
:10AED00080FD03C091E0863009F490E09DBD0895A7
:10AEE000CF93DF93EB010E948038CE01DF91CF91A9
:10AEF0000C944AAF2F923F924F925F926F927F9243
:10AF00008F929F92AF92BF92CF92DF92EF92FF9279
:10AF10000F931F93CF93DF93009709F0AAC110926C
:10AF2000910C1092900C90939C0580939B05BAE035
:10AF3000CB2EB0E2DB2EE12CF12C15E002E846012D
:10AF40005701C4E1D0E0109216131092151310931C
:10AF5000091300930C1380920D1390920E13A0927C
:10AF60000F13B092101389EB92E10E94D034219715
:10AF70002FEF821A920AA20AB20A209721F744E11F
:10AF8000C40ED11CE11CF11C8AE5C81680E2D8066B
:10AF9000E104F104A1F6C12CA0E2DA2EE12CF12C9F
:10AFA000D5E0C2E81092161310921513D09309132E
:10AFB000C0930C13C0920D13D0920E13E0920F1396
:10AFC000F092101389EB92E10E94D0341092161384
:10AFD00010921513D0930913C0930C13D701C60117
:10AFE0008C529F4FAF4FBF4F80930D1390930E1312
:10AFF000A0930F13B093101389EB92E10E94D03409
:10B00000EFEFCE1ADE0AEE0AFE0AFAE0CF16F0E201
:10B01000DF06E104F10431F6FEEDCF2EF0E2DF2E83
:10B02000E12CF12CD5E0C2E8109216131092151302
:10B03000D0930913C0930C13C0920D13D0920E132A
:10B04000E0920F13F092101389EB92E10E94D0343A
:10B050002FEFC21AD20AE20AF20A46EEC41640E202
:10B06000D406E104F10401F7CC24C394E2E1DE2E1E
:10B07000E12CF12C0AE010E0D5E0C2E810931613A1
:10B0800000931513D0930913C0930C13C0920D13A2
:10B09000D0920E13E0920F13F092101389EB92E10D
:10B0A0000E94D0341093161300931513D0930913F4
:10B0B000C0930C13D701C6018096A11DB11D8093CA
:10B0C0000D1390930E13A0930F13B093101389EBED
:10B0D00092E10E94D0348FEFC81AD80AE80AF80A21
:10B0E000E5E0CE16E2E1DE06E104F10439F6009176
:10B0F000900C1091910C0115110509F0D6C08091AA
:10B100008F0C882309F4E1C02AE030E240E050E0EF
:10B110006CEE73E089EB92E10E9410E1C1E0D0E0B7
:10B1200003E010E0E090900CF090910C35E0332EAD
:10B1300042E8242E44244A94542C64E0662E712C58
:10B140007FE1C72E74E0D72E8091900C9091910CE6
:10B15000800F911FE816F90608F0D5C0C7010E94BC
:10B160002BE2882309F481C08091A7116AE971E17B
:10B17000882311F067EA71E1FB0101900020E9F7F3
:10B18000CF010197861B970BF4E1FC9F9001FD9F77
:10B19000300D1124265F3F4D50E040E0459710F000
:10B1A000FB01128A89EB92E10E9410E1CE018F5FD0
:10B1B0009D4EB0E0A0E021964E0124E0880C991C41
:10B1C0002A95E1F7FDEF8F1AFFE99F0AB12CA12C18
:10B1D0002091391424FF7EC07092161360921513CB
:10B1E0003092091320920C1380930D1390930E1339
:10B1F000A0930F13B093101389EB92E10E94D03407
:10B20000D0921613C09215133092091320920C138A
:10B2100080920D1390920E13A0920F13B092101300
:10B2200089EB92E10E94D034B7018BE498E10E944F
:10B230004A418091A71167EA71E1811102C06AE970
:10B2400071E188E498E10E9470576EEF7BE084E43E
:10B2500098E10E9470576AE971E183E498E10E94E5
:10B2600070578FE398E10E9480382FEFE21AF20ABC
:10B270006BCF2091900C3091910CA9014150510954
:10B2800060919B0570919C056817790738F42C5FD5
:10B290003F4F3093910C2093900C45CE4430510594
:10B2A00008F43DCE24503109F4CF0430110569F47F
:10B2B00080918F0C882331F083E090E09093910C83
:10B2C0008093900CD0E0C0E02DCFD0E0C0E004E04F
:10B2D00010E028CF10921613109215133092091314
:10B2E00020920C1380930D1390930E13A0930F13C1
:10B2F000B093101389EB92E10E94D0345092161350
:10B300004092151381CFDF91CF911F910F91FF9044
:10B31000EF90DF90CF90BF90AF909F908F907F90F5
:10B320006F905F904F903F902F900895AF92BF9293
:10B33000CF92DF92EF92FF920F931F93CF93DF9301
:10B34000CDB7DEB7E6970FB6F894DEBF0FBECDBF20
:10B3500000914F0510915005F80101900020E9F788
:10B3600031976F01C01AD10AF801CF01801B910BF0
:10B370008C159D053CF481918F32B9F7DF0111974F
:10B380001C92F3CF8BE1E9E5F4E1DE015C960190DC
:10B390000D928A95E1F7F12CE12CEC14FD040CF0F0
:10B3A0005DC0F801EE0DFF1D8081811103C08FEF9C
:10B3B000E81AF80A5801AE0CBF1CF50180818823F9
:10B3C00009F44CC0FFEFEF1AFF0AF801EE0DFF1D64
:10B3D0007F01E01AF10A81918111FACFCE014C96DA
:10B3E0000E94DDB38BE1FE017C96DE011196019097
:10B3F0000D928A95E1F7B501CE0101960E94EBAB63
:10B40000CE0101960E94DC2F8FE20E944738809186
:10B41000A71181113BC089EF93E00E944AAF809150
:10B42000391484FF1BC019821C8221E0A501BE01D2
:10B43000645E7F4FCE0101960E941FB6811129C024
:10B440008AE00E9447380E94534EB5018AE297E194
:10B450000E947057CE0101960E94DC2F8AE00E9464
:10B460004738CE014C960E94DC2FE6960FB6F89432
:10B47000DEBF0FBECDBFDF91CF911F910F91FF9027
:10B48000EF90DF90CF90BF90AF90089587EA91E161
:10B49000C4CFCE014C960E944CB38BE1FE01319695
:10B4A000DE015C9601900D928A95E1F7CE0101963E
:10B4B0000E94DC2F72CF2F923F924F925F926F9239
:10B4C0007F928F929F92AF92BF92CF92DF92EF9234
:10B4D000FF920F931F93CF93DF9300D000D000D043
:10B4E0001F921F92CDB7DEB7B82E8091990D843090
:10B4F00008F0D1C10E9451FD6B017C018091990D32
:10B50000811108C08091AC0C9091AD0C891B8F7794
:10B5100009F4A4C681E6A82E13C08A3019F08D3034
:10B5200009F0F6C01092940D8091320D9091330D78
:10B53000FC01E25DF24F1682892BF1F40E944DC2AC
:10B540008091990D843008F0ECC08091AC0C909102
:10B55000AD0C891B8F7709F4E4C00E944D5697FF0C
:10B56000DCCF0E944F4E85EB95E00E9480388091A1
:10B57000AC0C8093AD0CE4CF1092330D1092320DD1
:10B5800004E31DE0F8018191803209F446C08E3455
:10B5900009F0A9C060EB75E0C8010F946E254C015D
:10B5A000892B41F06EE470E0C80104960F940F30CF
:10B5B000009709F4C8014AE050E070E060E00196AD
:10B5C0000F94DE222B013C0180912E0D90912F0DC6
:10B5D000A091300DB091310D0196A11DB11D4816FD
:10B5E00059066A067B0629F060E08DE795E0892818
:10B5F00051F16AE270E0C8010F943E309C0100975F
:10B6000029F1982F901B912C992349F09150F80122
:10B61000E90FF11D80819826F7CF8F01B3CF4AE063
:10B6200050E070E060E0C90101960F94DE22292D00
:10B6300030E050E040E0621773078407950751F04F
:10B6400060E08EE595E00E94A6E77ACF60E084E3B3
:10B6500095E0F9CF40922E0D50922F0D6092300D53
:10B660007092310D809100078130E1F067E470E065
:10B67000C8010F940F300097A9F04AE050E070E045
:10B6800060E001960F94DE2264307105810591051A
:10B6900048F483E994E00E94803860E089E894E00F
:10B6A0000E94EE3FC0929F07D092A007E092A107B0
:10B6B000F092A2078091340D8B3309F441CF809131
:10B6C000990D843008F03CCF80919B0D8A9DC0017C
:10B6D000112464E37DE08456924F0F941A3080E089
:10B6E0000E9460E72DCF8091391480FFBBCF61E9C4
:10B6F0007DE2C8010F946E25009731F0FC01838133
:10B7000080538A3008F0AECF60E08AE095E09BCFAE
:10B7100022E33DE044E35DE064E97DE00E94451DF5
:10B720000FCF8091391482FFB6C01A82198271E658
:10B73000F72EE0E1EE2EF9E6DF2E8091990D8430B0
:10B7400008F0A9C00E947D1D8111A5C041E050E014
:10B75000BE016B5F7F4F8DE995E10E949FB10D8126
:10B7600010E0019711F00FEF1FEF8091A515909158
:10B77000A615A091A715B091A815809335149093A4
:10B780003614A0933714B09338140E947D1D0F3FD8
:10B79000100749F4811107C00E944F4E83ED95E0D8
:10B7A0000E948038CACF40919B0D242F30E00A3090
:10B7B00061F00D3051F0882309F45FC089819A81CE
:10B7C000009719F001969A8389831092B2048981B7
:10B7D0009A81F29EF001F39EF00D1124E756F24F8C
:10B7E000E80FF91F1382892B69F50E944DC20E9450
:10B7F0007D1D882309F4A1CF0E94C5618DE995E1E3
:10B800000E944CB380913014882391F18150809331
:10B8100030148D9DC001112462E0885C994F0E9414
:10B82000A1B8E091301424E0E29FF0011124EC5C17
:10B83000F94F60817181828193810E9496220E94DA
:10B8400054AB7BCF1A82198281E00E9460E780911D
:10B85000351490913614A0913714B0913814809318
:10B86000950D9093960DA093970DB093980DBFCF23
:10B870000E9455B3E092000760CF4F9DA0011124B4
:10B880004456524F9E012F5F3F4F62EB74E0802F72
:10B890000E94451D52CF0E9451FD6B017C01B110E9
:10B8A00004C080912B11882351F0C0927E11D09258
:10B8B0007F11E0928011F0928111BB24B3948091AA
:10B8C000270590912805A0912905B0912A05009798
:10B8D000A105B105B1F040917E1150917F116091A9
:10B8E000801170918111840F951FA61FB71FA701AA
:10B8F0009601281B390B4A0B5B0BDA01C901B7FF14
:10B9000092C18091130290911402A0911502B091FE
:10B910001602892B8A2B8B2B09F099C10E9451FDAD
:10B920004B015C0180913E0C811108C02091911265
:10B930009091921281E0291301C080E02091F311CF
:10B940003091F41191E089272A3A31050CF480E016
:10B9500091E04091B7045091B8046091B90470919E
:10B96000BA04452B462B472B09F490E0981789F031
:10B97000882309F4BDC1D501C40180569444A24F67
:10B98000BF4F8093B7049093B804A093B904B093C9
:10B99000BA0440906D0250906E0260906F027090F9
:10B9A00070022091B3043091B4044091B5045091D9
:10B9B000B604C301B2010F94F125882319F18091D7
:10B9C000B7049091B804A091B904B091BA04409220
:10B9D000B3045092B4046092B5047092B604892BFB
:10B9E0008A2B8B2B09F449C0D501C401805694449D
:10B9F000A24FBF4F8093B7049093B804A093B904AB
:10BA0000B093BA048091B7049091B804A091B9049E
:10BA1000B091BA040097A105B10579F1881A990A85
:10BA2000AA0ABB0AB7FC29C01092B7041092B80446
:10BA30001092B9041092BA0483E396E00E94803811
:10BA400060E08FE196E00E94EE3F8091F5119091C9
:10BA5000F6111816190624F490E080E00E944D1F9C
:10BA600080918A1190918B111816190634F4109256
:10BA70008B1110928A110E94D3BE8091BF049091C5
:10BA8000C004A091C104B091C20446015701881AB4
:10BA9000990AAA0ABB0AD501C401B7FDB9C1209110
:10BAA00091129091921240912D0280912C022913B3
:10BAB00023C190911809899FC0011124880F892FF3
:10BAC000881F990B91958D8380911909489FC0011A
:10BAD0001124880F892F881F990B91958E830E94BE
:10BAE00051FD69837A838B839C8340E0BE016F5F45
:10BAF0007F4FCE0105960E94971C6D8170E089E012
:10BB00000E9448FC41E0BE016F5F7F4FCE01059669
:10BB10000E94971C6E8170E087E00E9448FC809133
:10BB20003306882309F467C1009120021091210295
:10BB3000C80102972091F5113091F61128173907A5
:10BB40000CF459C1809092128F82188619861A8639
:10BB50001B86809191129F80891509F4E7C0892D79
:10BB600090E03CE5A32EA89EF001A99EF00D1124C3
:10BB7000E35EF64F458956896789708D452B462BC4
:10BB8000472B81F4418D528D638D748D452B462B4F
:10BB9000472B41F4458D568D678D70A1452B462B63
:10BBA000472BE1F12CE5B22EB89E9001B99E300DE5
:10BBB0001124A901435E564F1A01FA016181728175
:10BBC000838194810F946F2F4B015C01F10161A17E
:10BBD00072A183A194A10F94F6252B013C01F101E0
:10BBE00065A176A187A190A50F94F6259B01AC01D4
:10BBF000C301B2010F94BB2DA50194010F945726E8
:10BC00004B015C01288539854A855B850F94212F7E
:10BC1000181624F488869986AA86BB868F818F5F42
:10BC200087708F8396CF0E944F4E60919D077091D1
:10BC30009E0782EE95E00E9470578AE00E94473886
:10BC400040E070E060E090E080E00E9482559091DA
:10BC5000911280919212981749F0C0927E11D09261
:10BC60007F11E0928011F092811158CEBB2019F023
:10BC70001092C30453CE0E9451FD00917E11109189
:10BC80007F1120918011309181118090130290904A
:10BC90001402A0901502B0901602080D191D2A1D5D
:10BCA0003B1D601B710B820B930B97FDE1CF8091C5
:10BCB000C304811133CE81E08093C3045F9A8091E5
:10BCC0003F0C8E7F80933F0C8A9A80913F0C8D7F32
:10BCD00080933F0C809108018095817080930601CC
:10BCE00080913F0C8B7F80933F0C0E942F1F16CEBC
:10BCF00080E090E0DC0145CE209192125CE5259F2A
:10BD000090011124235E364FF901EA5AFF4F9081CA
:10BD1000899FC0011124880F892F881F990B919545
:10BD20008D83295A3F4FF9018081D0CE20911A028C
:10BD300030911B0240911C0250911D02688579854B
:10BD40008A859B850F9457264B015C01B801012E13
:10BD5000000C880B990B0F94F8259B01AC01C501D1
:10BD6000B4010F94C12C69837A838B839C834091A7
:10BD70001E0250911F02B801CE0101960E940BC213
:10BD800089809A80AB80BC804090BB045090BC04FA
:10BD90006090BD047090BE04A3019201C501B4017E
:10BDA0000F94F12587FF16C028E431EE4AE75FE3E0
:10BDB000C301B2010F94572620E037ED43EA5CE35C
:10BDC0000F94C12CA50194010F94572669837A839F
:10BDD0008B839C8369817A818B819C816093BB0476
:10BDE0007093BC048093BD049093BE040F942D2ED9
:10BDF000CB010E944D1FF4E6CF0ED11CE11CF11CBB
:10BE0000C092BF04D092C004E092C104F092C20478
:10BE10000E944DC280910007882309F4E0C18091FF
:10BE20002602882309F4A3C08091010581119FC0D7
:10BE300080912B11811108C080912C11813021F04B
:10BE40008091391482FF93C0F894649B10C0809154
:10BE5000220290912302A0912402B09125028093A6
:10BE6000010690930206A0930306B0930406609126
:10BE70000106709102068091030690910406789461
:10BE800020E030E0A9010F94F12587FF70C001E0A8
:10BE90000093010580912B11811167C088E496E021
:10BEA0000E9480388AE00E94473884E08093A60C84
:10BEB00082E08093920C81E09AE59093D013809376
:10BEC000CF138EE490E09093D2138093D11387E048
:10BED0008093C31382E88093C61384E890E0A0E0C7
:10BEE000B0E08093C7139093C813A093C913B09385
:10BEF000CA1383E793E10E94D0340E946B40009301
:10BF0000991140E36CE876E084E799E00E94704084
:10BF100061E088E699E00E94524010912B0560E0B4
:10BF200010278CE399E069F48AE796E00E94BB3F12
:10BF300080E30E9447388AE00E94473860E08DE540
:10BF400096E00E94BB3F88E696E00E94803880E33E
:10BF50000E9447388AE00E944738112331F083E677
:10BF600096E090938E0C80938D0C0E94C561909109
:10BF70000901892F80958170109100021817C9F06E
:10BF8000209139142062209339148093000290FD8F
:10BF90003FC164EF71E080E090E00E9439260E948A
:10BFA00077B38091391483FD7CC1111133C10E9494
:10BFB00015360E9451FD6B017C011091170211236F
:10BFC000F1F080912C058823D1F04091C404509168
:10BFD000C5046091C6047091C70446015701841AD4
:10BFE000950AA60AB70AB501A40177FD1AC08330E5
:10BFF00009F42FC10CF01EC181300CF023C1212F98
:10C0000030E0A8EEB3E00F94892CC60ED71EE81ED0
:10C01000F91EC092C404D092C504E092C604F09206
:10C02000C70480912C11813009F073C00E9451FD2A
:10C030006B017C018091CC049091CD04A091CE0441
:10C04000B091CF04A7019601281B390B4A0B5B0B5B
:10C05000DA01C901B7FD3AC0D701C601805F984D2A
:10C06000AF4FBF4F8093CC049093CD04A093CE04E8
:10C07000B093CF048090CA059090CB05A090CC05DA
:10C08000B090CD050E94C62BAB01BC014093CA0500
:10C090005093CB056093CC057093CD058091AF068E
:10C0A0009091B006A091B106B091B2068819990995
:10C0B000AA09BB09840F951FA61FB71F8093AF065F
:10C0C0009093B006A093B106B093B2068091C804D5
:10C0D0009091C904A091CA04B091CB0446015701C4
:10C0E000881A990AAA0ABB0AD501C401B7FD11C072
:10C0F00020E8C20E2EEED21E26E3E21EF11CC092F4
:10C10000C804D092C904E092CA04F092CB040E9401
:10C1100004540E94BE390E948841809126058823DC
:10C1200079F10E9451FD6B017C0180912205909173
:10C130002305A0912405B091250546015701881AD1
:10C14000990AAA0ABB0AD501C401B7FD19C02091FA
:10C15000260530E0A8EEB3E00F94892CC60ED71E5A
:10C16000E81EF91EC0922205D0922305E092240514
:10C17000F092250580E00E9431BB8AE00E9447389A
:10C1800080912105882359F10E9451FD6B017C01AA
:10C1900080911D0590911E05A0911F05B09120056D
:10C1A000A7019601281B390B4A0B5B0BDA01C90169
:10C1B000B7FD15C02091210530E0A8EEB3E00F9443
:10C1C000892CC60ED71EE81EF91EC0921D05D092FE
:10C1D0001E05E0921F05F09220050E9412AB2B96DF
:10C1E0000FB6F894DEBF0FBECDBFDF91CF911F9188
:10C1F0000F91FF90EF90DF90CF90BF90AF909F9006
:10C200008F907F906F905F904F903F902F90089508
:10C210000E9466B3123008F0CCCE0E94153660E062
:10C2200085EC96E056C083ED96E090938E0C80935B
:10C230008D0CBFCE843009F0E2CE0E94534E8AEDC1
:10C2400096E004C00E94534E89E097E00E94803837
:10C25000D6CE0E94534E82EF96E0F8CF80919F0792
:10C260009091A007A091A107B091A207A701960104
:10C27000281B390B4A0B5B0BDA01C901885E93401E
:10C28000A109B109B7FD46C98DEC95E00E9480383F
:10C29000C0929F07D092A007E092A107F092A20758
:10C2A00039C91230C8F48DE996E00E9480388AE0DE
:10C2B0000E9447380E94F42C90E080E00E947A5758
:10C2C0001092AA0C1092A90C1092A80C60E086EBB8
:10C2D00096E00E94EE3F6DCE123009F06ACE0E94C9
:10C2E000D1B7882379F081E00E94A7B742EB50E0F4
:10C2F00069E278E08EE394E10E949FB18EE394E1DD
:10C300000E944CB30E94CA2F81118DCF0E94B42F7E
:10C310000E944DB80E94A2B74CCECF93DF9380917C
:10C32000911290919212891B8095877019F40E9446
:10C330005B5AF5CF809191128F5F8770A091911217
:10C340009CE5A99FD0011124FD01E35EF64FEF01AA
:10C3500019929A95E9F798E09083AE5CB64F90E118
:10C36000E3E9F2E101900D929A95E1F720919112A3
:10C3700090919212291303C094E690938E128093A9
:10C380009112DF91CF910C94E22F909191128091B4
:10C390009212981306C080911B0990911C09892B59
:10C3A00021F080E00E945B5AF0CF0895FC012081CB
:10C3B0003181428153816091610C7091620C809156
:10C3C000630C9091640C0F9457260F942E2F60935A
:10C3D0009F127093A0128093A1129093A212909139
:10C3E00091128091921298130C948D610E94C561F4
:10C3F0000E94392A40919F125091A0126091A1127F
:10C400007091A21240932306509324066093250650
:10C410007093260681110C94E22F08954F925F923B
:10C420006F927F928F929F92AF92BF92CF92DF9244
:10C43000EF92FF920F931F93CF93DF93EC018B0149
:10C440005A01F9012091610C3091620C4091630C0A
:10C450005091640C60817181828193810F94572681
:10C460000F942E2F6B017C0120915D0C30915E0C9E
:10C4700040915F0C5091600CF50160817181828167
:10C4800093810F9457260F942E2F4B015C0120911E
:10C49000590C30915A0C40915B0C50915C0CF80196
:10C4A00060817181828193810F9457260F942E2F82
:10C4B0002B013C012091550C3091560C4091570CAA
:10C4C0005091580C688179818A819B810F945726FD
:10C4D0000F942E2F60939312709394128093951261
:10C4E00090939612409297125092981260929912DD
:10C4F00070929A1280929B1290929C12A0929D121E
:10C50000B0929E12C0929F12D092A012E092A112FD
:10C51000F092A2129091911280919212981791F03C
:10C52000DF91CF911F910F91FF90EF90DF90CF900F
:10C53000BF90AF909F908F907F906F905F904F9043
:10C540000C948D610E94C5610E94392A40919B1212
:10C5500050919C1260919D1270919E1200919712C1
:10C56000109198122091991230919A12C0909312C2
:10C57000D0909412E0909512F0909612C092170607
:10C58000D0921806E0921906F0921A0600931B0644
:10C5900010931C0620931D0630931E0640931F0621
:10C5A00050932006609321067093220640919F12BB
:10C5B0005091A0126091A1127091A2124093230693
:10C5C000509324066093250670932606882391F0E5
:10C5D000DF91CF911F910F91FF90EF90DF90CF905F
:10C5E000BF90AF909F908F907F906F905F904F9093
:10C5F0000C94E22FDF91CF911F910F91FF90EF905C
:10C60000DF90CF90BF90AF909F908F907F906F9072
:10C610005F904F9008953F924F925F926F927F92FA
:10C620008F929F92AF92BF92CF92DF92EF92FF9242
:10C630000F931F93CF93DF93CDB7DEB768970FB6F5
:10C64000F894DEBF0FBECDBFD82E2A013B014801B2
:10C6500059013E2C20E030E0A901C501B8010F943A
:10C66000F125811110C081E08D1508F0B6C060E0A1
:10C6700070E080E793E420E030E040E752E40F947C
:10C68000BB2D4B015C018D8A9E8AAF8AB88E0D2D21
:10C6900010E0F801E056F64EE491BB24B3941E1668
:10C6A0000CF4B12CCC24C39420E030E0A901C301E8
:10C6B000B2010F94212F18160CF0C12CBC1471F08C
:10C6C00092E0D9120BC0332049F081E00E9420F99A
:10C6D00069E170E080E090E00E94392680E00E94ED
:10C6E000E82F69837A838B839C8381E00E94E82F03
:10C6F0006D837E838F83988782E00E94E82F69870D
:10C700007A878B879C8783E00E94E82F6D877E87DE
:10C710008F87988B000F111F000F111FE1E0F0E0D1
:10C72000EC0FFD1F0E0F1F1FF801108211821282E5
:10C7300013829E01235F3F4FAE01475F5F4FBE01F3
:10C740006B5F7F4FCE0101960E940E62F80140821E
:10C75000518262827382198A1A8A1B8A1C8A80918A
:10C760001B0990911C09892B91F4CE0141967C0103
:10C770008E010B5E1F4F9E01235F3F4FAE01475F4F
:10C780005F4FBE016B5F7F4F40970E94CAE70E94D8
:10C79000C561BC1451F092E0D91205C0332019F0E4
:10C7A00080E00E9420F90E943F5668960FB6F894E8
:10C7B000DEBF0FBECDBFDF91CF911F910F91FF90D4
:10C7C000EF90DF90CF90BF90AF909F908F907F9031
:10C7D0006F905F904F903F90089560E070E88BE31A
:10C7E00095E449CF4F925F926F927F928F929F9282
:10C7F000AF92BF92CF92DF92EF92FF920F931F936F
:10C80000CF93DF93CDB7DEB72C970FB6F894DEBF8A
:10C810000FBECDBF2B013C0129873A874B875C8730
:10C8200047015801F601E080F1800281138120E088
:10C8300030E0A901B701C8010F94F125882309F45C
:10C8400088C05E2D4F2D302F212F852F942FA32FA1
:10C85000B22F89839A83AB83BC8320E030E0A901A7
:10C86000B701C8010F94F125811108C0E0903D0285
:10C87000F0903E0200913F0210914002C701D801A2
:10C880008D839E83AF83B887A5019401609169026F
:10C8900070916A0280916B0290916C020F94F12565
:10C8A00087FF0CC08092690290926A02A0926B028C
:10C8B000B0926C02CE0101960E94142B409261024C
:10C8C00050926202609263027092640289859A8536
:10C8D000AB85BC858093650290936602A093670246
:10C8E000B0936802CE0105960E94142BA501940115
:10C8F0006091690270916A0280916B0290916C0262
:10C900000F94212F181664F48092690290926A02A3
:10C91000A0926B02B0926C02CE0101960E94142B81
:10C920000E94C5612C960FB6F894DEBF0FBECDBF36
:10C93000DF91CF911F910F91FF90EF90DF90CF90FB
:10C94000BF90AF909F908F907F906F905F904F902F
:10C95000089550E040E030E820E477CFCF92DF92B6
:10C96000EF92FF920F931F936A01E0906902F0909B
:10C970006A0200916B0210916C02FB0120813181EF
:10C9800042815381FC0160817181828193810E9487
:10C99000F2631F910F91FF90EF90DF90CF90089579
:10C9A000CF92DF92EF92FF920F931F936B01FC01E6
:10C9B000E080F18002811381E1E6F2E0248135819B
:10C9C0004681578160817181828193810E94F263E7
:10C9D0001F910F91FF90EF90DF90CF9008950F93EC
:10C9E0001F93CF93DF93EC018B0181E00E9420F92C
:10C9F00069E170E080E090E00E943926B801CE0144
:10CA00000E94D064C091FF0680E00E9420F910923D
:10CA1000FF0682E00E9412300E942F2BC2FBCC271F
:10CA2000C0F981E08C27DF91CF911F910F9108957C
:10CA3000AF92BF92CF92DF92EF92FF920F931F932C
:10CA4000CF93DF9300D01F92CDB7DEB7FC01E0801B
:10CA5000F18002811381611112C0A0906902B0902F
:10CA60006A02C0906B02D0906C029501A601B701DA
:10CA7000C8010F94F12587FF02C07501860120E0EF
:10CA800030E048EC53E4B701C8010F94F12587FD6D
:10CA900004C0E12CF12C08EC13E4C701D801898310
:10CAA0009A83AB83BC8360EF72E0CE0101960E9453
:10CAB000D0640F900F900F900F90DF91CF911F9146
:10CAC0000F91FF90EF90DF90CF90BF90AF900895BF
:10CAD0003F924F925F926F927F928F929F92AF920E
:10CAE000BF92CF92DF92EF92FF920F931F93CF935B
:10CAF000DF9300D01F92CDB7DEB7382E80E090E0F4
:10CB0000A0E2B1E489839A83AB83BC83C09088128E
:10CB1000D0908912E0908A12F0908B1220E030E0E1
:10CB2000A901C701B6010F94F12587FF0CC0A70129
:10CB3000960160E070E080E291E40F94C02C69837C
:10CB40007A838B839C8360E0CE0101960E941865F6
:10CB500040906102509062026090630270906402A3
:10CB60008090650290906602A0906702B090680283
:10CB7000332089F10E940A5519821A821B821C8275
:10CB8000E0906902F0906A0200916B0210916C02D1
:10CB9000CE0101966C01A5019401C301B2010E946E
:10CBA000F26330929B070E94B72B0F900F900F906B
:10CBB0000F90DF91CF911F910F91FF90EF90DF9039
:10CBC000CF90BF90AF909F908F907F906F905F902D
:10CBD0004F903F9008950E94C754CECF80919B07FD
:10CBE000882319F080E00E94686580E008952F9204
:10CBF0003F924F925F926F927F928F929F92AF92ED
:10CC0000BF92CF92DF92EF92FF920F931F93CF9339
:10CC1000DF93CDB7DEB766970FB6F894DEBF0FBED1
:10CC2000CDBFF82E282E312CF101E056F64ED490CF
:10CC300022E0821335C080919B07811103C081E0FF
:10CC40000E9468650E940A55811139C18CE999E1F9
:10CC50000E94B61D20E030E0A9010F94F125882341
:10CC6000F9F06D2DDD0C770B880B990B0F94F825DF
:10CC70002B013C018CE999E10E94B61D4B015C013E
:10CC800020E030E040EA50E40F94F12511E087FF06
:10CC90001CC0812C912C90EAA92E90E4B92E15C0CD
:10CCA0006D2DDD0C770B880B990B0F94F8252B015C
:10CCB0003C01C101880F991F880F991F8C56964E11
:10CCC0000E94B61D4B015C0110E0A3019201C50159
:10CCD000B4010F9457264B015C016101CC0CDD1CA3
:10CCE000CC0CDD1CC6018857964E0E94B61DEE2462
:10CCF000E394E12620E030E040EC5FE30F94572618
:10CD0000A30192010F945726AB01BC0100E010E093
:10CD100098018F2D0E940B6320E030E0A901C5012E
:10CD2000B4010F94F125F601E458F64EFA8BE98B25
:10CD3000882309F44DC0F2E000E010E020E431E483
:10CD4000FF1619F000E010E09801B501A401705839
:10CD5000E12C8F2D0E940B63A5019401C501B40144
:10CD60000F94C12C6B8B7C8B8D8B9E8B22E0F216EB
:10CD7000E9F0F101E758F64E6491611107C00E9495
:10CD8000534E87E599E10E9480386AE070E090E0B8
:10CD900080E00F94F6259B01AC0160E070E088E430
:10CDA00092E40F94BB2D8B019C0104C000E010E0C5
:10CDB00020EC30E4EE24E3944B895C896D897E8914
:10CDC0008F2D0E940B6332E0F312D0C00E94C75433
:10CDD00081E090E0A0E0B0E00F2C04C0880F991F24
:10CDE000AA1FBB1F0A94D2F720913F0C282B209337
:10CDF0003F0C2091B505822B8093B50589899A89CE
:10CE00000E94B61DF601EF59FD4F60837183828346
:10CE1000938382E0F8121AC020918812309189120F
:10CE200040918A1250918B126091690270916A024E
:10CE300080916B0290916C020F94C02C60936902F8
:10CE400070936A0280936B0290936C02F601EF5E1E
:10CE5000F74F10821182128213828F2D0E94D31CF1
:10CE60000E942F2BF601EF59FD4F80819181A28105
:10CE7000B381F601E557F84F80839183A283B38392
:10CE800092E0F916A9F18CE0ECEBF2E0DE011196EC
:10CE900001900D928A95E1F7E1E0F0E0EC0FFD1FC3
:10CEA000EC0DFD1D80809180A280B38020E030E0F9
:10CEB000A901C501B4010F94F12581111EC0669628
:10CEC0000FB6F894DEBF0FBECDBFDF91CF911F919B
:10CED0000F91FF90EF90DF90CF90BF90AF909F9019
:10CEE0008F907F906F905F904F903F902F9008951C
:10CEF0000E94EE658111E3CFC6CF20E030E0A901AA
:10CF0000C501B4010F94212F87FF04C0B7FAB09474
:10CF1000B7F8B094F601EF59FD4F6F01A3019201EC
:10CF2000C501B4010F9457269B01AC01F601608145
:10CF30007181828193810F94C02CF601608371838B
:10CF400082839383F2E080E090E0A0E4B1E4FF16F6
:10CF500021F080E090E0A8E4B2E48D879E87AF875F
:10CF6000B88BCE010D960E94142BA9CF81E090E0E2
:10CF7000A0E0B0E00F2C04C0880F991FAA1FBB1FB0
:10CF80000A94D2F720913F0C282B20933F0C20913C
:10CF9000B505822B8093B50589899A890E94B61DB3
:10CFA000F601EF59FD4F60837183828393834ECFE7
:10CFB000CF93DF9300D01F92CDB7DEB780E090E033
:10CFC000A0EAB0E489839A83AB83BC8361E0CE019D
:10CFD00001960E9418650F900F900F900F90DF91AF
:10CFE000CF9108958F929F92AF92BF92CF92DF928E
:10CFF000EF92FF920F931F93CF93DF93CDB7DEB7DE
:10D000002C970FB6F894DEBF0FBECDBF8B0140E06A
:10D0100050E068E472E44D835E836F83788740E07C
:10D0200050E060EA70E449875A876B877C878130DB
:10D03000B9F1823009F459C020E030E040E050E41A
:10D040006091690270916A0280916B0290916C020A
:10D050000F94C12C4B017C0120E030E048EC53E4FC
:10D060000F94212F181634F4812C912C88ECE82E83
:10D0700093E4F92EF801A084B184C284D38494018E
:10D08000A701B501C6010F94212F181614F0540101
:10D090006701C501D60189839A83AB83BC8348C0ED
:10D0A000BE01675F7F4FC80108960E94D064B80137
:10D0B0006C5F7F4FAE014B5F5F4FC8010E94AE6453
:10D0C0000E94E2302C960FB6F894DEBF0FBECDBFA3
:10D0D000DF91CF911F910F91FF90EF90DF90CF9054
:10D0E000BF90AF909F908F900895F8012085318573
:10D0F000428553856091690270916A0280916B024A
:10D1000090916C020F94C12C6B017C0120E030E007
:10D1100048EC53E40F94F12587FD06C0C12CD12CB7
:10D1200028ECE22E23E4F22EC982DA82EB82FC8222
:10D13000BE01675F7F4FCE010196B7CFEF92FF929E
:10D140000F931F93CF93DF937C018B010E94DC31FF
:10D15000C1E6D2E0209171023091720240917302D7
:10D1600050917402F70160817181828193810F94E3
:10D17000BB2D2C853D854E855F850F94C12C6C871A
:10D180007D878E879F87C8010E94142BDF91CF91E6
:10D190001F910F91FF90EF900C94C5614F925F9299
:10D1A0006F927F92AF92BF92CF92DF92EF92FF92F7
:10D1B0000F931F93CF93DF9300D000D01F921F9245
:10D1C000CDB7DEB75C0180E090E0A0E7B2E48983F0
:10D1D0009A83AB83BC8380E090E0A0E8B0EC8D83C1
:10D1E0009E83AF83B887BE016F5F7F4FCE010596E8
:10D1F0000E949E6868E873E180E090E00E94392612
:10D20000C12CD12C88ECE82E81E4F82EC982DA8278
:10D21000EB82FC8280E090E0A0E8B0E48D839E8306
:10D22000AF83B887BE016F5F7F4FCE0105960E9426
:10D230009E6801E41CE0F80140AC51AC62AC73ACF8
:10D24000C0AED1AEE2AEF3AE80E090E0A0E2B2E4D8
:10D2500089839A83AB83BC83F50180819181A2810C
:10D26000B3818D839E83AF83B887BE016F5F7F4F8D
:10D27000CE0105960E949E68F80140AE51AE62AEA6
:10D2800073AE129A64E670E080E090E00E94392666
:10D2900081E028960FB6F894DEBF0FBECDBFDF91B8
:10D2A000CF911F910F91FF90EF90DF90CF90BF90A3
:10D2B000AF907F906F905F904F9008951F93CF93A2
:10D2C000DF93CDB7DEB72C970FB6F894DEBF0FBE55
:10D2D000CDBF182F882379F020E030E0A9016091BC
:10D2E000ED057091EE058091EF059091F0050F949A
:10D2F000F1258823F9F08091400C8117D9F00E9424
:10D30000C5618CE0E8ECF2E0DE01119601900D922F
:10D310008A95E1F7CE0101960E94621F8091400C30
:10D32000882391F081E692E00E943B271092400C06
:10D330000E942F2B2C960FB6F894DEBF0FBECDBFE8
:10D34000DF91CF911F91089581E08093400C81E699
:10D3500092E00E944F21ECCF2F923F924F925F922A
:10D360006F927F928F929F92AF92BF92CF92DF92F5
:10D37000EF92FF920F931F93CF93DF93CDB7DEB75A
:10D38000CB54D1090FB6F894DEBF0FBECDBF2DB779
:10D390003EB739AF28AF87E00E94634E81110BC0C2
:10D3A00061E086E50E9487248DA3853060F087E3E5
:10D3B0009EE00E948038A8ADB9AD0FB6F894BEBF0C
:10D3C0000FBEADBF40C33DA1332321F087E19EE0F6
:10D3D0000E9480386AE080E50E948724182F8CEF35
:10D3E000810F8F3218F083EF9DE0E3CF60E085E49A
:10D3F0000E94A324882309F448C081E08FABE09009
:10D400008C12F0908D12D7012D913D914D915C9130
:10D410006091610270916202809163029091640256
:10D420000F94C12CAB01BC0188E50E94F5246987EB
:10D430007A878B879C87F7012481358146815781C4
:10D440006091650270916602809167029091680216
:10D450000F94C12CAB01BC0189E50E94F5246D87B6
:10D460007E878F87988BBE01635F7F4FCE010996C1
:10D470000E94822E382E81110BC063E68FED9DE055
:10D480000E94EE3F87EC9DE094CF92E09FABB7CF38
:10D490008CE40E94771E082F882309F431C10E9472
:10D4A00073248EA3803118F080EA9DE082CFFEA124
:10D4B000F13009F427C160E083E50E94A3248AAF1C
:10D4C000882321F0011102C037E03EA38DA18330F3
:10D4D00020F086E89DE00E9480389091400C9DAF3E
:10D4E00080E00E945E690E940C1D1D8A1E8A1F8AB0
:10D4F000188E198E1A8E1B8E1C8E83EF9FE4A3EC60
:10D50000B7E48D8F9E8FAF8FB8A383EF9FE4A3EC1A
:10D51000B7EC89A39AA3ABA3BCA3A12FB0E0BCA78F
:10D52000ABA7EDB7FEB724E0129FE019F109112473
:10D530000FB6F894FEBF0FBEEDBF8DB79EB7019634
:10D540009CAF8BAF2DA14FA9BE01635F7F4FCE0172
:10D5500009960E94AFF99B01AC010F94B32F811182
:10D5600062C20E9451FD611571058105910511F09E
:10D570000F947721212C1BAA1CAA1DAA1EAAAEA1BA
:10D58000A150BB0B2C96BFAFAEAF2C97E22DF0E0B5
:10D59000F8A7EFA32BA53CA5E217F3070CF074C284
:10D5A0003196FEA7EDA73F932F93FF93EF9382E76A
:10D5B0009DE09F938F938CE79DE09F938F931F92A5
:10D5C0000E943EF98DB79EB709960FB6F8949EBF9C
:10D5D0000FBE8DBF9EA1992309F458C10F94282135
:10D5E0002AE030E040E050E00F94572C0F94F825EB
:10D5F00020E030E040EA50E40F94212F0FEF1FEFBE
:10D60000181614F001E010E00F94282128E631E00C
:10D6100040E050E00F94572C0F94F8252B013C016B
:10D620000F94282128E230E040E050E00F94572C7E
:10D630006B5F7F4F8F4F9F4F0F94F8254B015C011D
:10D64000ADA1A430D1F4BC01A40184E69DE00E9408
:10D650005C41B301A2018CE59DE00E945C4186E53E
:10D660009DE00E9480380130110519F483E40E9486
:10D67000473882E59DE00E948038312CC801110FA7
:10D68000AA0BBB0B2A968CAF9DAFAEAFBFAF2A974C
:10D690002C96AEADBFAD2C973A161B060CF0F6C01B
:10D6A0002A966CAD7DAD8EAD9FAD2A970F94F8256F
:10D6B0006B017C01BAADBB2341F1AC019B010F941E
:10D6C000C12C20E030E040E952E40F9457269B0142
:10D6D000AC01C301B2010F94C12C2B013C0120E02D
:10D6E00030E044EB53E40F94212F1816FCF420E0B3
:10D6F00030E044EB53E4C301B2010F94C02CEDCFF2
:10D700001EA2D9CE22E02EA3D6CE0F94282124E14A
:10D7100030E040E050E00F94572C675E7F4F8F4F12
:10D720009F4F0F94F825A7019601CFCF20E030E05E
:10D73000A901C301B2010F94F12587FF0BC020E0BE
:10D7400030E044EB53E4C301B2010F94C12C2B0130
:10D750003C01ECCF00918C1210918D12F8012481C4
:10D760003581468157816D857E858F8598890F9497
:10D77000C02C22966CAF7DAF8EAF9FAF22972BED62
:10D780003FE049E450E4C301B2010F94572620E082
:10D7900030E044E353E40F94BB2D6B017C010F9404
:10D7A000B62D6FA778AB89AB9AABD8012D913D917F
:10D7B0004D915C9169857A858B859C850F94C02CF1
:10D7C00026966CAF7DAF8EAF9FAF2697A5019401D3
:10D7D0006FA578A989A99AA90F9457269B01AC0136
:10D7E00026966CAD7DAD8EAD9FAD26970F94C12C66
:10D7F00069837A838B839C83C701B6010F94612F61
:10D80000A50194010F94572622962CAD3DAD4EAD47
:10D810005FAD22970F94C12C6D837E838F83988791
:10D8200048E651E070E060E0CE0101960E940BC234
:10D8300048E651E070E060E0CE0105960E940BC220
:10D84000BDA1B43099F449815A816B817C8186E411
:10D850009DE00E945C414D815E816F8178858EE6FE
:10D860009FE20E945C418AE00E944738198A1A8A26
:10D870001B8A1C8AAE014F5E5F4FBE016B5F7F4FFC
:10D88000CE0101960E94AE64339402CF20E04FA9EE
:10D89000BE01635F7F4FCE0109960E94AFF94B0135
:10D8A0005C01312CAC019B010F94B32F811102C09C
:10D8B00033243394A5019401C501B4010F94B32F0F
:10D8C0008111E2C0EFA1F8A5EE0FFF1FEE0FFF1FC1
:10D8D0002BAD3CADE20FF31F80829182A282B38216
:10D8E000A50194016D8D7E8D8F8D98A10F94212FB0
:10D8F000181624F48D8E9E8EAF8EB8A2A5019401C9
:10D9000069A17AA18BA19CA10F94F12587FF04C086
:10D9100089A29AA2ABA2BCA2A50194016BA97CA981
:10D920008DA99EA90F94C12C6BAB7CAB8DAB9EAB2C
:10D93000ADA5BEA5BD01BB0F880B990B0F94F825B3
:10D940006FA378A789A79AA79B01AC016BA97CA9B3
:10D950008DA99EA90F94BB2D2B013C014D8A5E8A97
:10D960006F8A788EEBADFCADF8ABEFA710E0C12C61
:10D97000D12C7601AFA5B8A96D917D918D919D9126
:10D98000B8ABAFA7A30192010F94C02C9B01AC01CF
:10D990000F9457269B01AC01C701B6010F94C12C0F
:10D9A0006B017C011F5F211628F72FA138A549A51F
:10D9B0005AA50F94BB2D0F946F2F698F7A8F8B8F81
:10D9C0009C8FBDA1B23068F18DA59EA50E946EE12D
:10D9D0006BA57CA581E49DE00E947E418BE39DE0E8
:10D9E0000E94803843E0C501B4010E948DBA80E2F4
:10D9F0000E94473881E0EDA1E3300CF480E0E12C97
:10DA00008E010F5D1F4F9E01235E3F4FAE01475EAB
:10DA10005F4FBE016B5E7F4F0E943D3F8AE00E94D8
:10DA200047382394B3CD0E94EE650E94F31C8DAD60
:10DA30000E945E690E94E23088AD99AD0FB6F894FD
:10DA40009EBF0FBE8DBFE8ADF9AD0FB6F894FEBF17
:10DA50000FBEEDBFC55BDF4F0FB6F894DEBF0FBE44
:10DA6000CDBFDF91CF911F910F91FF90EF90DF908D
:10DA7000CF90BF90AF909F908F907F906F905F906E
:10DA80004F903F902F9008950E94EE65332069F2E9
:10DA900080E39DE00E94803881E0FDA11F160CF01C
:10DAA00080E0EE24E3948E010F5D1F4F9E01235E04
:10DAB0003F4FAE01475E5F4FBE016B5E7F4F0E94DE
:10DAC0003D3F698D7A8D8B8D9C8D0052110926E02A
:10DAD00042E00F94BE209F938F938FE19DE09F9330
:10DAE0008F9389E29DE09F938F931F920E943EF94E
:10DAF0002DB73EB7295F3F4F0FB6F8943EBF0FBE1C
:10DB00002DBF93CF2F923F924F925F926F927F9251
:10DB10008F929F92AF92BF92CF92DF92EF92FF923D
:10DB20000F931F93CF93DF93CDB7DEB76A970FB6EE
:10DB3000F894DEBF0FBECDBF83E50E94771E182F7D
:10DB40003090400C882319F00E949324382E409086
:10DB50006102509062026090630270906402809152
:10DB6000650290916602A0916702B09168028B8B6A
:10DB70009C8BAD8BBE8B8091690290916A02A091C3
:10DB80006B02B0916C028F8B988FA98FBA8F112383
:10DB900029F0311003C080E00E945E6986E50E9492
:10DBA000771E8A8B20E030E0A9016091ED0570912D
:10DBB000EE058091EF059091F0050F94F1258823F3
:10DBC00009F4C9C083E40E94771E882309F49DC02C
:10DBD0000E94CB246B017C01A7EAB7E0B987A88734
:10DBE000BF83AE83F5E0FD831D861E8628EC2F875C
:10DBF00002EC1A86212C88EC8B8792E49C87AE81FC
:10DC0000BF81B98BA88B15E0E889F9898190919043
:10DC1000A190B190F98BE88B2A85322D4B855C85DC
:10DC2000C501B4010F94F12587FF04C08A86292C11
:10DC3000AB86BC862D853E854F85502FC501B4012E
:10DC40000F94212F181624F48D869E86AF860B2DF7
:10DC50001150D1F6FD81F150FD838E819F81449654
:10DC60009F838E83F111CBCF2D853E854F85502F1D
:10DC70006A85722D8B859C850F94C12C20E030E045
:10DC800040E05FE30F945726A70196010F94C12C43
:10DC90004B015C012DEB37E346E855EB0F94212F48
:10DCA00087FD0AC02DEB37E346E855E3C501B40113
:10DCB0000F94F12518164CF580E00E945E6910E083
:10DCC000E884F98400E0D7016D917D918D919D915B
:10DCD0007D016D01B4E0CB1AD108A50194010F9428
:10DCE000C02CF6016083718382839383602F812F20
:10DCF0000E9413F80F5F053031F71F5F8885998503
:10DD00004496998788871530D9F6AA89AA2381F085
:10DD100020E030E0A9016091ED057091EE05809161
:10DD2000EF059091F0050F94F12581110E94C540F7
:10DD30008AE50E94771E882351F00E94CB246983D4
:10DD40007A838B839C83CE0101960E94DBF6832D20
:10DD50000E945E690BC0311003C09A89992341F378
:10DD60000E94534E80E69CE00E948038332051F0A0
:10DD70008091400C811106C00E944F4E81E49CE0CE
:10DD80000E9480380E94534E83E39CE00E948038BA
:10DD90008091400C0E943E410E94534E86E29CE0DE
:10DDA0000E948038C090E308D090E408E090E50835
:10DDB000F090E60820E030E0A901C701B6010F9419
:10DDC000212F18160CF053C042E0C701B6010E9483
:10DDD0008DBA8DE00E9447388AE00E944738A3013F
:10DDE0009201609161027091620280916302909150
:10DDF00064020F94F12581111FC02B893C894D8944
:10DE00005E896091650270916602809167029091CF
:10DE100068020F94F12581110FC02F89388D498D2B
:10DE20005A8D6091690270916A0280916B029091A3
:10DE30006C020F94F12581110E94E2306A960FB6B0
:10DE4000F894DEBF0FBECDBFDF91CF911F910F9130
:10DE5000FF90EF90DF90CF90BF90AF909F908F900A
:10DE60007F906F905F904F903F902F90089581E248
:10DE70009CE00E948038B3CF8F929F92AF92BF9266
:10DE8000EF92FF920F931F93CF93DF9380E00E9456
:10DE90005E691092E9051092EA051092EB05109266
:10DEA000EC051092E5051092E6051092E705109238
:10DEB000E8051092F1051092F2051092F305109208
:10DEC000F4051092ED051092EE051092EF051092F8
:10DED000F00507EA17E0C0E0812C912C80ECA82E19
:10DEE0008FE7B82E7801D0E0F70181929192A1924C
:10DEF000B1927F016D2F8C2F0E9413F8DF5FD53018
:10DF000099F7CF5F0C5E1F4FC53061F7DF91CF915E
:10DF10001F910F91FF90EF90BF90AF909F908F90C7
:10DF200008959091911280919212981308C0809157
:10DF30001B0990911C09892B11F40C94311F80E06E
:10DF40000E945B5AEECF83E50E94C51E8823E9F04C
:10DF50000E9451FD60937E1170937F118093801118
:10DF6000909381110E94CB2420E030E04AE754E4F2
:10DF70000F9457260F94342E60931302709314025B
:10DF80008093150290931602089580914B0584FDAD
:10DF90000AC080914D0587FD06C080914E058370B3
:10DFA00011F40C94916F0E94C56188E50E94771E60
:10DFB000882331F05F9A80913F0C8E7F80933F0CD5
:10DFC00089E50E94771E882331F08A9A80913F0C60
:10DFD0008D7F80933F0C8AE50E94771E882359F03D
:10DFE00080910801809581708093060180913F0C9B
:10DFF0008B7F80933F0C85E40E94771E81110C94E7
:10E000002F1F08952F923F924F925F926F927F92AF
:10E010008F929F92AF92BF92CF92DF92EF92FF9238
:10E020000F931F93CF93DF93CDB7DEB7A6970FB6AD
:10E03000F894DEBF0FBECDBF8BE897E00E945C2A4C
:10E040008091FD0B83FD7EC020916D0230916E02A8
:10E0500040916F02509170026091970770919807FC
:10E060008091990790919A070F94F125882309F4DC
:10E0700069C010911A09111161C080915F029091DD
:10E08000600201972091F3113091F411281739079C
:10E090003CF40E94534E8AE299E10E94803811E0DC
:10E0A00020916D0230916E0240916F02509170028A
:10E0B00060919707709198078091990790919A07BE
:10E0C0000F94C02C6B017C0120E030E0A9010F947B
:10E0D000212F87FF04C0F7FAF094F7F8F09420910D
:10E0E0007102309172024091730250917402C70123
:10E0F000B6010F94572620E030E84BE354E40F9428
:10E10000212F1816ECF40E94534E8BE099E10E94E7
:10E1100080388091970790919807A0919907B091C6
:10E120009A0780936D0290936E02A0936F02B09352
:10E13000700287E997E00E94D66104C010E0B0CF7A
:10E140001111E7CF2AE037ED43E25CE36091410231
:10E150007091420280914302909144020F9457269D
:10E160006B017C016091770270917802072E000CA0
:10E17000880B990B0F94F8259B01AC01C701B601E0
:10E180000F945726698B7A8B8B8B9C8B8091400CDC
:10E19000882309F18090E3089090E408A090E508B6
:10E1A000B090E608C0909307D0909407E090950750
:10E1B000F090960720E030E0A901C501B4010F946A
:10E1C000F1258823D1F1A7019601C501B4010F946F
:10E1D000212F181694F1C12CD12C76018E010F5EDF
:10E1E0001F4F27E937E043E957E06FE877E08BE816
:10E1F00097E00E9494F480E1EBE8F7E0A1E6B2E05A
:10E2000001900D928A95E1F7A6960FB6F894DEBFBD
:10E210000FBECDBFDF91CF911F910F91FF90EF9077
:10E22000DF90CF90BF90AF909F908F907F906F9036
:10E230005F904F903F902F90089520916102309110
:10E240006202409163025091640260918B07709169
:10E250008C0780918D0790918E070F94C02C6D8B49
:10E260007E8B8F8B988F2091650230916602409152
:10E2700067025091680260918F07709190078091BA
:10E280009107909192070F94C02C698F7A8F8B8F92
:10E290009C8F2091690230916A0240916B025091EB
:10E2A0006C02C701B6010F94C02C6D8F7E8F8F8FCB
:10E2B00098A320916D0230916E0240916F025091AF
:10E2C00070026091970770919807809199079091DB
:10E2D0009A070F94C02C6B017C0120E030E0A9016B
:10E2E0006D897E898F89988D0F94F12581110CC0DD
:10E2F00020E030E0A901698D7A8D8B8D9C8D0F9483
:10E30000F125882309F467CF2D893E894F89588DDF
:10E31000CA01B9010F9457264B015C01298D3A8D32
:10E320004B8D5C8DCA01B9010F9457269B01AC013E
:10E33000C501B4010F94C12C4B015C012D8D3E8DA4
:10E340004F8D58A1CA01B9010F9457269B01AC010A
:10E35000C501B4010F94C12C4B015C01A7019601CA
:10E36000C701B6010F9457269B01AC01C501B4014A
:10E370000F94C12C0F946F2F4B015C012DEB37E3F1
:10E3800046E855E30F94F12587FF0FC020E030E009
:10E39000A901C701B6010F94212F4601570187FF3C
:10E3A00004C0B7FAB094B7F8B0942DEB37E346E861
:10E3B00055E3C501B4010F94F12587FD1CCF20E082
:10E3C00030E040EA51E4C501B4010F94BB2D0F9435
:10E3D000342E1B01672B19F422242394312CB10114
:10E3E00090E080E00F94F6259B01AC0160E070E0C6
:10E3F00080E89FE30F94BB2D2B013C01AC019B01F6
:10E40000C501B4010F9457264B015C01A301920191
:10E410006D897E898F89988D0F9457266D8B7E8BA1
:10E420008F8B988FA3019201698D7A8D8B8D9C8D36
:10E430000F945726698F7A8F8B8F9C8FA30192013F
:10E440006D8D7E8D8F8D98A10F9457266D8F7E8F49
:10E450008F8F98A3A3019201C701B6010F9457268D
:10E4600069A37AA38BA39CA380E1E1E6F2E08E018D
:10E470000F5F1F4FD80101900D928A95E1F70E941E
:10E4800051FD2B013C0128EC420E511C611C711CFA
:10E490000DA31EA381E0281A310809F460C00E9470
:10E4A00051FD8B019C01041915092609370937FD17
:10E4B00059C02B013C0128EC420E511C611C711CFF
:10E4C00080E00E945B5A2D893E894F89588D698171
:10E4D0007A818B819C810F94C12C69837A838B8391
:10E4E0009C83298D3A8D4B8D5C8D6D817E818F81D2
:10E4F00098850F94C12C6D837E838F8398872D8D93
:10E500003E8D4F8D58A169857A858B859C850F94AA
:10E51000C12C69877A878B879C8729A13AA14BA157
:10E520005CA16D857E858F8598890F94C12C6D8740
:10E530007E878F87988B750164018E010F5E1F4F58
:10E540009E01235F3F4FAE01475F5F4FBE016B5F90
:10E550007F4F8DA19EA10E9494F481119BCF7501E4
:10E5600064013CCE0E944DC2AECF8F929F92AF927B
:10E57000BF92CF92DF92EF92FF92CF93DF93809082
:10E58000410290904202A0904302B0904402FC01EC
:10E59000C080D180E280F38020E030E0A901C70193
:10E5A000B6010F94F125882341F0C0924102D09228
:10E5B0004202E0924302F0924402C0917702D0916D
:10E5C000780284E690E09093780280937702C0907E
:10E5D0007102D0907202E0907302F090740280E0B9
:10E5E00090E0A0E8BFE38093710290937202A09341
:10E5F0007302B09374020E94027080924102909262
:10E600004202A0924302B0924402D0937802C09397
:10E610007702C0927102D0927202E0927302F0927D
:10E620007402DF91CF91FF90EF90DF90CF90BF9079
:10E63000AF909F908F9008950F931F93CF93DF9388
:10E6400000D01F92CDB7DEB79C010BE817E090E138
:10E65000E1E6F2E0D80101900D929A95E1F7F90117
:10E660002081318142815381F801608571858285E5
:10E6700093850F94C12CF8016087718782879387F7
:10E6800080E090E0A0EAB0E489839A83AB83BC8306
:10E69000CE0101960E94B5720F900F900F900F90CF
:10E6A000DF91CF911F910F9108952F923F924F923A
:10E6B0005F926F927F928F929F92AF92BF92CF9212
:10E6C000DF92EF92FF921F93CF93DF93CDB7DEB728
:10E6D0002C970FB6F894DEBF0FBECDBF7A0119019B
:10E6E000DC012D913D914D915C912D833E834F83B3
:10E6F0005887FB0140805180628073808090610266
:10E7000090906202A0906302B0906402A50194010F
:10E710006D817E818F8198850F94F12581110EC0C6
:10E7200011E0A301920160916502709166028091EF
:10E730006702909168020F94F125811110E0D101D8
:10E740002D913D914D915C9129873A874B875C874C
:10E75000F701C080D180E280F38020910B023091DC
:10E760000C0240910D0250910E02C701B6010F94A8
:10E77000F125882309F44EC0C0920B02D0920C02FE
:10E78000E0920D02F0920E0280916D0290916E0265
:10E79000A0916F02B09170024091650250916602A3
:10E7A000609167027091680280928B0790928C074B
:10E7B000A0928D07B0928E0740938F0750939007D9
:10E7C0006093910770939207C0929307D092940739
:10E7D000E0929507F0929607809397079093980799
:10E7E000A0939907B0939A0720E030E040E05FE300
:10E7F00060916D0C70916E0C80916F0C9091700C0B
:10E800000F94572669837A838B839C83CE0101966C
:10E810000E94B5722D813E814F81588520938B07D0
:10E8200030938C0740938D0750938E0740928F074B
:10E83000509290076092910770929207D1012D91AA
:10E840003D914D915C9160919707709198078091EF
:10E85000990790919A070F94C12C60939707709332
:10E8600098078093990790939A0711112FC020E081
:10E8700030E0A90169857A858B859C850F94F12507
:10E88000811133C060E070E088EC92E469837A83A0
:10E890008B839C83CE0101960E94B5722C960FB695
:10E8A000F894DEBF0FBECDBFDF91CF911F91FF90D7
:10E8B000EF90DF90CF90BF90AF909F908F907F9020
:10E8C0006F905F904F903F902F9008952AEF3EE712
:10E8D0004AE25FE36091710C7091720C8091730C4D
:10E8E0009091740C0F945726D1CF60E070E080EACD
:10E8F00091E4CCCF0F931F93CF93DF9300D000D040
:10E900001F921F92CDB7DEB78B01FC0123A5211109
:10E9100002C00E949CFB1D821E821F82188620E07E
:10E9200030E040E05FE36091690270916A0280919B
:10E930006B0290916C020F94C12C69837A838B8354
:10E940009C839E012B5F3F4FAE014F5F5F4F65E69B
:10E9500072E081E692E00E9455731D821E821F8242
:10E96000188620E030E040E05FE3F80160857185C3
:10E97000828593850F94C12C69837A838B839C83D2
:10E98000B8016C5F7F4F9E012B5F3F4FAE014F5F21
:10E990005F4FC8010E94557328960FB6F894DEBFEA
:10E9A0000FBECDBFDF91CF911F910F9108959B01B5
:10E9B000AC01485F5F4FBC016C5F7F4F0C94557397
:10E9C0002F923F924F925F926F927F928F929F927F
:10E9D000AF92BF92CF92DF92EF92FF920F931F936D
:10E9E000CF93DF93CDB7DEB7A6970FB6F894DEBF0F
:10E9F0000FBECDBF8C011B015A8749874090610231
:10EA00005090620260906302709064028090650290
:10EA100090906602A0906702B0906802DB018D9131
:10EA20009D910D90BC91A02D8B8B9C8BAD8BBE8B43
:10EA30009C01AD01C301B2010F94C02C6B017C019C
:10EA4000D10114968D919D910D90BC91A02D8F8B2D
:10EA5000988FA98FBA8F9C01AD01C501B4010F94A5
:10EA6000C02C6B8F7C8F8D8F9E8FA985BA858D91E1
:10EA70009D910D90BC91A02D8B879C87AD87BE8703
:10EA80009C01AD01C301B2010F94C02C6F8F78A31C
:10EA900089A39AA3A985BA8514968D919D910D900D
:10EAA000BC91A02D8F87988BA98BBA8B9C01AD014F
:10EAB000C501B4010F94C02C6BA37CA38DA39EA3AE
:10EAC000A7019601C701B6010F9457266B017C017F
:10EAD0002B8D3C8D4D8D5E8DCA01B9010F9457264B
:10EAE0009B01AC01C701B6010F94C12C4B015C0125
:10EAF0002B893C894D895E896B857C858D859E85BA
:10EB00000F94C02C2B013C012F89388D498D5A8DD3
:10EB10006F85788989899A890F94C02C6B017C0153
:10EB2000A3019201C301B2010F9457262B013C01AE
:10EB3000A7019601C701B6010F9457269B01AC01AE
:10EB4000C301B2010F94C12C0F946F2F6B017C0194
:10EB50002F8D38A149A15AA1CA01B9010F94572696
:10EB60002B013C012BA13CA14DA15EA1CA01B90121
:10EB70000F9457269B01AC01C301B2010F94C12C25
:10EB80009B01AC01C501B4010F94212F1816B4F5F7
:10EB900020E030E0A901C701B6010F94212F87FFC3
:10EBA0002AC0C701B601905820E030E040EA50E4A6
:10EBB0000F94212F181614F5A10169857A85C801D3
:10EBC0000E94E074A6960FB6F894DEBF0FBECDBFCC
:10EBD000DF91CF911F910F91FF90EF90DF90CF9039
:10EBE000BF90AF909F908F907F906F905F904F906D
:10EBF0003F902F900895C701B601D6CF20E030E0B6
:10EC000040E050E4C501B4010F94212F181624F4FC
:10EC1000B101C8010E947A7419821A821B821C8277
:10EC2000BE016F5F7F4FC1010E94D7742DEC3CEC99
:10EC30004CEC5CE3C701B6010F9457269B01AC0175
:10EC4000F80160817181828193810F9457266D83D1
:10EC50007E838F839887D8019B968C919B9788237E
:10EC6000C9F02AE939E949E95FE314966D917D918C
:10EC70008D919C9117970F94572669837A838B8384
:10EC80009C83BE016F5F7F4F8BE897E00E94D77433
:10EC9000F80113A6BE016B5F7F4F89859A850E949C
:10ECA000D77490CF3F924F925F926F927F928F92E4
:10ECB0009F92AF92BF92CF92DF92EF92FF920F930B
:10ECC0001F93CF93DF93CDB7DEB76C970FB6F89451
:10ECD000DEBF0FBECDBFDB010C91142F100F15301E
:10ECE00008F067C11196DC90C22ECD0CB4E0BC15C3
:10ECF00008F45FC1ED2DF0E0EE5EFA4F8080912CBC
:10ED0000B12CA12C002E04C0B694A794979487949C
:10ED10000A94D2F780FE4DC1EC2DF0E0EE5EFA4F82
:10ED20008080912CB12CA12C012E04C0B694A79404
:10ED3000979487940A94D2F780FE3BC1322E642FB9
:10ED40007C014090E5055090E6056090E7057090E5
:10ED5000E8058091ED059091EE05A091EF05B09149
:10ED6000F005898F9A8FAB8FBC8F660F770B072EBC
:10ED7000000C880B990B0F94F8254B015C01602F58
:10ED8000000F770B880B990B0F94F825298D3A8D7E
:10ED90004B8D5C8D0F945726A30192010F94C12CCB
:10EDA000A50194010F94C12C6D877E878F87988B66
:10EDB000612F110F770B880B990B0F94F825298D74
:10EDC0003A8D4B8D5C8D0F945726A30192010F94C1
:10EDD000C12CA50194010F94C02C69837A838B8385
:10EDE0009C834090E9055090EA056090EB05709097
:10EDF000EC058091F1059091F205A091F305B09199
:10EE0000F405898F9A8FAB8FBC8F632D660F770BBC
:10EE1000072E000C880B990B0F94F8254B015C0111
:10EE20006D2DDD0C770B880B990B0F94F825298D30
:10EE30003A8D4B8D5C8D0F945726A30192010F9450
:10EE4000C12CA50194010F94C12C698B7A8B8B8BFB
:10EE50009C8B6C2DCC0C770B880B990B0F94F825A1
:10EE6000298D3A8D4B8D5C8D0F945726A30192010D
:10EE70000F94C12CA50194010F94C02C6D837E8347
:10EE80008F839887F70180859185A285B3858987CF
:10EE90009A87AB87BC878D8B9E8BAF8BB88F47E6ED
:10EEA00051E061E070E0CE0141960E940BC247E65E
:10EEB00051E061E070E0CE0105960E940BC247E68A
:10EEC00051E061E070E0CE010D960E940BC247E672
:10EED00051E061E070E0CE0101960E940BC289888A
:10EEE0009A88AB88BC8827E137EB41ED58EBC50128
:10EEF000B4010F94212F87FD5CC023E030E044EB88
:10EF000053E4C501B4010F94F12518160CF451C057
:10EF10008D849E84AF84B88827E137EB41ED58EBB0
:10EF2000C501B4010F94212F87FD43C023E030E0D9
:10EF300044EB53E4C501B4010F94F1251816CCF14C
:10EF40008D809E80AF80B88427E137EB41ED58EB90
:10EF5000C501B4010F94212F87FD2BC023E030E0C1
:10EF600044EB53E4C501B4010F94F12518160CF1DC
:10EF700089809A80AB80BC8027E137EB41ED58EB6C
:10EF8000C501B4010F94212F87FD13C023E030E0A9
:10EF900044EB53E4C501B4010F94F12518164CF06D
:10EFA000AE014F5F5F4FBE01635F7F4FC7010E949D
:10EFB000E0746C960FB6F894DEBF0FBECDBFDF9144
:10EFC000CF911F910F91FF90EF90DF90CF90BF9066
:10EFD000AF909F908F907F906F905F904F903F90F9
:10EFE00008952F923F924F925F926F927F928F92ED
:10EFF0009F92AF92BF92CF92DF92EF92FF920F93C8
:10F000001F93CF93DF93CDB7DEB7CC58D1090FB69E
:10F01000F894DEBF0FBECDBF80E19CE00E94803837
:10F0200087E00E94634E81116EC084E50E94C51E78
:10F03000882329F00E94B82481110E947BBA80E0C5
:10F0400090E0A0E8BFE389839A83AB83BC838D8380
:10F050009E83AF83B8878DEC9CECACE4BEE38987DC
:10F060009A87AB87BC8780E090E0A0E2B1E48D870F
:10F070009E87AF87B88B8CE390E09A8B898B8DEC61
:10F0800090E09C8B8B8B8DEC9CECACECBEE38D8B81
:10F090009E8BAF8BB88F80E090E0A0EEBFE3898FAE
:10F0A0009A8FAB8FBC8F1BA61CA64AE959E969E968
:10F0B0007EE38FE40E94F5246D8F7E8F8F8F98A35F
:10F0C00060E083E40E94A32489A360E08BE40E94B3
:10F0D000A3248AA382E40E94C51E882381F10E9492
:10F0E000B824009761F19C01285231092536310579
:10F0F00020F16CE870E082EE9BE00E947E418DED95
:10F100009BE00E948038C457DF4F0FB6F894DEBFF3
:10F110000FBECDBFDF91CF911F910F91FF90EF9068
:10F12000DF90CF90BF90AF909F908F907F906F9027
:10F130005F904F903F902F9008959A8B898B8CE42D
:10F140000E94C51E8823E1F00E94CB246B017C0144
:10F15000C986DA86EB86FC8620E030E0A9010F94B0
:10F16000212F87FD0AC020E030E040E050E4C701D5
:10F17000B6010F94F12518161CF485EB9BE0C1CF66
:10F1800081E50E94771E882331F180911B059091C3
:10F190001C05892BE9F00E94CB246B017C01CD82F8
:10F1A000DE82EF82F8862DEC3CEC4CE45DE30F94BC
:10F1B000212F87FD0AC020E030E040E751E4C7017D
:10F1C000B6010F94F125181634F484E89BE099CF2A
:10F1D00089E59BE096CF83E50E94C51E8823E9F070
:10F1E0000E94CB246B017C01CD8ADE8AEF8AF88EE7
:10F1F0002DEC3CEC4CEC5DE30F94212F87FD0AC015
:10F2000020E030E040E050E4C701B6010F94F12562
:10F2100018161CF482E39BE074CF80E50E94771EF1
:10F22000882341F180911B0590911C05892B19F4CD
:10F230008AEF9AE066CF8BA58F5F8BA70E94CB24C5
:10F240006B017C01CD86DE86EF86F88A20E030E017
:10F25000A9010F94212F87FD0AC020E030E048EC7F
:10F2600051E4C701B6010F94F12518161CF482ED84
:10F270009AE047CF86E40E94C51E8823E9F00E94E9
:10F28000CB246B017C01C98EDA8EEB8EFC8E20E0E4
:10F2900030E040E85FE30F94212F87FD0AC020E0B3
:10F2A00030E040E850E4C701B6010F94F12518168C
:10F2B0001CF489EA9AE025CFC98CDA8CEB8CFC8CA3
:10F2C0008D889E88AF88B88CA7019601C701B601CA
:10F2D0000F9457269B01AC0160E070E084E490E459
:10F2E0000F94BB2D29813A814B815C810F94572665
:10F2F0002B013C01A5019401C501B4010F945726CF
:10F30000A70196010F9457262CEE31E548EB5DE3FB
:10F310000F94BB2D9B01AC01C301B2010F94572682
:10F3200069837A838B839C8388E40E94C51E88232B
:10F3300079F00E94B824009759F09C01255A3109B0
:10F340002838310518F08BE79AE0DBCE9C8B8B8B4D
:10F3500085E50E94771E8823C9F00E9451FD611542
:10F3600071058105910511F00F94772180911B059E
:10F3700090911C05892B91F00E94CB246093170576
:10F38000709318058093190590931A0582E50E94E1
:10F39000771E811108C087E49AE0B3CE60E070E088
:10F3A00088E492E4EBCF80911B0590911C05892B9A
:10F3B00061F00E94B824AD969FAF8EAFAD9718163E
:10F3C00019064CF083E19AE09CCE2AE130E0AD963C
:10F3D0003FAF2EAFAD9789E50E94C51E882381F10E
:10F3E0000E94CB242091EB083091EC084091ED086D
:10F3F0005091EE080F94C02C6B017C0188E50E94AF
:10F40000C51E882331F10E94CB242091E70830915A
:10F41000E8084091E9085091EA080F94C02C6BA3CA
:10F420007CA38DA39EA3CFA2D8A6E9A6FAA6CE015F
:10F4300083960E94361E811115C089EE99E061CE37
:10F44000C0906502D0906602E0906702F09068027A
:10F45000D5CF6091610270916202809163029091B8
:10F460006402DDCF84E40E94771E91E089270E9428
:10F470005E6980E090E0A0EAB0E48DA79EA7AFA708
:10F48000B8AB60E0CE018D960E94186530911008EF
:10F49000CD57DF4F3883C358D040109210080E94D8
:10F4A000301C88EC99E00E94803889899A898A31D9
:10F4B00091050CF044C08B899C890E944D1F61E02E
:10F4C00080E00E941BBD811142C06FEF8DED99E07D
:10F4D0000E94EE3F8CA5811104C0CE0101960E94CE
:10F4E0009CFB80E090E0A0EAB0E4809393079093C7
:10F4F0009407A0939507B09396071DA61EA61FA676
:10F5000018AABE01635D7F4F8BE897E00E94D77415
:10F51000CD57DF4F5881C358D040509310080E94F8
:10F52000301C8AA18111EFCD10928B1110928A119B
:10F530000E94D3BE90E080E00E944D1FE4CD0E9467
:10F540008B2281E00E94A4BB8111B5CFBECF109267
:10F550006D0210926E0210926F02109270028DE690
:10F5600092E00E94D6618BA5882309F452C020E066
:10F5700030E040E751E46091710C7091720C809121
:10F58000730C9091740C0F94BB2D6DA77EA78FA761
:10F5900098AB80E1E1E6F2E0ABE8B7E001900D92D4
:10F5A0008A95E1F72D853E854F85588960919707AB
:10F5B000709198078091990790919A070F94C12CA8
:10F5C00060939707709398078093990790939A0791
:10F5D000CE018D960E94B5722D853E854F85588946
:10F5E00060919707709198078091990790919A0779
:10F5F0000F94C02C60939707709398078093990796
:10F6000090939A078CA5811104C0CE0101960E94A7
:10F610009CFBE2E1F5E085E0DF011D928A95E9F7C8
:10F6200080E1E1E6F2E0ABE8B7E001900D928A9567
:10F63000E1F789859A85AB85BC8580939307909384
:10F640009407A0939507B09396071DA61EA61FA624
:10F6500018AABE01635D7F4F8BE897E00E94D774C4
:10F66000BE01635E7F4F8BE897E00E94D77489A14B
:10F67000882309F41CC420916102309162024091F8
:10F68000630250916402E5962CAF3DAF4EAF5FAF81
:10F69000E5978091650290916602A0916702B09112
:10F6A0006802E1968CAF9DAFAEAFBFAFE197312C52
:10F6B000212C9FEFA4969FAFA497AFEFA896AFAF72
:10F6C000A897BFEFC158DF4FB883CF57D040EFE4C2
:10F6D000C058DF4FE883C058D040F3ECCF57DF4F1E
:10F6E000F883C158D04027E4CE57DF4F2883C25853
:10F6F000D04081E090E0A0E0B0E0022C04C0880F90
:10F70000991FAA1FBB1F0A94D2F7CC57DF4F8883DB
:10F710009983AA83BB83C458D040A2E1B5E0E796A1
:10F72000BFAFAEAFE79710E000E09101032C000CF3
:10F73000440B550BC857DF4F288339834A835B83BB
:10F74000C858D040C457DF4F2882CC58D040E796E5
:10F75000AEADBFADE7978D91E796BFAFAEAFE79780
:10F7600090E0B0E0A0E0CC57DF4F288139814A819A
:10F770005B81C458D04082239323A423B523892BD3
:10F780008A2B8B2B09F024C1C857DF4F6881798100
:10F790008A819B81C858D0400F94F8252091ED05AF
:10F7A0003091EE054091EF055091F0050F945726EA
:10F7B0002091E5053091E6054091E7055091E80577
:10F7C0000F94C12CEB966CAF7DAF8EAF9FAFEB97D4
:10F7D000B801012E000C880B990B0F94F82520918D
:10F7E000F1053091F2054091F3055091F4050F9425
:10F7F00057262091E9053091EA054091EB0550919B
:10F80000EC050F94C12C6B017C01EB962CAD3DAD4A
:10F810004EAD5FADEB97E5966CAD7DAD8EAD9FAD1A
:10F82000E5970F94C02C2B013C01A7019601E196AE
:10F830006CAD7DAD8EAD9FADE1970F94C02C4B01AB
:10F840005C01A3019201C301B2010F9457262B0161
:10F850003C01A5019401C501B4010F9457269B01F9
:10F86000AC01C301B2010F94C12C0F946F2F4B0157
:10F870005C01EB962CAD3DAD4EAD5FADEB976BA152
:10F880007CA18DA19EA10F94C02C2B013C01A7014E
:10F8900096016FA178A589A59AA50F94C02C6B013C
:10F8A0007C01A3019201C301B2010F9457262B01E1
:10F8B0003C01A7019601C701B6010F9457269B0191
:10F8C000AC01C301B2010F94C12C0F946F2F20E043
:10F8D00030E040E751E40F94BB2DA50194010F9453
:10F8E000C12C6B017C018090170590901805A090A9
:10F8F0001905B0901A0520E030E040E85FE3C5014B
:10F90000B4010F94212F1816F4F4C501B4010F941B
:10F910002D2E4B015C0160E070E0CB01181419043E
:10F920001A041B0434F40F942821A50194010F94A8
:10F93000572C0F94F8259B01AC01B601C7010F9419
:10F94000C12C6B017C01C158DF4F2881CF57D040BB
:10F95000C058DF4F3881C058D040CF57DF4F488163
:10F96000C158D040CE57DF4F5881C258D040B60161
:10F97000C7010F94F12587FF2BC0A4960FAFA49762
:10F98000C457DF4F3881CC58D040A8963FAFA897D6
:10F99000EC96CFAEEC97ED96DFAEED97EE96EFAE30
:10F9A000EE97EF96FFAEEF97C158DF4FC882CF5763
:10F9B000D040C058DF4FD882C058D040CF57DF4F1B
:10F9C000E882C158D040CE57DF4FF882C258D040AD
:10F9D0000F5F1F4F0530110509F0B9CE4FEF241A04
:10F9E000340A55E02516310409F083CEA4968FAD74
:10F9F000A497E82FF0E0EE5EFA4F208181E090E0DE
:10FA0000A0E0B0E0A8960FACA89704C0880F991F9B
:10FA1000AA1FBB1F0A94D2F7822B8083A8969FADA2
:10FA2000A8976A969FAF6A97A496AFADA4976B9676
:10FA3000AFAF6B97EC968FADEC97ED969FADED97D2
:10FA4000EE96AFADEE97EF96BFADEF976F968CAF9A
:10FA50009DAFAEAFBFAF6F97A896BFADA897BF3FA2
:10FA600009F409C2A496EFADA497EF3F09F403C2CD
:10FA70006B2FBB0F770B880B990B0F94F8252091F8
:10FA8000ED053091EE054091EF055091F0050F9492
:10FA900057262091E5053091E6054091E705509104
:10FAA000E8050F94C12C162F072F382E292E862FEC
:10FAB000902FA32DB22D65968CAF9DAFAEAFBFAF8B
:10FAC0006597A496FFADA4976F2FFF0F770B880B58
:10FAD000990B0F94F8252091F1053091F205409192
:10FAE000F3055091F4050F9457262091E9053091C4
:10FAF000EA054091EB055091EC050F94C12C6B0188
:10FB00007C016996CCAEDDAEEEAEFFAE6997CE015C
:10FB10008F5A9F4F0E94361E882309F4B0C120E0FF
:10FB200030E040EA50E4612F702F832D922D0F9426
:10FB3000C12C4B015C01CB01D50121968CAF9DAF4F
:10FB4000AEAFBFAF21972596CCAEDDAEEEAEFFAE29
:10FB50002597A8962FADA8972111E3C1A4963FAD94
:10FB6000A4973111B3C120E030E040EA50E4C7016E
:10FB7000B6010F94C12C6B017C01A4964FADA497E4
:10FB8000442309F4C5C1A4968FADA49784300CF02A
:10FB9000BFC122ED422E23E5522E2BE7622E21E437
:10FBA000722E21968CAC9DACAEACBFAC2197259645
:10FBB0008CAD9DADAEADBFAD2597A7968CAF9DAF7B
:10FBC000AEAFBFAFA7979C01AD0169966CAD7DAD9F
:10FBD0008EAD9FAD69970F94C02CAB966CAF7DAF87
:10FBE0008EAF9FAFAB97A501940165966CAD7DADCF
:10FBF0008EAD9FAD65970F94C02C2D966CAF7DAFE9
:10FC00008EAF9FAF2D97AB962CAD3DAD4EAD5FAD9A
:10FC1000AB9761962CAF3DAF4EAF5FAF6197A5013B
:10FC200094016091610270916202809163029091EF
:10FC300064020F94C02C4B015C01A7962CAD3DAD26
:10FC40004EAD5FADA797609165027091660280919D
:10FC50006702909168020F94C02CA7966CAF7DAF9D
:10FC60008EAF9FAFA797812F902FA32DB22D8DA779
:10FC70009EA7AFA7B8ABC9AADAAAEBAAFCAAC98407
:10FC8000DA84EB84FC84CDAADEAAEFAAF8AE2DECD0
:10FC90003CEC4CEC5CE3C301B2010F945726298184
:10FCA0003A814B815C810F94572620916D023091EF
:10FCB0006E0240916F02509170020F94C12C69AF97
:10FCC0007AAF8BAF9CAFA5019401C501B4010F942D
:10FCD00057264B015C01A7962CAD3DAD4EAD5FADF7
:10FCE000A797CA01B9010F9457269B01AC01C50122
:10FCF000B4010F94C12C20E030E040E050E40F94B8
:10FD0000212F1816ACF420E030E040E05FE3C7019B
:10FD1000B6010F94C12C29966CAF7DAF8EAF9FAF0B
:10FD20002997BE01635C7F4FCE0101960E947A74D1
:10FD300089859A85AB85BC8529968CAF9DAFAEAF82
:10FD4000BFAF2997A3961CAE1DAE1EAE1FAEA397E4
:10FD5000BE01615A7F4FCE01CD960E94D7748CA50B
:10FD60008823C1F02AE939E949E95FE36D817E81A1
:10FD70008F8198850F945726A3966CAF7DAF8EAF79
:10FD80009FAFA397BE01615A7F4F8BE897E00E9417
:10FD9000D7741CA6E090690CF0906A0C00916B0C73
:10FDA00010916C0CA090650CB090660CC090670C24
:10FDB000D090680C9501A601B701C8010F94212FBE
:10FDC000181614F475018601809041029090420249
:10FDD000A0904302B09044022DEC3CEC4CEC5DE36F
:10FDE000B701C8010F9457266093410270934202F5
:10FDF000809343029093440240E0BE01675B7F4FD3
:10FE0000CE018D960F942A1580E1E1E6F2E0ABE891
:10FE1000B7E001900D928A95E1F7809241029092AD
:10FE20004202A0924302B092440220E04FEFBE0192
:10FE3000675A7F4FCE0101960E94527620E041E042
:10FE4000BE01675A7F4FCE0101960E9452762FEF76
:10FE500040E0BE01675A7F4FCE0101960E94527664
:10FE600021E040E0BE01675A7F4FCE0101960E941B
:10FE700052760E94C5618091AC0C8093AD0CAD961A
:10FE80004EAD5FADAD9741505109AD965FAF4EAFEE
:10FE9000AD97452B09F419CB6A968FAD6A9787FD0C
:10FEA00014CB6B968FAD6B9787FFE1CB0ECB2BA15D
:10FEB0003CA14DA15EA1E5962CAF3DAF4EAF5FAF2B
:10FEC000E5978FA198A5A9A5BAA5EBCB812F902F77
:10FED000A32DB22D21968CAF9DAFAEAFBFAF2197B2
:10FEE00020E030E040EA50E4C701B6010F94C02C96
:10FEF00025966CAF7DAF8EAF9FAF2597A4965FAD73
:10FF0000A49754300CF42FCE182D092D3A2C2B2CFD
:10FF100092ED492E93E5592E9BEF692E90E4792EB0
:10FF200040CEA8969FADA89794300CF452C0A496EA
:10FF3000AFADA497A4300CF120E030E040EA50E4EB
:10FF4000612F702F832D922D0F94C02C21966CAFB2
:10FF50007DAF8EAF9FAF219720E030E040EA50E4C4
:10FF6000C701B6010F94C02C6B017C01A496EFADC4
:10FF7000A497E4300CF40DCECBCF812F902FA32D7E
:10FF8000B22D21968CAF9DAFAEAFBFAF219720E0D1
:10FF900030E040EA50E4C701B6010F94C12C259629
:10FFA0006CAF7DAF8EAF9FAF2597A496BFADA497E2
:10FFB000B111D2CF20E030E040EA50E4612F702F41
:10FFC000832D922D0F94C02C162F072F382E292EFB
:10FFD0009FCFA496FFADA497F1110DC020E030E0B3
:10FFE00040E251E4B401C5010F94C02C162F072F35
:10FFF000382E292ECECDA4962FADA49724309CF078
:020000021000EC
:1000000020E030E040E251E4B401C5010F94C02C7F
:1000100021966CAF7DAF8EAF9FAF2197182D092D24
:100020003A2C2B2CB6CD182D092D3A2C2B2C82EDE9
:10003000482E83E5582E8BEF682E81E4782EB1CDC3
:100040002F923F924F925F926F927F928F929F92E8
:10005000AF92BF92CF92DF92EF92FF920F931F93D6
:10006000CF93DF93CDB7DEB7EE970FB6F894DEBF30
:100070000FBECDBF8091400C888B87E50E94771E14
:10008000882309F423C120E030E0A9016091ED0547
:100090007091EE058091EF059091F0050F94F12598
:1000A000811108C00E944F4E8DE09DE00E94803873
:1000B00010E01FC18AE50E94C51E882339F10E9405
:1000C000CB242091EF083091F0084091F108509135
:1000D000F2080F94C02C6B017C0120E030E040E27C
:1000E00051ECC701B6010F94212F87FD0AC020E013
:1000F00030E040E251E4C701B6010F94F125181633
:1001000074F40E944F4E80E09DE0D0CFC090690211
:10011000D0906A02E0906B02F0906C02DECF40E07B
:1001200050E060EC7FE788E50E94F5242091E70825
:100130003091E8084091E9085091EA080F94C02CEA
:100140002B013C0140E050E060EC7FE789E50E9434
:10015000F5242091EB083091EC084091ED08509186
:10016000EE080F94C02C4B015C016FEF89E40E94F4
:100170008724182F6FEF8AE40E948724082FA30199
:100180009201C301B2010F94B32F81116EC0A5017A
:100190009401C501B4010F94B32F811166C08BA1E6
:1001A0009CA1ADA1BEA18BAB9CABADABBEAB209176
:1001B000E5053091E6054091E7055091E805C3015A
:1001C000B2010F94C02C2B013C0120E030E040E054
:1001D0005FE36BA97CA98DA99EA90F9457269B016B
:1001E000AC01C301B2010F94C12C2BA93CA94DA9AC
:1001F0005EA90F94BB2D0F942D2E162F4FA058A43F
:1002000069A47AA42091E9053091EA054091EB05B3
:100210005091EC05C501B4010F94C02C4B015C0159
:1002200020E030E040E05FE3C301B2010F945726C5
:100230009B01AC01C501B4010F94C12CA301920133
:100240000F94BB2D0F942D2E062F812F012E000C05
:10025000990B97FD33C005979CF5802F002E000C5D
:10026000990B97FD2FC005977CF5153008F020CF2E
:10027000053008F01DCF80E00E945E6995E019020C
:10028000F0011124E00FF11D07FDFA95EE0FFF1F9D
:10029000EE0FFF1FE955F84FC082D182E282F38250
:1002A000602F812F0E9413F888890E945E698889D7
:1002B000882309F4FDCE0E94E230FACE10E0CDCFC3
:1002C00014E0CBCF00E0D1CF04E0CFCF8AE40E948E
:1002D000771E182F811127C070E060E086E50E942C
:1002E000BC249A838983059708F18BED9CE00E94DA
:1002F0008038812FEE960FB6F894DEBF0FBECDBFCB
:10030000DF91CF911F910F91FF90EF90DF90CF90F1
:10031000BF90AF909F908F907F906F905F904F9025
:100320003F902F9008950E943C6FC2CE60E084E41D
:100330000E94A3248F8740E050E0BA018AE50E9422
:10034000F5246BA77CA78DA79EA740E050E86BE340
:1003500076E483E50E94F52420E030E040E752E4B3
:100360000F94BB2D60933D0270933E0280933F0239
:1003700090934002E0908C12F0908D12D7018D90F6
:100380009D90AD90BC9020E030E0A901C501B40182
:100390000F94C12C6BAF7CAF8DAF9EAF20E030E0EF
:1003A00040E450E40F94F12587FF06C01BAE1CAE5D
:1003B000B0E4BDAFE0E4EEAF20E030E044EB53E466
:1003C000C501B4010F94C12C662E7BAB8FAB98AFE7
:1003D00020E030E842EB53E40F94212F18163CF450
:1003E000612CF0E8FBAB22EB2FAB33E438AFD70145
:1003F00014968D909D90AD90BC90179720E030E0C2
:10040000A901C501B4010F94C12CD62EE72EF82EF8
:10041000092F20E030E040EE51E40F94F12587FFF2
:1004200005C0D12CE12CF0EEFF2E01E420E030E0FD
:1004300044EB53E4C501B4010F94C12CB62EC72E72
:1004400089AF9AAF20E030E046EA53E40F94212FC1
:10045000181634F4B12CC12CB6EAB9AFE3E4EAAF14
:1004600088E40E94771E882309F416C20E94CB24D8
:100470000F942D2E1B0177FF02C06F5F7F4F759584
:1004800067957195619571096C547F4F072E000C2B
:10049000880B990B0F94F825762E872E982EA92E6F
:1004A0002D2D3E2D4F2D502F0F94212F18161CF45B
:1004B000D72C74010A2D2BAD3CAD4DAD5EAD672D33
:1004C000782D892D9A2D0F94212F181624F07BACAE
:1004D0008CAC9DACAEAC872D982DA92DBA2D8B8BF5
:1004E0009C8BAD8BBE8B8D2D9E2DAF2DB02F8F8B0A
:1004F000988FA98FBA8FB101330C880B990B0F9489
:10050000F8251B012C01AC019B016D2D7E2D8F2D3B
:10051000902F0F94C12CD62EE72EF82E092F2B2DBD
:100520003C2D49AD5AAD0F94F12587FF04C0BD2C79
:10053000CE2CF9AE0AAFA2019101672D782D892D3D
:100540009A2D0F94C12CD62EE72EF82E092F262D8A
:100550003BA94FA958AD0F94F12587FF04C06D2C1E
:10056000EBAAFFAA08AF862D9BA9AFA9B8AD8B8FC8
:100570009C8FAD8FBE8F8B2D9C2DA9ADBAAD8F8F6B
:1005800098A3A9A3BAA3BE01695E7F4FCE0143968B
:100590000E94822E882309F4B0C1BE01615E7F4FA4
:1005A000CE014B960E94822EE82E882309F4A5C125
:1005B0002F89388D498D5A8D6F8D78A189A19AA187
:1005C0000F94C02C20E030E040E85EE30F94572603
:1005D0004B015C012B893C894D895E896B8D7C8D3B
:1005E0008D8D9E8D0F94C02C20E030E040E85EE3BE
:1005F0000F9457266BA37CA38DA39EA38FA298A6CE
:10060000A9A6BAA689819A811816190674F489EAEE
:100610009CE00E9480388F85882321F08FE99CE040
:100620000E9480388AE00E9447380E94C5610E947B
:100630000C1D80E00E945E6980E090E0A0E2B1E4E1
:100640008FA798ABA9ABBAAB60E0CE018F960E94A2
:1006500018652091ED053091EE054091EF05509120
:10066000F0056BA17CA18DA19EA10F94F1258111B4
:1006700030C02091F1053091F2054091F305509181
:10068000F4056FA178A589A59AA50F94F12581118C
:1006900020C02091E5053091E6054091E705509195
:1006A000E8056B897C898D899E890F94F1258111DC
:1006B00010C02091E9053091EA054091EB05509179
:1006C000EC056F89788D898D9A8D0F94F12588239B
:1006D000A9F00E943C6F88E0FE01B396ADEEB5E054
:1006E00001900D928A95E1F788E0FE017396A5EEE0
:1006F000B5E001900D928A95E1F7188A60E085E4F3
:100700000E94A324882309F4FBC0F1E0FBAB1B8605
:100710001C861D861E861A8A9E2C4FE6C42E4CE02F
:10072000D42E5DE7A52E5CE0B52E1A8915300CF0AD
:10073000F7C06B857C858D859E859B01AC010F94F0
:10074000B32F8111EDC0992009F4DDC031E03FAB3A
:1007500035E0232E91E09926F12EFF0CFF0CF10ECF
:10076000F394898B19896A89121509F4D5C0062E6C
:10077000000C770B880B990B0F94F8252FA138A547
:1007800049A55AA50F9457262F89388D498D5A8D22
:100790000F94C12C2B013C01612F110F770B880B9B
:1007A000990B0F94F8252BA13CA14DA15EA10F94AC
:1007B00057262B893C894D895E890F94C12C6B8308
:1007C0007C838D839E834F82588669867A86898151
:1007D0009A81892B79F06F2D8BE89CE00E9454411F
:1007E00069E170E089E89CE00E947E4186E89CE037
:1007F0000E9480381F9299E19F931F92FF92DF928F
:10080000CF92BF92AF921F920E943EF929814BA9CD
:10081000BE01695F7F4FCE0103960E94AFF92B01A5
:100820003C014B865C866D867E860FB6F894DEBFF3
:100830000FBECDBFAC019B010F94B32F811169C0D6
:1008400089883A8825E0382D320380011124030D70
:10085000111D37FC1A95000F111F000F111F0955AC
:10086000184FA30192016BA57CA58DA59EA50F94A1
:10087000C12CD8016D937D938D939C931397632D19
:10088000882D0E9413F8188A81E00E945B5AF39425
:100890008989BFA98B0F65CF4D2D5E2D6F2D702FD0
:1008A00086E40E94F5241B012C014BAD5CAD6DADBF
:1008B0007EAD8CE40E94F5246B8B7C8B8D8B9E8BA4
:1008C0002F8A388E498E5A8E4B2D5C2D69AD7AADAC
:1008D00082E40E94F5246B017C01462D5BA96FA97F
:1008E00078AD82E50E94F5246B8F7C8F8D8F9E8F73
:1008F000CF8ED8A2E9A2FAA246CE8FEB9CE0F7CC2D
:1009000022E02BAB04CF8FEF8FAB22242A9484E01C
:1009100021CF88890E945E698A898F5F8A8B05CF83
:100920000E94A9E40E94EE65882359F088890E94FC
:100930005E6980E090E0A0ECBFE78B879C87AD8785
:10094000BE876B857C858D859E859B01AC010F9450
:10095000B32F811159C08F85811126C082E0F82EF6
:1009600002E094E0C92E12E0DC2CD11A21E041E033
:10097000612F802F0E94A42221E04FEF612F8F2D45
:100980000E94A4222FEF41E06D2D802F0E94A4220F
:100990002FEF4FEF6D2D8F2D0E94A422115020F7C5
:1009A0000150F3940F3FF9F60E94C5400E94D21EF9
:1009B0008F85811124C089E692E00E94BC1D4B0105
:1009C0005C0181E692E00E94621F9B01AC01C501BF
:1009D000B4010F9457269B01AC016091690270919C
:1009E0006A0280916B0290916C020F94C02C60930C
:1009F000690270936A0280936B0290936C028F85F8
:100A00008111E888E092400C0E94F31C8091400C18
:100A100081110E942F2B0E94D8670E94E2306B85C3
:100A20007C858D859E8511E09B01AC010F94B32FD1
:100A300081115FCC3DCB8F929F92AF92BF92CF92AC
:100A4000DF92EF92FF920F931F93CF93DF9300D02B
:100A50001F92CDB7DEB75C016B017A01122F002324
:100A6000E1F10E94534E88E999E00E94803861E0EC
:100A7000812F0E94743A90902C0583E080932C057E
:100A800081E080933E0C0E946B4082E0809399113C
:100A900040E368E879E084E799E00E94704040E034
:100AA00069E171E18DE699E00E94704061E088E6BD
:100AB00099E00E9452408AE799E00E94602280916A
:100AC0003E0C882341F060E0812F0E94743A81E05F
:100AD0000E945B5AF4CF90922C0520E030E0A901EF
:100AE000F50160817181828193810F94F1258823C2
:100AF00071F080E090E0A0ECB0E489839A83AB834E
:100B0000BC83BE016F5F7F4FC5010E949E6820E0DD
:100B100030E0A901F60160817181828193810F9497
:100B2000F125882351F18090790C90907A0CA09057
:100B30007B0CB0907C0C80E090E0A0E7B1E4809367
:100B4000790C90937A0CA0937B0CB0937C0C80E092
:100B500090E0A0EAB1E489839A83AB83BC83BE01B1
:100B60006F5F7F4FC6010E949E688092790C9092C1
:100B70007A0CA0927B0CB0927C0C20E030E0A901B2
:100B8000F70160817181828193810F94212F181662
:100B900074F480E090E0A0E4B0E489839A83AB83AE
:100BA000BC83BE016F5F7F4FC7010E949E6880912A
:100BB000010529E131E1882311F029E439E047E515
:100BC00059E061E679E081E00E9493400E946B4029
:100BD00081E00F900F900F900F90DF91CF911F91B8
:100BE0000F91FF90EF90DF90CF90BF90AF909F90CC
:100BF0008F900895CF93C82F8091FD0B83FD14C073
:100C000080911A09811110C080915F029091600259
:100C10009C01215031094091F5115091F611421774
:100C2000530714F40E944D1FCC2329F061E080E0AB
:100C3000CF910C941BBD80911A0991E08927809374
:100C40003C0280913C02882389F08091F3119091BD
:100C5000F4112091F5113091F611821B930B97FF3F
:100C600003C0919581959109029744F410923C023A
:100C70008091FD0B83FF06C0C1E01AC080E00E9496
:100C80005B5ADFCFC0911A09C11112C080915F0277
:100C90009091600201972091F5113091F61128177B
:100CA000390754F70E94534E8BE299E00E94803836
:100CB0008C2FCF910895AF92BF92CF92DF92EF9297
:100CC000FF920F931F93CF93DF93CDB7DEB7649757
:100CD0000FB6F894DEBF0FBECDBF0E94524F87FD06
:100CE000AFC08AE50E94C51E882309F4BAC040E05F
:100CF00050E0BA018AE50E94F5247B018C01209125
:100D0000690230916A0240916B0250916C0260E07E
:100D100070E088EC93E40F94C02C5B016C019701A8
:100D2000A8010F94212F181614F07501860120E0F8
:100D300030E0A901B701C8010F94212F181624F43F
:100D4000E12CF12C00E010E0B701C8010F942D2E2A
:100D5000072E000C880B990B0F94F825698B7A8B62
:100D60008B8B9C8B20E030E0A9010F94F125882328
:100D700021F0CE0141960E941C7380E090E0A0EA31
:100D8000B1E48D879E87AF87B88B19861A861B863C
:100D90001C868CE40E94771E882309F467C00E9499
:100DA000CB246B017C0120E030E0A901C701B60132
:100DB0000F94212F87FF04C0F7FAF094F7F8F0940E
:100DC000CD82DE82EF82F8862091F5113091F61106
:100DD0002430310574F08091F3119091F411821B4D
:100DE000930B97FF03C091958195910901E00497BA
:100DF0000CF400E080E00E94FA85882359F022E09C
:100E0000AE01435F5F4FBE016B5F7F4FCE0109961E
:100E10000E941B8569897A898B899C898B019C0139
:100E2000305809831A832B833C8320E030E0A901EA
:100E30000F94F125882321F0CE0101960E941C73A6
:100E400064960FB6F894DEBF0FBECDBFDF91CF9191
:100E50001F910F91FF90EF90DF90CF90BF90AF90D8
:100E60000895E12CF12C00E211E449CFC090E00597
:100E7000D090E105E090E205F090E30594CF7F92F9
:100E80008F929F92AF92BF92CF92DF92EF92FF929A
:100E90000F931F93CF93DF9300D000D01F921F9228
:100EA000CDB7DEB76C015B014A01722E780100916B
:100EB0002D060E94591F8091F5119091F6118E1503
:100EC0009F051CF4C7010E944D1F80E00E94FA8517
:100ED000882331F0272DA401B501C6010E941B858E
:100EE0001E141F043CF4C7010E944D1F60E080E007
:100EF0000E941BBD81E00E94FA8580E090E0A0E79F
:100F0000B2E489839A83AB83BC8380E090E0A0E85D
:100F1000B0EC8D839E83AF83B887BE016F5F7F4F38
:100F2000CE0105960E949E6887E00E94462A8111A4
:100F300058C08091690290916A02A0916B02B091B1
:100F40006C0240910605509107056091080570916B
:100F50000905C0900205D0900305E0900405F090CB
:100F60000505C0928B07D0928C07E0928D07F09216
:100F70008E0740938F07509390076093910770936B
:100F800092078093930790939407A0939507B0934B
:100F9000960780E090E0A8E4B2E489839A83AB836B
:100FA000BC83CE0101960E94B57280910A05909192
:100FB0000B05A0910C05B0910D05809393079093BC
:100FC0009407A0939507B093960780E090E0A0EA7D
:100FD000B0E489839A83AB83BC83CE0101960E94DF
:100FE000B572C12CD12C80E7E82E82E4F82EC9829C
:100FF000DA82EB82FC8280E090E0A0E8B0E48D83AE
:101000009E83AF83B887BE016F5F7F4FCE01059689
:101010000E949E6820E030E0A90160910E05709169
:101020000F0580911005909111050F94F12587FF10
:101030000BC0C982DA82EB82FC82BE016F5F7F4FF8
:101040008EE095E00E949E6880910E0590910F05BC
:10105000A0911005B091110580936D0290936E02DE
:10106000A0936F02B09370028093970790939807B4
:10107000A0939907B0939A0787E997E00E94D661F9
:101080008091E40581110E9459F761E087EB99E0B6
:101090000E94BB3F80912B11815080932B1140E720
:1010A00058E16FEB79E085E00E942EE380912B11EF
:1010B000882339F00E9454AB80912B11815080938A
:1010C0002B1180E00E9420F90E94DC3180912C11CC
:1010D000823011F40E948E380E94A9E428960FB63F
:1010E000F894DEBF0FBECDBFDF91CF911F910F915E
:1010F000FF90EF90DF90CF90BF90AF909F908F9038
:101100007F900895CF92DF92EF92FF920F931F93FB
:10111000CF93DF9300D01F92CDB7DEB77C016B0178
:101120008A0161E08CE399E00E94BB3F40E758E10F
:1011300063E479E085E00E942EE390912B1181E039
:10114000890F80932B118091391482FF06C08B7F09
:10115000809339149E5F90932B110E94803980E117
:10116000E1E6F2E0A2E0B5E001900D928A95E1F7A8
:101170000E94C56181E00E9420F920E030E0A901D1
:10118000F70160817181828193810F94F125882319
:10119000F1F080911A0981110CC080915F02909149
:1011A000600201972091F3113091F411281739074B
:1011B00074F080E090E0A0E7B2E489839A83AB8387
:1011C000BC83BE016F5F7F4FC7010E949E6887E0AE
:1011D0000E94462A811103C0B6010E94F26720E0F6
:1011E00030E0A901F80160817181828193810F94BF
:1011F000F125882341F080E00E94FA85882319F0C8
:10120000C8010E94CE68129A64E670E080E090E027
:101210000E94392681E00F900F900F900F90DF9180
:10122000CF911F910F91FF90EF90DF90CF90089595
:10123000CF92DF92EF92FF92CF93DF936B017C010D
:10124000D42FC0912C0583E080932C0581E08093FE
:101250003E0CC114D104E104F10431F00E9451FDAF
:10126000C60ED71EE81EF91E80913E0C882389F019
:10127000C114D104E104F10421F48D2F0E945B5AC2
:10128000F3CF0E9451FD6C197D098E099F0997FDCE
:10129000F4CF10923E0CC0932C05DF91CF91FF90BC
:1012A000EF90DF90CF9008950F931F93CF93DF932C
:1012B000C82F162F0E94534EC11194C0CFE8D8E01A
:1012C000CE010E94803861E0812F0E94743A0E9412
:1012D00051FD685370458F4F9F4F6093290670935F
:1012E0002A0680932B0690932C0610922D060091CF
:1012F0002C0583E080932C0530E020E049E151E1AA
:101300006DE179E082E00E9493408DE199E00E94D6
:10131000602281E080933E0C80913E0C882309F48A
:1013200064C060E0812F0E94743A80912D0688236A
:1013300009F454C00E94534E83E099E00E94803823
:1013400030E020E04DEE58E064EF78E082E00E946B
:10135000934084EF98E00E94602241E060E070E0FA
:10136000CB010E94188930E020E050E040E060EEC0
:1013700078E085E00E94934080EE98E00E94E3359B
:101380000E94591F80E00E94FA850E94534ECE01B0
:101390000E9480380E9451FD685370458F4F9F4FC7
:1013A0006093290670932A0680932B0690932C064F
:1013B00010922D0630E020E049E151E164ED78E043
:1013C00082E00E94934083EC98E00E94602281E0DA
:1013D00080933E0C61E0812F0E94743A81E00E946C
:1013E0005B5A9ACFC4EAD8E06BCF00932C05DF910B
:1013F000CF911F910F910895CF92DF92EF92FF92BC
:101400000F931F93CF93DF93CDB7DEB7A0970FB69F
:10141000F894DEBF0FBECDBF0E94524F87FDCCC0F7
:1014200085E40E94771E882309F4D5C00E94CB244E
:101430006B017C0120E030E0A9010F94212F87FF90
:1014400004C0F7FAF094F7F8F094F7FAF094F7F88C
:10145000F094CD8EDE8EEF8EF8A28CE0E4EDF2E01B
:10146000DE01119601900D928A95E1F78AE50E94BE
:10147000C51E882351F040E050E0BA018AE50E9481
:10148000F52469877A878B879C8788E50E94C51E2B
:10149000882351F040E050E0BA0188E50E94F5242D
:1014A00069837A838B839C8389E50E94C51E882388
:1014B00051F040E050E0BA0189E50E94F5246D83C7
:1014C0007E838F83988785E50E94771E882309F4A1
:1014D00089C00E94CB246B017C0120E030E0A9018F
:1014E000C701B6010F94212F87FF04C0F7FAF094CB
:1014F000F7F8F094F7FAF094F7F8F094C98EDA8ED2
:10150000EB8EFC8E1D8A1E8A1F8A188E8CE40E9428
:10151000771E882309F46FC00E94CB246B017C01E5
:1015200020E030E0A901C701B6010F94212F87FF09
:1015300004C0F7FAF094F7F8F094C98ADA8AEB8AD3
:10154000FC8A62E070E082E40E94BC24F82E809164
:101550002B11811131C021E0AE01475E5F4FBE010A
:101560006F5F7F4FCE014D960E948288882321F1C4
:101570006F2D81E00E94548982E50E94C51E882358
:1015800009F442C00E94B82440E050E060EA71E4EF
:101590004D875E876F87788B20912B11222361F016
:1015A0008C012F2DAE01435F5F4FBE016F5E7F4FF9
:1015B000CE0145960E943F87A0960FB6F894DEBFF5
:1015C0000FBECDBFDF91CF911F910F91FF90EF9094
:1015D000DF90CF900895C12CD12C80E8E82E80E4D4
:1015E000F82E33CFC090DC05D090DD05E090DE050D
:1015F000F090DF0572CFC090E005D090E105E0905B
:10160000E205F090E3058CCF90E080E0BDCFCF9273
:10161000DF92EF92FF920F931F93CF93DF93CDB79B
:10162000DEB76C970FB6F894DEBF0FBECDBF8CE46B
:101630000E94771E882309F4B0C00E94CB246B015E
:101640007C0120E030E0A9010F94212F87FF04C026
:10165000F7FAF094F7F8F094F7FAF094F7F8F094BA
:10166000C98EDA8EEB8EFC8E8CE0E4EDF2E0DE01CA
:10167000119601900D928A95E1F788E50E94C51EAA
:101680008823A1F040E050E0BA0188E50E94F524EB
:101690002091E7083091E8084091E9085091EA0864
:1016A0000F94C02C69837A838B839C8389E50E9485
:1016B000C51E8823A1F040E050E0BA0189E50E94F0
:1016C000F5242091E7083091E8084091E90850910D
:1016D000EA080F94C02C6D837E838F8398878AE5F8
:1016E0000E94C51E882351F040E050E0BA018AE50F
:1016F0000E94F52469877A878B879C871D861E86C2
:101700001F86188A80912B11811138C020E0AE010C
:10171000435F5F4FBE016F5F7F4FCE0149960E94CE
:101720008288882359F18091E40581110E9459F73C
:1017300060E080E00E945489898D9A8DAB8DBC8DCC
:10174000B0588D8B9E8BAF8BB88F198A1A8A1B8AE3
:101750001C8A1D861E861F86188A80912B1188235D
:1017600069F010E000E020E0AE014B5E5F4FBE018B
:101770006F5E7F4FCE010D960E943F876C960FB62D
:10178000F894DEBF0FBECDBFDF91CF911F910F91B7
:10179000FF90EF90DF90CF900895C12CD12C80E87E
:1017A000E82E80E4F82E58CF2F923F924F925F920E
:1017B0006F927F928F929F92AF92BF92CF92DF9261
:1017C000EF92FF920F931F93CF93DF93CDB7DEB7C6
:1017D000E5970FB6F894DEBF0FBECDBF8DAB20915D
:1017E0002C052CAB21E020932C0580914A058D34EB
:1017F00009F403C6843511F40C9425A1873409F04B
:1018000091C180914805909149058B31910509F46A
:10181000DDC108F079C18430910508F030C1209114
:1018200000078230910508F48EC1213009F091C182
:1018300011E0029709F010E00E940C2519821A822B
:101840001B821C821D821E821F82188682E50E94D6
:10185000C51E882309F490C10E94CB246B017C0132
:1018600020E030E0A9010F94F125882309F4EAC0B3
:101870004090610250906202609063027090640236
:101880008091650290916602A0916702B091680212
:101890008CA79DA7AEA7BFA780908B0790908C07C1
:1018A000A0908D07B0908E0780918F079091900740
:1018B000A0919107B091920788AB99ABAAABBBAB53
:1018C000A5019401C301B2010F94F12581110DC04E
:1018D00028A939A94AA95BA96CA57DA58EA59FA5B4
:1018E0000F94F125882309F4ADC0A3019201C5012D
:1018F000B4010F94C02C20E030E040E05FE30F948F
:10190000572668A779A78AA79BA72CA53DA54EA512
:101910005FA568A979A98AA99BA90F94C02C20E08A
:1019200030E040E05FE30F9457262B013C0120E0BC
:1019300030E0A901C701B6010F94F125881F88275F
:10194000881F181709F40FC180E090E0A0E8BFEBF2
:101950008CA79DA7AEA7BFA728A539A54AA55BA5BB
:10196000CA01B9010F9457264B015C01A3019201F2
:10197000C301B2010F9457269B01AC01C501B4010C
:101980000F94C12C0F946F2F4B015C01AC019B0194
:10199000C701B6010F94C02C68AB79AB8AAB9BAB87
:1019A000A5019401C701B6010F94C12C9B01AC01A4
:1019B00068A979A98AA99BA90F9457266B017C0174
:1019C00020E030E0A9010F94212F87FDD1C0C7018D
:1019D000B6010F946F2F6B017C01C301B2019058C7
:1019E000A50194010F94BB2D2CA53DA54EA55FA587
:1019F0000F945726A70196010F94572628A539A5BD
:101A00004AA55BA50F94C12C69837A838B839C8341
:101A1000A501940168A579A58AA59BA50F94BB2D66
:101A20002CA53DA54EA55FA50F945726A7019601AD
:101A30000F945726A30192010F94C12C6D837E83CE
:101A40008F83988720E030E0A90169817A818B81BA
:101A50009C810F94F1258111A3C020E030E0A90101
:101A60006D817E818F8198850F94F125811198C0B9
:101A70000E944F4E8BEB9FE00E9480386AC08531F8
:101A8000910509F466C08A31910509F49CC0049758
:101A900009F048C080E50E94C51EC12CD12C7601FA
:101AA000882321F00E9445246B017C0183E50E947C
:101AB000C51E882361F00E94CB2420E030E04AE775
:101AC00054E40F9457260F94342E6B017C010E942E
:101AD000C56180912D11811105C060E081ED9FE00D
:101AE0000E94EE3F0E9451FDC60ED71EE81EF91E51
:101AF0000E9451FD6C197D098E099F0997FF29C02D
:101B000080E00E945B5AF4CF8A32910509F4EAC260
:101B100060F48D31910509F413C208F470C04E973A
:101B200009F466C20E9472F914C08B35910509F45C
:101B3000BCC38C35910509F4BCC38A35910591F776
:101B400010920B0806C0213021F40E940C250E943F
:101B500002703DA9311102C00F94D7148CA9809353
:101B60002C050C94869980E090E0A0E8BFE3F0CECD
:101B7000C12CD12C760131CF89E40E94C51E882367
:101B800031F00E94CB2469837A838B839C838AE41F
:101B90000E94C51E882309F455CF0E94CB244ECF46
:101BA000412FBE016F5F7F4F8BE897E00F942A159E
:101BB0000E9451FD60937E1170937F11809380117C
:101BC00090938111C6CF0E94F177C3CF87E00E9426
:101BD000634E8111BECF8CE0E0EEF2E0DE011196A3
:101BE00001900D928A95E1F770E060E080E50E9437
:101BF0006524BE016F5F7F4F0E94F267AACF87E026
:101C00000E94462A811106C060E08FE40E94A3244E
